:020000040800F2
:10C00000106B0120018002086DA40208B5A202088D
:10C010006BA40208F9940208ADB002080000000009
:10C02000000000000000000000000000BBA50208A6
:10C03000B996020800000000B9A5020859A8020834
:10C040001B8002081B8002081B8002081B8002085C
:10C050001B8002081B8002081B8002081B8002084C
:10C060001B8002081B8002081B80020851950208F1
:10C070001B800208BDC10008A59502081B800208AC
:10C080001B800208E19502081B8002081B80020841
:10C0900011B002081B800208FD9402081B800208F0
:10C0A0001B8002081B8002081B8002081B800208FC
:10C0B000C1A802081B8002081B8002081B8002081E
:10C0C0001B8002081B8002081B8002081B800208DC
:10C0D0001B80020835AF0208A5AF02081B800208CA
:10C0E0001B8002081B8002081B8002081B800208BC
:10C0F0001B8002081B8002081B8002081B800208AC
:10C100001B8002081B8002081B8002081B8002089B
:10C11000FDAE02081B8002081B8002081B8002087B
:10C120001B8002081B8002081D96020879960208EF
:10C130001B8002081B8002081B8002081B8002086B
:10C1400000000000000000000000000000000000EF
:10C150001B8002081B8002081B8002081B8002084B
:10C160001B8002081B8002081B8002081B8002083B
:10C170001B8002081B8002081B8002081B8002082B
:10C180001B800208DFF80CD000F006F800480047DA
:10C1900007790308106B0120064C074D06E0E068A4
:10C1A00040F0010394E8070098471034AC42F6D3FE
:10C1B000FFF7ECFF509E0108709E010810B54FF488
:10C1C0000074204623F0A6FB002819D0204623F057
:10C1D00011FB0C4814F08CFE0B4C802120682EF0D3
:10C1E0000CFD0028F9D1002108482EF001FD0021A6
:10C1F000074823F0E9FABDE8104001201EF00AB913
:10C2000010BD00000CD30020785000200030014009
:10C210003000024002E008C8121F08C1002AFAD10B
:10C2200070477047002001E001C1121F002AFBD1B6
:10C230007047000010B5442107480EF0B0FB002203
:10C24000062106480BF030FF054CA06000F074FB9F
:10C250000020207010BD000000D50020EDC90008AE
:10C26000F8520020F8B5044618F0C2FF0026374DFA
:10C270000746009634B1E068686020460BF0E2FFA4
:10C28000686802E014F03AFE686000690BF0B8FDDF
:10C290006868406908B10BF0B3FD6868C0690BF0CD
:10C2A000AFFD6868006A0BF0ABFD6868016991B189
:10C2B0000BF042FE0CF054FE0CF0A2FC6868B0F8E3
:10C2C0005011D9B30068017CC9071DD0C06840680F
:10C2D000D0B1002413E0A0F85061F8BD011991F825
:10C2E000301151B900F5AC700EF0B0FB696801EB8C
:10C2F000C4010A6B0260496B4160641CA4B26868A7
:10C30000B0F85011A142E9D868684FF4807130301C
:10C310001BF0E7FE6868202100F598701BF0E1FE35
:10C320006868A0F85061384618F05BFF00906868B4
:10C330000068436A13B12A680099984717F022F9F8
:10C340000EF000F8BDE8F84000F002B8705200208E
:10C3500070B5094E0024C4EBC40556F8250008B199
:10C3600017F084F906EB85001C2108F03CFA641CE8
:10C37000E4B2042CEFD370BD1CD600207FB50D466F
:10C38000040003D114F0BAFD04002CD014F02AFEEE
:10C39000002828D094F82800400724D4002605B3AC
:10C3A000ADF80060ADF80260204614F0BFFD401EFD
:10C3B000ADF80400204614F0FFFD401EADF8060065
:10C3C0006A46294602A80DF00AFE00280BD0206814
:10C3D000017C890708D5DDE90001C4E90C010120D1
:10C3E00029E0A4F850617FBD82690AB102A9904793
:10C3F00000250AE004EBC501002202A830310DF04F
:10C4000016FE0028EFD16D1CADB2B4F85001A84261
:10C41000F0D880B2202804D204EBC00002A930304A
:10C4200004E0A4F8506104F13000694605F070F9A9
:10C43000B4F85001401CA4F8500160680028D2D024
:10C440000BF012FF7FBD10B50446006882680AB188
:10C450002146904720680068002801D02060F5E759
:10C4600010BD8068002801D0B0F9160070478068C0
:10C47000002801D0807E8009704770B515460646B9
:10C480000C4651EA05001AD0304608F059FAB06857
:10C4900001232A46018A21440182B068418A294445
:10C4A0004182214630460AF041FB00220B213046F2
:10C4B00014F016FE012803D130460AF091FA01204B
:10C4C00070BD77B581B00E46050017D0622209F025
:10C4D0008AFE040012D0206880B1284631466322CB
:10C4E00009F081FE10F0FF0208D02368204603996E
:10C4F00098470090BDF80000ADF80C00039804B018
:10C5000070BD00002DE9F047054692B0408C1A9CA2
:10C5100040F00800688490462A8499468A46228919
:10C52000284609F060FE0646A5F82090228951466B
:10C53000284609F058FE0746688CBE4220F00800E5
:10C54000688403D13104B1EB074F68D0A5F820808F
:10C5500022895146284609F046FE06468046A5F83F
:10C5600020905146284604F094FC21890068324608
:10C5700018F032FA20890B2823D147F6FF794E456F
:10C5800001D04F451DD1284609F079FF00EBD0704E
:10C590004610284609F067F800EBD0704010C845F7
:10C5A00006D1711C431C994200DA00E01946884606
:10C5B0004F4506D1711C421C914201DA0F4600E042
:10C5C000174619480EF0F3F906002BD03560C6E97E
:10C5D00003872089B0806846C6F808A004F0D8FF19
:10C5E0001248FF21CDE900601148029011480390E4
:10C5F00000200890CDE9090120880B9060889DF803
:10C60000421040420C90E0680790002060F3000167
:10C610008DF8421020690690684605F029F812B09E
:10C62000BDE8F087FEE7000024D5002071980108DE
:10C63000759A0108CD990108142101480EF0AFB98F
:10C6400024D500202DE9F84F00249046894606465F
:10C6500025464FF0040AE3E0F1680AEBC5000858EC
:10C6600082017AD480B230EA090210D0002230EA86
:10C6700008000ED0002082426FD051F835706A4613
:10C680001021384617F0A4FF002871D103E00122E1
:10C69000EDE70120EFE76A461121384617F098FFD1
:10C6A000002865D16A461221384617F091FF00280C
:10C6B0005ED16A461321384617F08AFF002857D109
:10C6C0006A461521384617F083FF002850D16A4684
:10C6D0001421384617F07CFFF0BB6A460A21384621
:10C6E00017F076FFC0BB6A466B21384617F070FF23
:10C6F00090BB6A466C21384617F06AFF60BB6A46F9
:10C700000121384617F064FF30BB6A4604213846E1
:10C7100017F05EFF00BB6A460221384617F058FF4B
:10C72000D0B96A460321384617F052FFA0B96A46CD
:10C730000521384617F04CFF70B96A460621384685
:10C7400017F046FF40B96A463221384617F040FFDD
:10C7500010B96A466E2101E00AE060E0384617F041
:10C7600037FF28B96A466D21384617F031FF10B1FE
:10C770000320BDE8F88F6A466921384617F028FF84
:10C78000F0BB6A466A21384617F022FFC0BB6A46F2
:10C790006E21384617F01CFF90BB6A466D21384663
:10C7A00017F016FF60BB6A463721384617F010FFB6
:10C7B00030BB6A463821384617F00AFF00BB6A468C
:10C7C0003521384617F004FFD0B96A464021384673
:10C7D00017F0FEFEA0B96A464521384617F0F8FE6C
:10C7E00070B96A464121384617F0F2FE40B96A46F0
:10C7F0004221384617F0ECFE10B96A46432100E0AA
:10C8000009E0384617F0E4FE28B96A46492138465F
:10C8100017F0DEFE08B1022401E004B901246D1C0A
:10C82000708CC0F30510A8423FF616AF2046A0E773
:10C8300001484068704700007052002070470000B7
:10C8400010B5182103480EF0AAF80349012008701A
:10C8500010BD0000D0D40020405300202DE9F84F37
:10C860008146407A0D4600F00700022819D0104694
:10C870008046954200DD2A46164603202A4F2B4B60
:10C8800000EB460020F00304B86819681034411A20
:10C890007A6804EB010C944505D2416821F000410F
:10C8A00024E00846E4E7944219D89A464FF0FF3B4B
:10C8B00008197968884210D9002269461C48CDF8C9
:10C8C00000B004F05BFB002269461A4804F056FBF6
:10C8D000B968DAF80000091AEAE7B868DDE7204627
:10C8E00016F038FEC0B1416841F0004188EA6502A7
:10C8F000416089EA02010160416801F04041491C40
:10C9000031F0804141608681A0F80E8005D500F1AC
:10C9100010018160BDE8F88FFEE7B96801F11002EF
:10C9200021448260B960F5E778520020205300204E
:10C93000430A0108F90F010810B5084C01202070C6
:10C9400007480EF00FF80028A06803D0BDE810409B
:10C950000BF08ABCBDE810400BF074BCF85200200C
:10C9600000D5002010B5044690F84200A16B820764
:10C9700009D4B4F840204AB1A2F57F43FF3B1BD055
:10C98000521EA4F84020B4F84020AAB909B1820789
:10C9900012D5214614480EF080F8FFF7CDFFE1686C
:10C9A00009B120468847216909B1204688472046B9
:10C9B000BDE8104016F05ABEE26B524222630029D5
:10C9C00011D0820702D4626B524222634210521C81
:10C9D00062F3410084F84200A26A206A2262A062E7
:10C9E000E06AE162A06310BD00D5002070B5304E52
:10C9F000706818F0F6FB0546707880F001007070E2
:10CA000047E00020307094F842007178C0F3800253
:10CA10008A4242D061F3820084F84200216B4A19B5
:10CA2000030719D4002917DC002A15DBC00709D138
:10CA3000616939B120468847216A01442162A16AAF
:10CA40000844A062A16809B12046884794F84200D2
:10CA500040F0080084F84200206B4019206316D48F
:10CA6000E16A884200DD2163E1692046884701468A
:10CA7000606A884204D0616262680AB120689047A7
:10CA8000D4E90B01814202DB2046FFF76BFF3078CF
:10CA900018B108480DF066FF03E0214605480DF087
:10CAA00073FF0400ADD118F0A3FB706070BD0000EF
:10CAB000F852002000D500202DE9FF4F8BB01E4614
:10CAC000DDE91801CDE90601002004901F981E9DA4
:10CAD000042809D0052809D006280CD014287CD1B8
:10CAE00001200290022004E00020FAE701200290D9
:10CAF0000320059008E00120029002200590FFF736
:10CB000097FE0068806B04900D98002416FB00F0DF
:10CB10000A900C98401E09900D98401E08902CE138
:10CB20001A980699604301EB20231B9807996043EC
:10CB300001EB202219124FEA222007D40C9FB942A0
:10CB400004DA002802DB0D9FB84201DB002011E16E
:10CB5000DBB2D2B2802B05DAC3F17F034FF0FF378F
:10CB60005B0003E001275B00A3F580739A46802AEF
:10CB700005DAC2F17F024FF0FF33520003E00123D8
:10CB80005200A2F58072914600FB0618DDF814C031
:10CB90000B9A08FB0C2201EB070C5FEA0C0E73D416
:10CBA000DDF82480C6456FDC10EB03086CD4DDF89B
:10CBB00020C0E04568DCDDF814C017FB0C2B13FB2C
:10CBC00006F707FB0C23029FF7B31F9F052F05D025
:10CBD000142F09D0062F47D053E0D2E092F802C0BC
:10CBE00099789BF8020010E0DDE90A7C0CEB47071E
:10CBF000394400FB06FC00FB067708FB06F81CF82E
:10CC000001C017F80E0018F80110614507D011FB9C
:10CC100009F7C9F580711CFB0171C1F3072160455B
:10CC200007D010FB0AF7CAF580701CFB0070C0F338
:10CC3000072008444008285556D01078517800EB5A
:10CC40000120ADF8000000E01FE01878597800EBF3
:10CC50000120ADF80C009BF800109BF8010001EBDF
:10CC60000020ADF804001CE00498118880B28142D5
:10CC70003FF46CAF19888142FAD0BBF800108142B2
:10CC8000F6D0FF210846D4E72FE01088ADF8000069
:10CC9000BBF80000ADF804001888ADF80C00FF20C8
:10CCA0002855BDF80000BDF80C10884203D1BDF82E
:10CCB0000410884212D009F0FF020099039804F092
:10CCC0008BFE0390DDE900100AF0FF0204F084FE01
:10CCD0007F220190039904F07FFE00901D98BDF81B
:10CCE000001000EB4400018045E092F800C092F88B
:10CCF00001800CEB082C1FFA8CF8DDF874C02CF8BE
:10CD00001480DDF87CC0BCF1050F06D0BCF1060F25
:10CD100005D0BCF1140F08D109E092780FE0049A15
:10CD200092B2904501D1002209E0FF2207E00B9A60
:10CD300000FB062C0A9A01EB42021CF8022009B9FA
:10CD4000002F05DBDDF824C0614504D1002F02DD92
:10CD5000CAF1FF000BE008B9002B06DB08998842F6
:10CD60007FF4F4AE002B7FF7F1AEC9F1FF0010FBAA
:10CD700002F0000A2855641C24B21C988442FFF675
:10CD8000CFAE0FB0BDE8F08F2DE9F05F00228046F6
:10CD900011460AF067FD0021404609F08CF904466F
:10CDA0000021404609F013FA204407B20021404612
:10CDB00009F0E9F920440FFA80FB404609F024F914
:10CDC000C11901EB0B000FFA80F9274C404608F01F
:10CDD00097FB824600252BE0D8F80800234900681D
:10CDE00050F82560304609F070FB00BB304609F072
:10CDF0004FFE60BB0021304609F02AF938B3012804
:10CE000025D0022823D0032821D00021304609F064
:10CE10007DFA60B906F11400064604F0A6FC384419
:10CE2000A04203DB304604F0A0FCC41924B26D1C00
:10CE30005545D1D341F6FF70C44212D004EB0B002C
:10CE400000B24946484500DC0846BDE8F09FB6F907
:10CE50001A10B8F91600081A411CA142E6DB0C466C
:10CE6000E4E74846F1E7000001E0FFFF01000400AD
:10CE70002DE9F05F0022054611460AF0DDFC002195
:10CE8000284609F018F904460021284609F093F9CC
:10CE900020440FFA80F90021284609F080F9204447
:10CEA0000FFA80F8284609F0BDF800EB080101EB05
:10CEB00009000FFA80FB4B4C284608F021FB824604
:10CEC0000021284609F0CAF801284FF000062CD0AE
:10CED0006AE0A8684449006850F82670384609F0AE
:10CEE000F4FA08BB384609F0D3FD38BB00213846B8
:10CEF00009F0AEF810B3032820D006281ED0082869
:10CF00001CD00021384609F0FBF968B907F114007C
:10CF1000074604F048FC4844A04204DB384604F0CD
:10CF200042FC00EB090424B2761C5645D1D341F6ED
:10CF3000FF70C44241D004EB08003DE0B5F9180091
:10CF4000B7F91410401A411CA142ECDB0C46EAE789
:10CF5000A8682549006850F82670384609F0B5FAE7
:10CF600008BB384609F094FD88BB0021384609F01B
:10CF70006FF860B301282BD0042829D0072827D0C8
:10CF80000021384609F0C2F968B907F114000746D4
:10CF900004F009FC4044A04204DB384604F003FCE2
:10CFA00000EB080424B2761C5645D1D341F6FF703D
:10CFB000C44202D004EB090004B241F6FF70C4423F
:10CFC000584602D05C4500DD2046BDE8F09FFFE7F3
:10CFD000B7F91800B5F91410401A411CA142E1DB61
:10CFE0000C46DFE701E0FFFF010004001CB50B88E1
:10CFF00004892344ADF800304B8844892344ADF8BC
:10D0000002308B8804892344ADF80430C9884389F1
:10D010001944ADF806104369694698471CBD2DE9CF
:10D02000F04F8BB05FEA010A054643D0A5F818A07F
:10D03000286808B116F01AFB0AEB4A00062101EB3A
:10D04000400016F087FA286058B3022202EB4A012A
:10D0500001440422E96002EB8A010144C5E90101AF
:10D0600001210024BAF1010F1CD04FEACA00083098
:10D0700016F09EFA064600EB8A074FEA8A0000B2D5
:10D08000ADF80000C0F101022146ADF80240801069
:10D09000A146A346ADF824204C463F1D01910590C2
:10D0A000B3E0FEE7B4220270E8680480E8684180DB
:10D0B000A86804800BB0BDE8F08F4FF00008BDF900
:10D0C0002400002808DCBDF80210032202EB410115
:10D0D0000844ADF824000DE0BDF80220BDF80010B2
:10D0E0000523521A03EB42021044491EADF82400F6
:10D0F000ADF80010BDF80200401CADF80200684613
:10D1000000F0F0F878B1BDF9000005AB821043F8EB
:10D11000282001AA00F0030142F8281008F10108B4
:10D12000B8F1040FCBDBB8F1040F74D1089905985E
:10D13000884212D126F8140027F81490DDE9010185
:10D140000844DDE903121144084469680855696818
:10D1500000010855641C24B255E00699884219D094
:10D1600026F8140027F814906A68019810556A6828
:10D1700000011055641C059A20B2521E26F810209A
:10D1800027F81090DDE902120A440499091D1144A0
:10D190006A6832E0079926F814008842494627F861
:10D1A000149015D0DDE9012010446A6810556A68B2
:10D1B00000011055641C059A20B2521E26F810205A
:10D1C00027F81010DDE90312114408316A6814E0F1
:10D1D000DDE901021044039A10446A6810556A6838
:10D1E00000011055641C059A20B2521E26F810202A
:10D1F00027F8101004996A680C3111546A68090103
:10D200001154401C04B209F10109684600F06AF8A3
:10D2100000287FF452AF40F2D3211AFB01F106EB54
:10D220004402881232F9022C824205D107EB4402F3
:10D2300032F9022C82421AD0A1EB8021B1F5007F95
:10D2400003DC494341F3CF3106E0C1F58061494336
:10D2500041F3CF31C1F10F0126F8140027F8140073
:10D2600068680155686809010155641C24B2A01E54
:10D270000DE037F8101026F8141036F8101027F8C3
:10D28000141069680A5C0A55641C24B2401E002808
:10D29000EFDAEB6800210846A3F800B01CE0EA686A
:10D2A00022F81100AB6836F8102023F811200BE0AB
:10D2B000D5F808C036F910303CF811209A4200DB4E
:10D2C0001A462CF81120401C37F910208A4201D14F
:10D2D000A042EDDB491C09B2A042E0DB304616F06B
:10D2E000B3F9E7E6B0F90210B0F90000814201DCC1
:10D2F000012070470020704717B581B0022ABDF8A1
:10D30000080036D9BDF80410C0F3C403C1F3C40447
:10D3100023441F2B00D31F2363F3C70143079B0E36
:10D3200003EB503301F0070403EBC40303EB513369
:10D33000ADF804103F2B00D33F23DC0864F3020157
:10D3400063F34F31C0F30420C1F304231844ADF854
:10D3500004101F2800D31F2060F30C21ADF8041027
:10D36000FF2A08D0DDE9010104F010FB0090BDF8B0
:10D37000000004B010BD88B2FBE717B581B0022AE7
:10D3800003D8BDF8080004B010BDBDF80410BDF806
:10D390000800C1F3C403C0F3C40413FB04F35B0926
:10D3A00063F3C701C1F30423C0F3042413FB04F3A4
:10D3B0005B0963F30C214B079B0E4407A40E03EBA0
:10D3C000513304EB503013FB00F35B0A63F30201AB
:10D3D0004B079B0E03EB513313FB00F0800960F306
:10D3E0004F31ADF80410FF2A07D0DDE9010104F048
:10D3F000CDFA0090BDF80000C5E788B2C3E717B5C5
:10D4000081B0022ABDF8080036D9BDF80410C0F377
:10D41000C403C1F3C4041B1B002B00DC002363F313
:10D42000C70143079B0E03EB503301F0070403EBE6
:10D43000C40303EB5133ADF80410002B00DC0023D0
:10D44000DC0864F3020163F34F31C0F30420C1F33D
:10D450000423C01AADF80410002800DC002060F39B
:10D460000C21ADF80410FF2A08D0DDE9010104F019
:10D470008DFA0090BDF8000004B010BD88B2FBE743
:10D480002DE9FF4F83B00746DDF84080DDE91365E5
:10D490004FEA4800DDF848A000B2049C0190BAF1C0
:10D4A000040F1DD0BAF1060F1AD0BAF1050F5AD0E9
:10D4B000BAF1140F54D1B7F90010B7F9022008FBE4
:10D4C000021004EB4009384604F061F983463846FF
:10D4D00004F081F9044640004FF0000A009084E017
:10D4E000384612F05EFD014600902846FF221AF0F1
:10D4F000F1FDB7F90010B7F9022008FB021004EBA8
:10D500004008384604F067F98346400002903446EC
:10D51000B7F902000BE020464146029A1AF0B9FD25
:10D52000019909F10100884404EB4B0400B2B7F9FA
:10D53000061081464945EEDABAF1060F10D14EF2D7
:10D5400007000021ADF804000246084605E036F861
:10D550001030934200D12954401C009B9842F6D3CE
:10D5600007B0BDE8F08FB7F90010B7F9022008FB4B
:10D57000021000EB40000444384604F02CF9A8EBFC
:10D58000000000EB40000FFA80F8384604F0FFF886
:10D590008146384604F01FF90146002215E00020BC
:10D5A0000BE0A3782B5414F8013B14F8027B03EB37
:10D5B000072326F81030401C00B28842F1DB521CD1
:10D5C00006EB41060D44444412B24A45E7DBC7E787
:10D5D00030464946009A1AF05CFD01990AF10100B3
:10D5E00006EB440689440FFA80FADA45F0DBDDE900
:10D5F00004014A000699B7F9023002FB0100B7F9AD
:10D60000002008FB03210E18002708E028463146B9
:10D6100022461AF03EFD7F1C254446443FB25F453A
:10D62000F4DB9DE72DE9F04F0646C87A89B0154630
:10D630000F46022803D8012009B0BDE8F08F184634
:10D640003A69B9680CF042FF041EF5D0207D00F065
:10D650001F0007F053F84FF4807808B1062010E05F
:10D66000207D00F01F000E2806D0142809D007F0F6
:10D6700035F840B1052004E038884FF00E0938B97C
:10D6800003E0814608E00420FBE77888404503D0AA
:10D6900000204FF00509A061226A22B129463046D8
:10D6A0000CF0BFF8B7E0A069F0B3294602A804F077
:10D6B00038F8B7F9003013B97888404529D0A888E0
:10D6C00029886A88401A401C01B2E88807F1040CD6
:10D6D000801A401C02B27888CDE9000C02A80CF038
:10D6E0003FFEBDF8080029880844ADF80800BDF8E1
:10D6F0000A0069880844ADF80A00BDF80C002988C2
:10D700000844ADF80C00BDF80E0069880844ADF877
:10D710000E0002AA04A8B1680CF061FC00287AD0BF
:10D7200004A8D6F8088000E00BE0B060CDF80090C7
:10D730002A4639463046A36904F0DAFBC6F8088069
:10D7400069E02A4603A8B1680CF049FCF0B3BDF8C3
:10D750001000BDF80C10401A401C0FFA80FA0AEBBA
:10D760004A0015F025FF059003A901A8D6F808B0D6
:10D7700003F0D7FF012101A812F060FCBDF90C00F5
:10D78000B5F90010401A0890BDF90E80B5F90200F5
:10D79000A8EB000536E001AA594606A80CF01FFCCC
:10D7A00070B3059800900898534601B22AB22046FB
:10D7B00014F038FE01280ED0204614F088FD05989C
:10D7C00015F042FF204614F082FD00E023E0002027
:10D7D000C6F808B030E706A8B060CDF8009001AAFE
:10D7E00039463046059B04F083FBBDF80600401C1B
:10D7F000ADF80600BDF80A00401CADF80A006D1C2B
:10D8000008F10108BDF912004045C4DAC6F808B0B5
:10D81000059815F019FF204614F059FD0BE700009C
:10D820001CB50C4814460078002812D088880A8855
:10D830004B88801A401C82B2C888C01A401C83B230
:10D8400050005843CDE900404C88088821461BF021
:10D8500064FF1CBD345200202DE9F74FC87898B002
:10D860000C4602287ED911460AA803F075FFB4F9C8
:10D870002000012829DD94F82200FD2825D32088E6
:10D8800018B394F82300BDF828104008C0F38002B4
:10D890001144ADF82810BDF82A10C0F34000084428
:10D8A000ADF82A0094F82310BDF82C004908C1F304
:10D8B000C001401AADF82C0094F82310BDF82E00DA
:10D8C000C1F34001401AADF82E0018980AA98268E9
:10D8D0000CA80CF084FB00287ED0E07B10F007053C
:10D8E00019D0E088ADF80000BDF8000061898842D9
:10D8F00000D100250AA805F055F807461C2103A809
:10D900001AF0EFFBA0788DF82500BDF80000ADF807
:10D9100014001FB105E060680090E5E7208800B9B9
:10D92000F5B3E078FD2800D3FF2083460AA803F072
:10D930005EFF81460AA803F030FF06464846B1451F
:10D9400000DB3046B4F90010B1EB600F00DB411092
:10D9500088460CA803F04BFF82464FF0FF3016902C
:10D96000002000E038E00090B8F1000F00DC77B153
:10D97000504615F01DFE0090002342460AA90EA84D
:10D9800005F07AFA00210EA804F01CFE1690BDF8EE
:10D990003000ADF80400BDF83400ADF8080000E038
:10D9A00011E00098069001A803900890FF208DF8E0
:10D9B000240032464946A01D06F00EFE060018D08F
:10D9C000022D0CD015E00AA80390E0788DF8240011
:10D9D00003A9189805F00FFD1BB0BDE8F08FBDF945
:10D9E0003010B06800EB4100BDF92810A0EB4100F9
:10D9F00004907FB3BDF9324027E027B2ADF806703E
:10DA0000ADF80A7052465946009806F0E7FEBDF997
:10DA1000301053463A46009804F086FF8DF81C00FB
:10DA2000012802D102208DF81C00012D08D1BDF97A
:10DA30002A10B068611A00EB41000088ADF81400AC
:10DA400003A9189805F0D7FC641CBDF93600A04264
:10DA5000D3DABCE0FFE7002054E0BDF82A1001EB68
:10DA60000900BDF82E1004B2A1EB090007B2BDF900
:10DA70003200A04203DDBDF93600B84240DB524619
:10DA80005946009806F0AAFEBDF9041053462246F6
:10DA9000009804F049FF8DF81C00012802D10220F3
:10DAA0008DF81C00BDF93200A04212DCADF8064032
:10DAB000ADF80A40012D08D1BDF92A10B068611AED
:10DAC00000EB41000088ADF8140003A9189805F098
:10DAD00092FCBDF93600B84212DBADF80670ADF825
:10DAE0000A70012D08D1BDF92A10B068791A00EB2F
:10DAF00041000088ADF8140003A9189805F07BFCDC
:10DB000009F1010081464045A7DBBDF82800ADF8CA
:10DB10005000BDF82C00BDF82A10ADF8540001EB00
:10DB20000800BDF82E10ADF85200A1EB0800ADF8CA
:10DB3000560014A804F036FF074628430DD0BDF95F
:10DB40002E100120A1EB0809BDF92A108DF824B090
:10DB50008DF81C0001EB080437E0BDF82A108DF8A1
:10DB600024B001EB0800ADF80600BDF82E10A1EBC3
:10DB70000800ADF80A000020069003A9189805F0E7
:10DB80003AFC24E06FB152465946009806F026FE52
:10DB9000BDF93010534622B2009804F0C5FE8DF84E
:10DBA0001C00ADF80640ADF80A40012D08D1BDF9C2
:10DBB0002A10B068611A00EB41000088ADF814002B
:10DBC00003A9189805F017FC641C4C45DADD009891
:10DBD00008B115F039FD1698401C05D0169805F0CF
:10DBE000F5F90EA804F0C2FE002E3FF4F5AE304663
:10DBF00006F0EBFCF0E62DE9F0410646086990B02E
:10DC000015460C4600287DD0A07E02287AD92946E8
:10DC10000DA8B2680CF0E3F9002873D00DA8D6F86F
:10DC20000880B060206906F071FD022806D001A9C5
:10DC3000206914F06DFB012849D0C9E0002741F6A6
:10DC4000FF70CDE900700297D4E904123B460FA89B
:10DC500017F0B8FC284603F0CAFD01462A88BDF932
:10DC60003C0001EBD17102EB610100EBD072A1EB42
:10DC700062010844401EADF83000ADF82C10284673
:10DC800003F08BFD01466A88BDF93E0001EBD171BE
:10DC900002EB610100EBD072A1EB62010844401E6F
:10DCA000ADF83200ADF82E1003A804F0D7FB606980
:10DCB0000390208BADF81800A07E8DF82600009709
:10DCC0000BAA03A93046236904F034F980E004A8C4
:10DCD00004F016F9A0788DF81C00208BADF8180020
:10DCE000E07E8DF81A00A07E8DF81B00207F4FF09B
:10DCF000FF3740B101996888ADF80A0007EB515130
:10DD000008445DE066E0284603F071FD298800EBD9
:10DD1000D07001EB60000199C1F38A21A0EB5100A2
:10DD2000ADF80800284603F038FD698800EBD07094
:10DD300001EB60010198A1EB9051C0F38A22ADF88C
:10DD40000A10BDF80830521E1A4407EB5050ADF8C7
:10DD50000C200844ADF80E0002AA04A9304623693D
:10DD600004F09AF834E001992888C1F38A21ADF8CB
:10DD70000800491E084410E002AA04A9304623699D
:10DD800004F08AF80198BDF80810C0F38A20014415
:10DD9000ADF80810BDF80C100844ADF80C00BDF942
:10DDA0000800B5F904108842E6DDBDF80A100198B4
:10DDB00001EB5051ADF80A10BDF80E1001EB5050B8
:10DDC000ADF80E00BDF90A00B5F906108842CADDAB
:10DDD000C6F8088010B0BDE8F0812DE9F04180461A
:10DDE00091F8220086B00C461646022868D9208C8D
:10DDF000002865D094F8230010F03E0F60D0C007D3
:10DE00005ED1104603F0F3FC0746304603F0C5FC34
:10DE1000B4F90050874200DA3846B5EB600F00DDF8
:10DE20004510314604A803F097FC94F82300BDF98F
:10DE30001020C0F344014807B4F9200001D428445D
:10DE400040421044ADF810000807BDF91420B4F9A1
:10DE5000200001D428444042101AADF8140094F870
:10DE60002300BDF9121040088007B4F9200001D446
:10DE7000284440420844ADF8120094F82300BDF94C
:10DE800016104008C007B4F9200001D128444042D0
:10DE9000081AADF81600208C281A01B2002900DA01
:10DEA0000021A27894F82200CDE90202E08BADF8BF
:10DEB000040000912B4604AA3146404600F003F8C6
:10DEC00006B0BDE8F0812DE9FF4FA3B01F46DDE9A4
:10DED000326ADDF8C08015460C46FF2E00D3FF26BF
:10DEE000084604F05FFD8146384350EA08006DD0D3
:10DEF00023982146826803A80CF071F800286CD0A2
:10DF000003A803F074FC02901C2108A806F06FFC23
:10DF1000029815F04DFB0B904FF0FF300090002F52
:10DF20000ADD00233A46214616A804F0A5FF002189
:10DF300016A804F047FB00900123424629461CA87E
:10DF400004F09AFF00211CA804F03CFB01900FA8EC
:10DF500008900D90BDF8C4008DF83860ADF8280029
:10DF60008DF839A0B4F90000B5F9001038448842A2
:10DF700000DC0846ADF85000B4F90400B5F904100F
:10DF8000C01B884200DB0846ADF85400B4F902001B
:10DF9000B5F902103844884200DC0846ADF852005A
:10DFA000B4F90600B5F90610C01B884200DB08462C
:10DFB000ADF8560014A803F01AFC0146B4F90200AB
:10DFC000B5F9022090420BDC01200AE000962A46B7
:10DFD0002146319B239800F0D0F927B0BDE8F08F9F
:10DFE00000208046B4F90600B5F90620904201DB16
:10DFF000012600E00026B9F1000F44D0BDF80C0066
:10E00000ADF83C00BDF81000ADF84000BDF90E4081
:10E0100022E0B8F1000F03D1BDF95200A0421ADC92
:10E020001EB9BDF95600A0421ADB25B2ADF8425028
:10E03000ADF83E5002990B9806F0DEFBBDF90C10CE
:10E040002A46029B0B9804F06FFC8DF8300008A95B
:10E05000239805F0D0F9641CBDF91200A042D8DA6B
:10E060001CA804F083FC019804F0B0FF0098401C49
:10E0700005D016A804F07AFC009804F0A7FF0B98CE
:10E0800015F0E2FAA9E7B4F90000B5F900209042D2
:10E0900001DC012000E000208146B4F90400B5F95C
:10E0A0000420904201DB012000E00020824609EAC2
:10E0B0000A0202EA08024FF0010B324203D0322971
:10E0C00001DA4FF0000B01208DF8300018EA0B0F39
:10E0D00012D0BDF85000ADF83C00BDF85400ADF8CA
:10E0E00040006088ADF83E00688808A9401EADF881
:10E0F0004200239805F07FF916EA0B0F12D0BDF805
:10E100005000ADF83C00BDF85400ADF84000E88880
:10E1100008A9401CADF83E00E088ADF84200239805
:10E1200005F069F9B9F1000F12D02088ADF83C0074
:10E13000288808A9401EADF84000BDF85200ADF88F
:10E140003E00BDF85600ADF84200239805F053F9A3
:10E15000BAF1000F12D0A88808A9401CADF83C0005
:10E16000A088ADF84000BDF85200ADF83E00BDF803
:10E170005600ADF84200239805F03DF9BDF80C00BB
:10E18000BBF1000FADF83C0008D0BDF95000BDF95F
:10E190001010421E914248DA084647E0BDF81000D0
:10E1A000ADF84000B5F90200B4F90210401AB842C7
:10E1B00000DB07460FFA87F8002533E06088284423
:10E1C00006B2E088401B07B2BDF90E00B04203DD85
:10E1D000BDF91200B84224DB02990B9806F00CFB43
:10E1E000BDF93C103246029B0B9804F09DFB8DF864
:10E1F0003000BDF90E00B04207DCADF83E60ADF86E
:10E20000426008A9239805F0F6F8BDF91200B8425B
:10E2100007DBADF83E70ADF8427008A9239805F011
:10E22000EAF86D1C4545C9DBA0E0401EADF8400092
:10E230000FA803F0DCFA051E41DD59EA08001DD0E5
:10E24000BDF90E4016E027B2ADF84270ADF83E7051
:10E2500029460B9806F0D0FABDF93C102B463A46F9
:10E260000B9804F061FB8DF8300008A9239805F0A5
:10E27000C2F8641CBDF95200A042E4DC59EA060071
:10E280001DD0BDF9564015E027B2ADF84270ADF88B
:10E290003E7029460B9806F0AFFABDF93C102B46AC
:10E2A0003A460B9804F040FB8DF8300008A92398FB
:10E2B00005F0A1F8BDF91200641CA042E4DABDF932
:10E2C0005400BDF90C10421C914201DD084600E0EB
:10E2D000401CADF83C00BDF81000ADF840000FA8A0
:10E2E00003F085FA051E41DD5AEA08001DD0BDF98C
:10E2F0000E4016E027B2ADF84270ADF83E702946E8
:10E300000B9806F079FABDF93C102B463A460B986B
:10E3100004F00AFB8DF8300008A9239805F06BF88B
:10E32000641CBDF95200A042E4DC5AEA06001DD08C
:10E33000BDF9564015E026B2ADF84260ADF83E603A
:10E3400029460B9806F058FABDF93C102B46324688
:10E350000B9804F0E9FA8DF8300008A9239805F02D
:10E360004AF8BDF91200641CA042E4DA1CA804F0CB
:10E37000FDFA019804F02AFE7BE62DE9FF478AB0FA
:10E380000C46824615461C216846169E06F02FFA5A
:10E3900007A80090BDF83400ADF808008DF81860AB
:10E3A000B4F90200B5F90210884201DC012700E04F
:10E3B0000027B4F90600B5F90610884201DB0126F2
:10E3C00000E00026B4F90000B5F90010884201DC35
:10E3D000012100E000218846B4F90410B5F90420B9
:10E3E000914201DB012100E00021ADF81C00A08872
:10E3F000ADF820006088ADF81E0068888946401E90
:10E40000ADF822001FB16946504604F0F4FFE888D9
:10E41000401CADF81E00E088ADF822001EB1694630
:10E42000504604F0E8FF2088ADF81C002888401E04
:10E43000ADF8200017B1B5F9020001E0B4F902000F
:10E44000ADF81E0016B1B5F9060001E0B4F90600FA
:10E45000ADF82200B8F1000F03D06946504604F031
:10E46000CAFFA888401CADF81C00A088ADF82000A9
:10E47000B9F1000F03D06946504604F0BCFF0EB05E
:10E48000BDE8F0872DE9F0412F4F0646786812F07D
:10E4900049FD04463068C56B696B09B12846884759
:10E4A000786800680188408811FB00F0E1688842C4
:10E4B00001D1012000E00020216859B1616849B113
:10E4C00028B107E078680068816A01B1884720694F
:10E4D0000028F7D10121216178680068C06882694D
:10E4E000D20704D08069800701D5616101E0002076
:10E4F0006061606908B1012700E000273068416968
:10E5000071B1016911F0300F06D0490704D5D5E982
:10E51000001000F01BF803E0D5E90021FEF766FDCE
:10E52000206800280BD06168002908D03268127C6E
:10E53000BA43D20703D1A268824202D1A160BDE8EA
:10E54000F081A060FBE70000705200202DE9F34F3E
:10E550000446854887B041680D682869820701D55F
:10E5600042076FD4C0F30110022829D0012801D03E
:10E57000032867D100200090084612F0D3FC8346A0
:10E58000204603F016F90646204603F0F4F84FF44F
:10E59000A051B1FBF6F20190824201DAB1FBF6F034
:10E5A0000390B4F902000290287CC0F30110012806
:10E5B00013D020886080711E0844E0800027C4E0EA
:10E5C00021462846089A00F0DBF8089A09B021464F
:10E5D0002846BDE8F04FFEF709BD68882188401A3B
:10E5E000401EE080801B401C6080E7E70399C01B51
:10E5F000884200DD08460FFA80F90120CBF81000B0
:10E600000FBB0198B0421EDB287CB146C0F301105D
:10E61000032810D000204946089A00F0E5F8287C2D
:10E62000C0F30110012808D029880298081A401E5A
:10E63000A080801B54E00120EDE702982080029822
:10E64000304463E08DE0009820B94FF4205014F07E
:10E65000AFFF0090287CC0F3011003281AD00020DF
:10E660008646DDF820C000984946069016FB01F06A
:10E67000401E0590701E4843049000208246884248
:10E6800021DA0498BEF1000F504401D0059A101A07
:10E69000002212E00120E3E7069BBEF1000F03EB2E
:10E6A000400863460CF1020C1B88A8F8003001D02A
:10E6B000084400E0401A521C12B2B242ECDB0AF1EC
:10E6C000010000B2DAE7287CC0F30110012819D05C
:10E6D00029880298081AC01B401EA080A0EB0900E0
:10E6E000401C208001984F44874212DBDBF8180061
:10E6F000C0070ED0DBF8180080070AD50120CBF840
:10E70000140009E00298384420804844401EA0804C
:10E71000E8E70021CBF81410009828B10246214602
:10E720002846FEF763FC05E0089AF8E7A96A09B1F4
:10E7300028468847DBF810000028F7D1089906FB27
:10E7400009F001EB40003FB2089001988742FFF6C4
:10E750004DAF0098002804D009B0BDE8F04F14F088
:10E7600073BF09B0BDE8F08F7052002030B5048847
:10E770000D88058010880880188810801C8030BDA6
:10E78000F8B5054616460C46084603F012F807464B
:10E79000204602F0F0FF17FB00F300200CE006EB30
:10E7A000430706EB40013A88ADF80020B1F800C0FD
:10E7B000A7F800C00A80401C5B1E8342EFD869881E
:10E7C0006288E088891A491EE1806988081A401E1B
:10E7D000608029882288A088891A491EA1802988FA
:10E7E000081A401E2080F8BD2DE9F0470C46164659
:10E7F0008246002701EBD47931E00025601C00EB54
:10E80000D07827E0E01B401E01B2601B401E00B222
:10E81000BAF1000F0AD015FB041206EB420311FBFC
:10E82000040106EB410210FB047009E010FB0472C6
:10E8300006EB420311FB040006EB400215FB04103B
:10E8400006EB400117FB045006EB4000FFF78EFF7C
:10E850006D1C2DB2B5EB680FD4DB7F1C3FB2B7EB5C
:10E86000690FCADBBDE8F0872DE9FF4F95B0987BB3
:10E870008A7E00F00F04DDF888800D46032C00D15D
:10E880000424012C19D0022C1FD0042C25D0082CD4
:10E890007DD1DFF890924FF0FF0A6101FD2A35D259
:10E8A000DFF884C29CF80000904203D1DCF8040039
:10E8B000A04225D000209D4F20E0DFF868924FF065
:10E8C000800AA9F116090221E8E7DFF858924FF013
:10E8D000C00AA9F114090421E0E7DFF848924FF0DB
:10E8E000F00AA9F110091021D8E719F80060FF2EED
:10E8F0001CD016FB02F6360A3E54401C8842F4D364
:10E90000DFF828928CF80020CCF804401798DE88B5
:10E910000996B0F900101598B3F808B066438068FE
:10E92000B0F90020914203DB002202E01646E3E743
:10E93000521A0A92099A8B18B0F90420934201DC0A
:10E94000099901E0511A491C0B911799B0F902205D
:10E95000B1F90210914201DB002200E0521A0E923E
:10E96000B0F9060001EB0B02824201DC584601E0DF
:10E97000401A401C0F900E980A99704301FB040046
:10E9800008EBD00700F0070668461C2100E0C5E050
:10E9900019F0A7FBA889ADF80800A87E8DF818002B
:10E9A000A87FC0F3C2008DF81900FDF741FF12F0F7
:10E9B000BDFA099901FB0BF1814200DC0846109079
:10E9C00014F0F6FD834603901798002501880A98F5
:10E9D0000A181798ADF81C2001880B98401E0144B6
:10E9E000ADF82010179843880E9818448B1A5B1CBA
:10E9F000ADF81E00ADF822001BB21193ADF8341033
:10EA0000ADF830200F99ADF832000844ADF836006B
:10EA10000CA803F0C7FF139007A800900590C4F15D
:10EA200008001290DDE9090101440B98081A6043BF
:10EA300014900E985BE02B462AFA06F04FF0000C7B
:10EA40000A991AE03A78DDF848800240A8EB0608F7
:10EA500032FA08F204D019F802800BF8058001E0C0
:10EA60000BF805C0129A964202D22644E04002E01A
:10EA7000002650467F1C491C6D1C0B9A9142E1DB1D
:10EA8000139880B10BEB0300BDF92220BDF91C10D7
:10EA90008046119B03F048FF8DF8100018B94046DE
:10EAA000119919F01EFBDDE90A10401A411910985E
:10EAB000814205D2BDF82200401CADF822000EE0D4
:10EAC00002208DF810006946159804F094FCBDF8FA
:10EAD0002200401CADF81E00ADF82200002514985D
:10EAE000304407EBD00700F007060998401C0F9947
:10EAF000099088429FDBBDF91E10BDF922008142BA
:10EB000009D0401EADF8220002208DF810006946A1
:10EB1000159804F070FC584614F096FD19B0BDE845
:10EB2000F08F0000269D0108845200207CD3002035
:10EB30002DE9F04F8346B1F902000C46401E41100A
:10EB400000F001004618B2F90000B3F9005089B096
:10EB5000A84200DB2846ADF80000B2F90000B3F986
:10EB60000030984200DC1846401EADF80400508882
:10EB7000801BADF8020050880844ADF806006946D5
:10EB80000846DBF808200BF02AFA002822D0E0889B
:10EB900018B1A08808B1012000E0002080460126BD
:10EBA000684603F0FFFE10B9B8F1000F00D0002650
:10EBB0001C2102A805F019FECDF808D02088ADF878
:10EBC0001000207A6D468DF8200036B102A9584613
:10EBD00004F011FC09B0BDE8F08FBDF80410BDF9D8
:10EBE0000000BDF906A0091A491C0EB2BDF80210BA
:10EBF000ADF806104FF00009B8F1000F08D0B4F9D5
:10EC00000610B4F90420114490FBF1F201FB120943
:10EC1000304614F0CDFC079505900746BDF902502B
:10EC20003EE03146384605F0E4FDBDF900103346BC
:10EC30002AB2384603F078FE8DF81800B8F1000FBC
:10EC40001FD0F0B1002148460B4615E0B4F904206E
:10EC5000824205DB121A1144104409B200B207E0E7
:10EC6000B4F906C06244824201DC002000E07B541B
:10EC7000491C401C09B200B2B142E7DB02208DF80A
:10EC8000180002A9584604F0B6FBBDF80200401C6B
:10EC9000ADF80200BDF80600401CADF806006D1C82
:10ECA0005545BEDD384614F0CFFC93E72DE9FF4F04
:10ECB000B2F90250B3F90240BBB0A54208DA12889B
:10ECC00065F31F4062F30F0064F31F411A8807E0E9
:10ECD0001B8864F31F40128865F31F4163F30F0024
:10ECE00062F30F010FFA81F906B20714A9EB0604CB
:10ECF0004FEA214AAAEB07053791002C01DD204697
:10ED000000E06042002D01DD294600E069428842B2
:10ED100001DD012000E0002000903C98B0F90210D5
:10ED2000009858B1002D01DD284600E068424201FC
:10ED3000002C01DD20460CE060420AE0002C01DDE1
:10ED4000204600E060424201002D01DD284600E03F
:10ED5000684292FBF0F0AB4A105C10FB01F03F30D0
:10ED6000C0114FEA600800F0010202EB080B4946AF
:10ED70004E4500DA3146A1EB0001ADF8601001DD2F
:10ED8000314600E049460144ADF86410514657450C
:10ED900000DA3946A1EB0001ADF8621001DD394619
:10EDA00000E051460844ADF866003B9818A9826817
:10EDB00008460BF014F900287ED0009800210028A6
:10EDC0007BD0002C16DDAAEB080000B2CDE90001D3
:10EDD000A7EB080002B24B46314602A803F080FEC2
:10EDE0000AEB0B00012100B2CDE900014B4607EB15
:10EDF0000B0015E00AEB0B0000B2CDE9000107EBB8
:10EE00000B0002B24B46314602A803F069FEAAEBA2
:10EE10000800012100B2CDE900014B46A7EB080034
:10EE200002B231460DA803F05BFE002102A803F0F8
:10EE3000C9FB399000210DA803F0C4FB38904FF0B6
:10EE4000FF30804600903C98407AC00623D43819A1
:10EE5000032100B2CDE90001701B03B23A463146EE
:10EE600021A803F03DFE379902200A14111909B2B6
:10EE7000CDE90010379801B2481B03B22CA803F06B
:10EE80002FFE002121A803F09DFB009000212CA85B
:10EE900003F098FB8046BDF86400BDF86010401A8E
:10EEA000401C06B2FDF7C4FC12F040F8044618A856
:10EEB00011F077F8A04201E0A1E028E003D218A801
:10EEC00011F06FF80446A146204614F071FB82460B
:10EED000BDF966B0BDF86200ADF866000024494691
:10EEE000504605F086FC1C211AA805F07EFC3C98D3
:10EEF00018A91A910088ADF870003C98007ACDF8F6
:10EF000074A08DF880001F91BDF9625044E009EBB8
:10EF10000B00CDE900A103B206EB0B0001B23A46AB
:10EF200002A803F0DDFD0121A9EB0800CDE900A155
:10EF300003B2A6EB080001B23A4673E70AEB0407F6
:10EF4000BDF9601033462AB2384603F0EDFC8DF867
:10EF5000780018B93846314605F047FC3444A11909
:10EF6000494505D2BDF86600401CADF8660012E0C8
:10EF700002208DF878001AA93B9804F03CFABDF8FD
:10EF800066000024401CADF86200ADF866004946FA
:10EF9000504605F02EFC6D1C5D45CFDDBDF96210BD
:10EFA000BDF96600814209D0401EADF8660002201E
:10EFB0008DF878001AA93B9804F01DFA504614F019
:10EFC00043FB02A803F0D2FC0DA803F0CFFC00988D
:10EFD000401C02D021A803F0C9FCB8F1FF3F02D0C9
:10EFE0002CA803F0C3FC399803F0F0FF389803F025
:10EFF000EDFF009803F0EAFF404603F0E7FF3FB063
:10F00000BDE8F08F269E01082DE9F04F8346B1F947
:10F0100002000C46401E411000F00100158889B026
:10F020000844281AADF8000010880844ADF8040020
:10F03000B2F90200B3F90210884200DB0846ADF8CD
:10F040000200B2F90200B3F90210884200DC08465F
:10F05000401EADF8060069460846DBF808200AF0B5
:10F06000BEFF00281FD0E08818B1A08808B1012792
:10F0700000E000270125684603F094FC00B907B1C1
:10F0800000251C2102A805F0B0FBCDF808D020888F
:10F09000ADF81000207A6E468DF8200035B102A937
:10F0A000584604F0A8F909B0BDE8F08FBDF8040097
:10F0B000BDF80010BDF90690401A401C0FFA80F808
:10F0C000BDF80200ADF80600404614F071FA824621
:10F0D00000250796059057B1B4F90600B4F904105D
:10F0E0000844BDF9021091FBF0F200FB1215BDF9C6
:10F0F00002602EE04146504605F07BFBBDF9001052
:10F10000434632B2504603F00FFC8DF818008FB121
:10F1100070B1B4F90400A84202DA00208DF818009A
:10F12000B4F90600B4F904100844A84200DC002534
:10F130006D1C2DB202A9584604F05DF9BDF802001D
:10F14000401CADF80200BDF80600401CADF80600FA
:10F15000761C4E45CEDD504614F076FAA3E770B526
:10F16000054691F82A0088B00C46022858D9E18C4F
:10F17000002955D0114604A802F0EEFA218DBDF801
:10F180001000491E401AADF81000BDF81200401AD8
:10F19000ADF81200BDF814000844ADF81400BDF835
:10F1A00016000844ADF8160004A906A802F0D4FA27
:10F1B000BDF81810E08C091AADF81810BDF81C1035
:10F1C0000844ADF81C00BDF81A00E18C401AADF8F7
:10F1D0001A00BDF81E00E18C0844ADF81E0004A81A
:10F1E00002F005FB064604A802F0D7FAB4F90010B5
:10F1F000864200DA3046B1EB600F00DD4110E08C52
:10F20000A278084403B294F82A00CDE90202A08C47
:10F21000ADF80400009104AA06A92846FEF753FEA3
:10F2200008B070BD7CB50446806961896D4686680A
:10F23000A08961B1002865D0814203D12289E38889
:10F240009A427CD302297BD003297AD0AFE010BB4D
:10F25000E088218988421ED2B4F9060016F0E6F84B
:10F26000B4F90410B4F90E20891A4843216849887A
:10F2700001EBE030ADF80200E0885A3000B216F041
:10F28000D5F8A18810FB01F02168098801EBE03076
:10F29000ADF8040040E020680088ADF80000206868
:10F2A000A18840880844ADF80600B4F9060016F0BD
:10F2B000BDF8B4F90410B4F90E20891A4843216846
:10F2C000498801EBE030ADF80200E0885A3000B226
:10F2D00016F0ACF8A18810FB01F0216832460988CD
:10F2E00001EBE030ADF80400694608460AF077FE0D
:10F2F00030B1A0698560D4E90520216903F076FE6C
:10F30000A08970BB2068A18800880844ADF804007B
:10F3100020684088ADF80200B4F9080016F086F8BD
:10F32000A18810FB01F02168498801EBE030ADF8BD
:10F33000060020895A3000B216F078F802E015E095
:10F3400012E00FE0B4F90410B4F90E20891A484312
:10F3500021683246098801EBE030ADF800006946CB
:10F360001AE024E0022801D0012820D1206832468A
:10F370000088ADF8000020684088ADF802002068E1
:10F38000A18800880844ADF804002068A18840885E
:10F390000844ADF80600294608460AF020FE30B1C0
:10F3A000A0698560D4E90520216903F01FFEA069EA
:10F3B00086607CBD7CB50446806961896D4686683F
:10F3C000A08901290CD0012867D0814203D122896C
:10F3D000E3889A427ED300297DD003297CD0B5E012
:10F3E000012822D1E088218988421ED2B4F9060082
:10F3F00016F01CF8A18810FB01F02168498801EB88
:10F40000E030ADF80600E0885A3000B216F00EF891
:10F41000B4F90410B4F90E20891A48432168098808
:10F4200001EBE030ADF8040042E02068A1880088DC
:10F43000401AADF8000020684088ADF80200B4F929
:10F44000060015F0F3FFA18810FB01F02168498840
:10F4500001EBE030ADF80600E0885A3000B215F05C
:10F46000E5FFB4F90410B4F90E20891A4843216865
:10F470003246098801EBE030ADF8040069460846E1
:10F480000AF0ADFD30B1A0698560D4E9052021699D
:10F4900003F0ACFDA089012858D120680088401EE7
:10F4A000ADF804002068A18840880844ADF8060043
:10F4B000B4F9080015F0BAFFB4F90410B4F90E203D
:10F4C000891A48432168498801EBE030ADF8020011
:10F4D000208902E018E010E014E05A3000B215F084
:10F4E000A5FFA18810FB01F021683246098801EBD5
:10F4F000E030ADF8000069461DE0022804D0032882
:10F5000002D023E0022821D12068A1883246008859
:10F51000401AADF8000020684088ADF8020020686D
:10F520000088401EADF804002068A1884088084487
:10F53000ADF80600294608460AF051FD30B1A06931
:10F540008560D4E90520216903F050FDA06986603B
:10F550007CBD7CB50446806961896D468668A0895A
:10F5600002290CD002287ED0814203D12289E3886F
:10F570009A4279D3002978D0012977D0D4E00228A3
:10F580003FD1E088218988423BD25A3000B215F041
:10F590004DFFA18810FB01F02168098801EBE030E4
:10F5A000ADF80000B4F9060015F040FFB4F90410FE
:10F5B000B4F90E20891A48432168498801EBE030EC
:10F5C000ADF80600B4F9080015F030FFA18810FB73
:10F5D00001F02168498801EBE030ADF80200208994
:10F5E0005A3000B215F022FFB4F90410B4F90E201D
:10F5F000891A48432168098801EBE030ADF804001E
:10F6000066E020680088401EADF804002068A188EC
:10F610004088401AADF80200E0885A3000B215F078
:10F6200005FFA18810FB01F02168098801EBE0309B
:10F63000ADF80000B4F9060015F0F8FEB4F90410B6
:10F64000B4F90E20891A484321683246498801EBF3
:10F65000E030ADF80600694608460AF0C0FC58B133
:10F66000A069856003E00AE03BE034E036E0D4E9DD
:10F670000520216903F0BAFCA089022854D1206832
:10F68000A1880088401AADF8000020684088401E1C
:10F69000ADF8060020895A3000B215F0C7FEB4F963
:10F6A0000410B4F90E20891A48432168098801EB37
:10F6B000E030ADF80400B4F9080015F0B7FEA188F9
:10F6C00010FB01F02168498801EBE030ADF8020041
:10F6D000324669461DE0032803D025E0032800D008
:10F6E00010BB2068A18832460088401AADF800009F
:10F6F0002068A1884088401AADF802002068294699
:10F700000088401EADF8040020684088401EADF817
:10F71000060008460AF063FC30B1A0698560D4E9B0
:10F720000520216903F062FCA06986607CBD7CB580
:10F730000446806961896D468668A08903290ED0D8
:10F74000032867D0814203D12289E3889A427ED37D
:10F7500002297DD001297CD002297BD0B1E0032889
:10F760001FD1E088218988421BD25A3000B215F09F
:10F770005DFEB4F90410B4F90E20891A48432168DB
:10F78000098801EBE030ADF80000B4F9060015F08F
:10F790004DFEA18810FB01F02168498801EBE030A3
:10F7A00040E02068A18800880844ADF80400206883
:10F7B0004088401EADF80600E0885A3000B215F0CF
:10F7C00035FEB4F90410B4F90E20891A48432168B3
:10F7D000098801EBE030ADF80000B4F9060015F03F
:10F7E00025FEA18810FB01F021683246498801EB13
:10F7F000E030ADF80200694608460AF0F0FB30B18F
:10F80000A0698560D4E90520216903F0EFFBA08998
:10F81000032856D120680088ADF800002068A18830
:10F820004088401AADF8020020895A3000B215F025
:10F83000FDFDA18810FB01F02168098801EBE03093
:10F84000ADF80400B4F9080015F0F0FD03E016E08F
:10F8500010E013E00FE0B4F90410B4F90E20891A97
:10F86000484321683246498801EBE030ADF8060094
:10F8700069461BE018B1012801D022E008BB2068CE
:10F8800032460088ADF800002068A1884088401A00
:10F89000ADF802002068A18800880844ADF8040093
:10F8A000206829464088401EADF8060008460AF048
:10F8B00096FB30B1A0698560D4E90520216903F089
:10F8C00095FBA06986607CBD70B5A4B00C4605466A
:10F8D00022AA20A906F069F820A810F062FB20B93E
:10F8E00022A810F05EFB00283ED012A9284609F09D
:10F8F000BFFD012838D12146684605F043FC1B486E
:10F9000001900220029012A804904FF480300D90D4
:10F9100020A810F046FB80B120A803906A461A2167
:10F92000284611F0DDFB20AA12A9204603F05EFB59
:10F930006A461B21284611F0D3FB22A810F031FBA8
:10F94000002811D022AE6A461A212846039611F0EB
:10F95000C7FB22AA12A92046039603F047FB6A467A
:10F960001B21284611F0BCFB24B070BDEC9C0108A3
:10F970002DE9F74FB1F92E00A2B014460D4600282C
:10F9800072D095F8361002296ED9012808D1B5F940
:10F990003400002804DC288E10B9688E0028EFD0CF
:10F9A0002088298EAA8E0844801AADF82000A388EA
:10F9B00019441144ADF8241062886B8E1A44AB8E42
:10F9C000D21AADF82220E3886E8E3344AE8E3344D3
:10F9D000ADF82630B5F92E6006EBD676A0EB6600C2
:10F9E000401EADF82800012000EB66063144ADF85A
:10F9F0002C10B5F92E1001EBD171A2EB6101491E5B
:10FA0000ADF82A10B5F92E1001EBD17100EB6100B1
:10FA10001844ADF82E0095F836000D90FD2801D958
:10FA2000FF200D9022980AA9826820A80AF0D7FA30
:10FA30000028A5D0214603A801F08EFE4FF0FF3725
:10FA400039463A4603A810F0D8FAB5F9009003A851
:10FA500001F0CDFE044603A801F09FFE844203A8F6
:10FA600003DA01F0C4FE02E0FEE301F096FEB9EB1A
:10FA7000600F01DD4FEA6009B5F9006008A801F0E8
:10FA8000B6FE044608A801F088FE844208A802DAFF
:10FA900001F0ADFE01E001F080FEB6EB600F00DD8D
:10FAA0004610B5F92E00841904FB04F0400013F051
:10FAB0007FFD00900146B5F92E20334608A809F0D5
:10FAC000EFFD0AA802F06EFF012620B9E878FF28B2
:10FAD00001D3A87800B100261F9756B901234A46E2
:10FAE00003A912A803F0C8F9002112A802F06AFDC8
:10FAF0001F900AA801F07BFE13F05AFD83461C21DB
:10FB000018A804F074FE01A81890CDF86CB01D90F0
:10FB1000A88DADF8680095F836008DF87800A878C3
:10FB20008DF879000AA801F062FEBDF8281000EBFC
:10FB3000D07001EB60000FFA80FA0AA801F02DFEE8
:10FB4000BDF82A1000EBD07001EB600007B2BDF8E1
:10FB50002C00ADF80800001B401C00B2621EADF87E
:10FB60000400ADF8061011440C9209B2ADF80A1069
:10FB70005246504500DC1046ADF80400B94200DBA7
:10FB800039462298ADF80A1001A9826805A80AF042
:10FB900026FAC0B34A4603A905A80AF048FA90BB62
:10FBA00005A801F024FEBDF91610BDF92A200E901B
:10FBB000891A0098BDF92C2001FB0400BDF914102E
:10FBC000121B891A0844401E119046B14A4603A9E7
:10FBD00005A80AF09CFA10B10120079000E00796F2
:10FBE0000E98002827DDBDF81400ADF80400CDF80C
:10FBF0006CB0BDF81800ADF8080002208DF8700058
:10FC0000BDF9168013E016E0ADF80A800798ADF84C
:10FC10000680E8B311981B9018A9229803F0EBFB1B
:10FC200011982044119008F101000FFA80F8BDF9F5
:10FC30001A104145E8DABDF82C00ADF80800001BA9
:10FC4000401C00B2ADF80400BDF82E20ADF80A202B
:10FC5000111B491C09B2ADF806105246504500DC94
:10FC60001046ADF80400781C0F90814200DC791C2E
:10FC70002298ADF8061001A9826805A80AF0AFF92C
:10FC8000D0B34A4603A905A80AF0D1F9A8B15FE0AC
:10FC9000FFE722465846119904F09EFDBDF9141065
:10FCA000424658460E9B02F03FFE8DF87000012838
:10FCB000B2D102208DF87000AEE705A801F097FDE3
:10FCC000BDF90A10BDF91A200E90891A0098BDF9E5
:10FCD0002C2001FB0400BDF91410121B891A0844E2
:10FCE000401E11904EB14A4603A905A80AF00FFA2A
:10FCF00018B10120079001E02AE007960E9800282D
:10FD000026DDBDF81400ADF80400CDF86CB0BDF8E8
:10FD10001800ADF8080002208DF87000BDF91A80B7
:10FD200012E0ADF80A800798ADF80680B0B31198DC
:10FD30001B9018A9229803F05EFB119820441190A3
:10FD4000A8F101000FFA80F8BDF916104145E8DD71
:10FD5000BDF828002044ADF80400BDF82C00001BBD
:10FD6000ADF80800BDF82A000C99ADF8060008446B
:10FD700000B2ADF80A00B84200DB3846ADF80A0020
:10FD8000229801A9826805A80AF029F990B34A4689
:10FD900003A905A80AF04BF9A8B178E0FFE72246CD
:10FDA0005846119904F018FDBDF914104246584602
:10FDB0000E9B02F0B9FD8DF870000128B9D1022028
:10FDC0008DF87000B5E705A801F011FD0E90BDF9A2
:10FDD0001610BDF906200098891A01FB0400119045
:10FDE0004EB14A4603A905A80AF091F918B10120BD
:10FDF000079001E04BE007960E98002847DD079832
:10FE000060B100201B90BDF81400ADF80400BDF8EF
:10FE10001800ADF80800BDF9160033E0CDF86CB05D
:10FE2000F1E7ADF80A800798ADF8068060B10D984B
:10FE3000FF281198007804D095F8361010FB01F0D7
:10FE4000000A8DF8780013E011980E9A0178584650
:10FE500004F0C4FCBDF91410424658460E9B02F053
:10FE600063FD8DF87000012802D102208DF870002A
:10FE700018A9229803F0BFFA11982044119008F1B4
:10FE8000010000B2BDF91A1080464145C9DA95F863
:10FE900036008DF87800BDF828002044ADF8040045
:10FEA000BDF82C00BDF82E10001BADF80800081B93
:10FEB000401CADF80A1000B20F99ADF80600884258
:10FEC00000DC781CADF80600229801A9826805A81C
:10FED0000AF085F8F0B34A4603A905A80AF0A7F886
:10FEE000C0BB05A801F083FC0790BDF90A10BDF95D
:10FEF0001A200098891A01FB040011900798002825
:10FF000055DD2EB14A4603A905A80AF000F900B94B
:10FF100066B100201B90BDF81400ADF80400BDF8D8
:10FF20001800ADF80800BDF91A003BE0CDF86CB040
:10FF3000F1E7ADF80680ADF80A802EB14A4603A974
:10FF400005A80AF0E4F800B976B10D98FF281198D9
:10FF5000007800E02BE004D095F8361010FB01F09B
:10FF6000000A8DF8780013E01198079A0178584636
:10FF700004F034FCBDF9141042465846079B02F0C9
:10FF8000D3FC8DF87000012802D102208DF870009A
:10FF900018A9229803F02FFA119820441190A8F183
:10FFA000010000B2BDF9161080464145C1DD95F84B
:10FFB00036008DF87800BDF82C00ADF80800011B64
:10FFC000BDF82A00491C09B22044ADF8041000B263
:10FFD000ADF80600BDF82E200F9B121B12B2ADF833
:10FFE0000A20984200DB781CADF80600BA4200DC1B
:10FFF0003A46ADF80A205046514500DC01462298A9
:020000040801F1
:10000000ADF8041001A9826805A809F0E8FFC8B39B
:100010004A464D4603A905A80AF009F890BB05A871
:1000200001F0E5FB10900C990098BDF92C2001FB24
:100030000400BDF91410121B891A0844401E1190C7
:1000400046B12A4603A905A80AF061F810B14FF09D
:10005000010802E0B6F1000801D0119800E058460E
:100060001B901098002832DDBDF81400ADF8040094
:10007000BDF81800ADF8080002208DF87000BDF939
:10008000165020E023E0ADF80650ADF80A50B8F164
:10009000000F12D1DDE91021584604F09DFBBDF997
:1000A00014102A465846109B02F03EFC8DF8700052
:1000B000012802D102208DF8700018A9229803F0BF
:1000C0009AF96D1C2DB2BDF91A00A842DBDA0023A3
:1000D000009815E000EB040EAEF10101002204EBE4
:1000E000D47C07E0057891F8008000F8018B01F8D6
:1000F0000159521CB2EB6C0FF4DB5B1C70461BB257
:10010000A342E7DBBDF828000C99ADF804000844D1
:1001100001B2BDF82A000F9B204400B2ADF80600E2
:10012000BDF82E20ADF80810121B12B2ADF80A204F
:10013000984200DB781CADF80600BA4200DC3A4673
:10014000AAF10100ADF80A201090814200DB0146BF
:100150002298ADF8081001A9826805A809F03FFFB0
:10016000B8B34A464D4603A905A809F060FF80BB15
:1001700005A801F03CFB0E900C990098BDF90420F5
:1001800001FB0400BDF91410891A0844119046B10E
:100190002A4603A905A809F0BAFF10B14FF00108DB
:1001A00002E0B6F1000801D0119800E058461B901B
:1001B0000E98002832DDBDF81400ADF80400BDF83B
:1001C0001800ADF8080002208DF87000BDF9165037
:1001D00020E023E0ADF80650ADF80A50B8F1000F6A
:1001E00012D158460E9A119904F0F6FABDF914107E
:1001F0002A4658460E9B02F097FB8DF870000128A6
:1002000002D102208DF8700018A9229803F0F3F8AB
:100210006D1C2DB2BDF91A00A842DBDABDF828002A
:100220000C99ADF80400084400B2ADF80800BDF820
:100230002A100C9AADF806101144109A09B2ADF8C4
:100240000A10904201DBAAF10100ADF80800B942A2
:1002500000DB39462298ADF80A1001A9826805A88A
:1002600009F0BDFEC8B300E044E14A464D4603A98B
:1002700005A809F0DCFE80BB05A801F0B8FABDF9BD
:100280001620BDF906100D90511A0098BDF90420F2
:1002900001FB0400BDF91410891A01EB000846B1F6
:1002A0002A4603A905A809F032FF10B101200790E2
:1002B00000E007960D98CDF86CB0002821DDBDF860
:1002C0001400ADF80400BDF81800ADF808000220D5
:1002D0008DF87000BDF916500FE012E0ADF80A502D
:1002E0000798ADF80650D0B3CDF86C8018A92298C5
:1002F00003F081F86D1CA0442DB2BDF91A00A8428C
:10030000ECDABDF82800ADF804000C99BDF82E20F9
:10031000084401B2101BADF80810401CADF80A20CB
:1003200000B20F9AADF80600904200DC781CADF8E0
:1003300006001098814201DBAAF101012298ADF874
:10034000081001A9826805A809F049FEC0B34A4611
:100350004D4603A905A809F06AFEA8B158E0FFE7D9
:1003600022464146584604F037FABDF914102A4691
:1003700058460D9B02F0D8FA8DF870000128B5D1CF
:1003800002208DF87000B1E705A801F030FABDF940
:100390000A10BDF91A208246891A0098BDF9042076
:1003A00001FB0400BDF91410891A0F184EB12A463A
:1003B00003A905A809F0ABFE18B14FF0010801E050
:1003C00026E0B046CDF86CB0BAF1000F20DDBDF8E4
:1003D0001400ADF80400BDF81800ADF808000220C4
:1003E0008DF87000BDF91A500EE0ADF80650ADF86A
:1003F0000A50B8F1000F2FD01B9718A9229802F0CD
:10040000FAFF6D1E27442DB2BDF91600A842ECDD9F
:10041000BDF8280001A92044ADF80400BDF82C0067
:10042000001BADF80800BDF82A002044ADF8060016
:10043000BDF82E00001BADF80A002298CDF86CB074
:10044000826805A809F0CBFDF0B34A4603A905A8C8
:1004500009F0EDFDA0B140E022463946584604F0CF
:10046000BBF9BDF9141053462A46584602F05CFA0F
:100470008DF870000128C0D102208DF87000BCE713
:1004800005A801F0B4F9051E27DDBDF81400ADF88C
:100490000400BDF81800ADF80800BDF9164018E0DA
:1004A000ADF80640ADF80A402946584604F0A4F9D4
:1004B000BDF914102B462246584602F035FA8DF845
:1004C000700018A9229800E007E002F094FF641C75
:1004D00024B2BDF91A00A042E2DA2EB912A802F045
:1004E00045FA1F9802F072FD009813F0ADF85846D7
:1004F00013F0AAF825B0BDE8F08F00002DE9FF4FFA
:1005000083B00446DDE910870E460846139D01F0CE
:100510005CF98346304601F034F90190012D0FD08B
:10052000022D0FD0032D3ED1404E6FB12088ADF883
:10053000000038784FF0000AFD2837D3424638E0F3
:100540003B4EF2E73B4EF0E72088ADF80800ADF8EF
:100550000000424602990698B047002702901FE02B
:10056000002517E0BDF8000034F8151088420BD0C4
:1005700004EB450042460088ADF80800ADF80000E5
:1005800002990698B047029004EB4500BDF80810A8
:1005900001806D1C5D45E5DB05987F1C04EB400484
:1005A00001988742DCDB07B0BDE8F08F00FB08F064
:1005B000020A00990698B0470290002030E000251A
:1005C00025E0785D10B3504505D1BDF8001034F832
:1005D0001520914215D0FD2801D3424602E000FBD0
:1005E00008F0020A04EB45000088ADF80800029903
:1005F0000698B047029017F805A034F81500ADF83A
:10060000000004EB4500BDF8081001806D1C5D453D
:10061000D7DB059804EB40041298074409F1010068
:10062000019981468842CADBBDE700007BD3000800
:10063000F9D20008FFD300082DE9FF4F85B004462A
:10064000DDE9127593460E46084601F0BEF8804675
:10065000304601F096F882466DB1BDF82000FD2FBE
:1006600000EB00497DD3A8F1040001900020009028
:10067000BDF820703AE1FD2F0ED3002507E0424679
:100680002046089910F044FA04EB4B046D1C5545C4
:10069000F5DB09B0BDE8F08FBDF80010002060F375
:1006A000020189B260F3C70189B260F30C2189B2FB
:1006B00060F34F31ADF8001088B20090BDF8000033
:1006C000009001463A46089801F060F93F1D0190FC
:1006D0000899F808C00689B2000EC1F3C40212FBE3
:1006E00000F2ADF808204A07920E02EB513212FBDD
:1006F00000F2ADF80A20C1F3042111FB00F1ADF8BE
:100700000C10C0F1FF02002556E000204FE0BDF8BC
:10071000001034F81030994243D004EB40010988AE
:10072000ADF80410ADF80010BDF80430BDF80810A5
:10073000C3F3C40616FB021101EBC11606EBC1316F
:10074000BDF81060C1F3C45161F3C7065907890EA3
:10075000BDF80A7001EB533111FB027101EBC117B7
:1007600000E0C9E007EBC137BF0E67F3020601EBFB
:10077000C11707EBC131C1F3C25161F34F36BDF868
:100780000C10C3F3042313FB021101EBC11303EBA1
:10079000C131C1F3C45161F30C26B1B2ADF81060A0
:1007A000019104EB4001BDF804300B80401C404532
:1007B000ADDB04EB4B046D1C5545A6DB69E7002659
:1007C00010E02A78FF2A12D02088ADF8080002999C
:1007D000089801F0DBF80290BDF808002080A41C06
:1007E0006D1C761C464557DAA807EAD154E02780ED
:1007F000F5E72868411C43D0F0B32A78FF2A4FD090
:100800002088ADF808000299089801F0BFF802901E
:10081000BDF80800208015F8012FA41CFF2A41D044
:100820002088ADF808000299089801F0AFF802900E
:10083000BDF80800208015F8012FA41CFF2A33D032
:100840002088ADF808000299089801F09FF80290FE
:10085000BDF80800208015F8012FA41CFF2A25D020
:100860002088ADF808000299089801F08FF80290EE
:10087000BDF80800208000E00BE0A41C6D1C0AE01D
:10088000A00704D02780C4F80290E78001E0C4E903
:10089000009908342D1D361D01988642A9DD18E007
:1008A0002780B8E72780C6E72780D4E72780E2E7DC
:1008B0002A78FF2A1ED02088ADF8080002990898EF
:1008C00001F064F80290BDF808002080A41C6D1CA3
:1008D000761C4645ECDBABEB080004EB40041498B7
:1008E000A0EB080005440098401C00905045FFF61E
:1008F00066AFCEE62780E9E700212388ADF8043013
:100900008946084633E0002627E0287818B3884255
:1009100005D0FF282FD000FB07F2120A914688422B
:1009200003D134F81600834210D0B9F1FF0F24D060
:1009300004EB46004A460088ADF804000199089887
:1009400001F024F80190297834F8163004EB4600C1
:10095000BDF8042002806D1C761C4645D5DB14983A
:1009600004EB4B04A0EB080005440098401C0090E9
:100970005045C8DB8DE63A46D0E70898E2E72DE916
:10098000FF4F85B00D46DDE912A7FBF751FFBDF81B
:10099000209080464FB1284600F017FF039028466C
:1009A00000F0EFFE8346002640E0B5F9026017E054
:1009B000B5F900400FFA86FB0DE0CDF808A0ADF8C0
:1009C0000490CDF800B0D8F8000023B2079AC769A8
:1009D0000599B847641CB5F90400A042EDDA761C0D
:1009E000B5F90600B042E3DA09B0BDE8F08F0024A3
:1009F00016E0385D98B100FB0AF0000A0290ADF8ED
:100A000004906888079A304400B2009028880599BD
:100A1000204403B2D8F80000D0F81CC0E047641CA2
:100A200003988442E5DB1498761C07445E45DEDBC0
:100A3000DAE700680968884201D101207047002088
:100A4000704740680A6820F04040904200D2086039
:100A50000020704770B50D46C06A24F0ECFE0446D5
:100A6000284612F003FE0CB10C2070BD002070BDB2
:100A700070B50D46C06A23F028F80446284612F0E7
:100A8000F5FD0CB10C2070BD002070BD70B5C56ABD
:100A90000E46342012F05EFD040009D001463246B5
:100AA000284623F0E1FF0028204602D012F0DEFDA8
:100AB000002070BD2DE9F043C3B00025D0F82C8094
:100AC000144689468DF808502F2602AF6A464946DB
:100AD000404624F015FA00280CDD9DF8000002289D
:100AE00004D03946204617F05DFB05E026703946F4
:100AF000601CF8E710D1257008A1204617F037FBDD
:100B00000028E3D006A1204617F031FB0028DDD0F5
:100B1000002043B0BDE8F0830C20FAE72F2E000040
:100B20002F2E2E002DE9F041C56A0E46022A17D05D
:100B3000012A17D0032A17D00024542012F00AFDEE
:100B4000071E0BD0014623463246284625F032F8D0
:100B50000028384602D012F089FD0020BDE8F0815F
:100B60000124EAE70224E8E70324E6E710B5C06AB7
:100B7000029C25F062F9002801DA0C2010BD2060EB
:100B8000002010BD10B5C06A23B1012B02D0022B8A
:100B900000D0002325F008FA002801DA0C2010BD4F
:100BA000002010BD10B51446C06A25F0CFFA002809
:100BB00001DA0C2010BD2060002010BD2DE9F041AD
:100BC000C56A0F46069E284625F0CAFA040005D4D9
:100BD0003946284625F04BFA002802DA0C20BDE8F9
:100BE000F08100203460FAE7B0F90C00032101EB3A
:100BF000400020F00300103070472DE9F041054619
:100C000000206B8C0E460427C3F30514EA680EE03F
:100C100007EBC00151585FEAC11C07D521F07F41A5
:100C2000B14203D152F83000BDE8F081401C84424B
:100C3000EED84FF0806000EBB3204FEAB0506884EC
:100C4000C0F30510C100104612F034FDE860C0B3D7
:100C5000688CC0F30514641E16D06FF003025300B5
:100C6000E86802EBC40141585FEAC11C0CD4890159
:100C70000AD400EBC40103EBC40C6044641ED0E949
:100C800000C0C1E900C0EBD1E868082100EBC40056
:100C900017F027FA082012F05DFCE96841F83400EB
:100CA00013F0E8FCEA6807EBC400115841F08071CA
:100CB0001150EA6866F317011150E86850F83400E3
:100CC000B2E7FFE7FEE700002DE9FC410068C068DD
:100CD000C068B0FBF1F5954200DD1546134F78680A
:100CE0000068806900B30020ADF80000ADF8040092
:100CF000ADF802002CB2601E06B2ADF8066078684E
:100D00006946006882699047684600F034FDA84251
:100D100002DD341EEFDC01E0002C02DC0020BDE827
:100D2000FC81BDF906506D1C2846F8E77052002082
:100D30002DE9FF4F83B0064698468B46059809F08B
:100D4000E0FE01218140B6F820A001F0FF096FEA22
:100D50000A0080B2019096F822004FF0FF37C0F3EE
:100D6000C00500241CE0F16801EBC4004268920158
:100D70003BD5A5B9042202EBC402895801F47F01D6
:100D800059450CD10068817911EA090F07D06A46EC
:100D9000059913F01DFC01282ED0022830D0641CC8
:100DA000708CC0F30510A042DDD81EE0F06850F84A
:100DB0003430997911EA090F16D0042101EBC401EE
:100DC000405800F47F0185B259450DD10198054284
:100DD0000AD1BD4208DD18466A46059913F0F8FBB2
:100DE000012810D002280BD0641C708CC0F30510B1
:100DF000A042DBD8002F0FDB00990120C8F80010BB
:100E000007B0BDE8F08F5545F6D0AF42ECDA009957
:100E10002F46C8F80010E7E70020F1E72DE9F0477A
:100E2000814642F30006C0F15A001D460F465408A1
:100E300000B2761C14F0FAFAA7EB040800FB08F0E5
:100E4000C711484614F0F2FA00FB08F0C011002F59
:100E500006DD7F3F39120A1B32442A80214405E017
:100E60007F3739120A1B21442A80891BA980002858
:100E700006DD7F380012011B31446980204405E003
:100E80007F300012011B20446980801BE880BDE890
:100E9000F0872DE9F04104460020678C0D460426BA
:100EA000C7F30513E2680AE006EBC00151585FEA98
:100EB000811C03D521F07F41A94202D0401C83420E
:100EC000F2D8834203D002EBC000BDE8F0814FF0BE
:100ED000806000EBB7204FEAB0506084C0F305108B
:100EE000C100104612F0E6FBE060608CC0F3051014
:100EF000401E0DD06FF00703E16803EBC00601EB65
:100F0000C0023144401ED1E90061C2E90061F3D161
:100F10000821E06817F0E5F8082012F01BFBE168F3
:100F2000086013F0A7FBE168486840F00070486073
:100F3000E16865F317004860E068C6E701460020F5
:100F4000A1F13002092A01D8D0B27047612901D33A
:100F50002039C9B241390629F7D2DFE801F003058B
:100F600007090B0D0A2070470B2070470C207047B3
:100F70000D2070470E2070470F2070472DE9F0417B
:100F8000064615460F46002005E039462046B04784
:100F900001280AD0204607F019FC040002D060683E
:100FA0008000F2D10020BDE8F08105B12C60012065
:100FB000F9E7000010B50C4621F040FD0D4998B14D
:100FC0000122A27306280DD2DFE800F00C0305070A
:100FD000090B0B2006E0092004E00A2002E01120A2
:100FE00000E01220086002E00020A0730868606042
:100FF00010BD0000385200202DE9F0410446406841
:10100000096820F04040884227D12046FFF7ECFDD8
:10101000DFF84C800546D8F80800021BA0EB05005D
:10102000561BC8F8080015D02746384661193246C5
:1010300017F02FF806E0A068401BA0602046FFF7DD
:10104000D3FD0444D8F808008442F4D1B8192946E5
:1010500017F047F80120BDE8F0810020FBE7000011
:10106000785200202DE9FC41064614468846D807F0
:1010700029D004F108000125002206F114010746D9
:1010800008F0D5FF58B100208DF800006A46122103
:101090003046019710F024F89DF8000098B160895F
:1010A000218A0844401EE081B4F90E10B4F906000C
:1010B000814200DDE08102B02A4621464046BDE87B
:1010C000F04101F0F1B90025EEE72DE9F0410746C6
:1010D00088B01C46164688460846FBF7C2F9054606
:1010E00002A9404604F096FA2A46114602A80EF0DC
:1010F00084FF022E05D0012E22D0002008B0BDE8CA
:10110000F081DDE90201CDE9040100231A4604A9BA
:10111000404605F001F904AA06A8B96808F05FFF87
:101120000028EBD0DDE90601CDE900010123002212
:101130006946404605F0F0F8694602AA084602E012
:1011400002AA6846B96808F04AFF0028D6D000987D
:101150002060019860600120D0E7000070B505466E
:1011600004F0CEF90646002406E0A868006850F8AE
:101170002400FFF7F3FF641CB442F6D3688CC10768
:101180001AD020F001006884284605F027FF284681
:1011900005F040FE86B10021284604F0ACFF58B1AE
:1011A0000C494968884207D80B49096801EBC0001F
:1011B00050E9022128469047688C810708D520F025
:1011C000020068842846BDE87040002105F068BD33
:1011D00070BD000064520020105300202DE9F0473C
:1011E0008046089D1F46E86900FB01F39B1200281A
:1011F00006DD934206DD95F8280080070DD489E0CE
:101200009342F8DBCB1943439B12002808DD93423D
:1012100037DA95F8280080077CD40120BDE8F087F4
:101220009342F6DCA869521C504340F39500021229
:10123000C0B2FF23002826D06E6AC0F1FF0404FB71
:1012400006F4A3EB2426A2EB0104A14636D0002C21
:1012500015DBBC4213DAC0F1FF00C6F1FF014843C1
:10126000A3EB6020C1B295F82800800701D5C1F139
:10127000FF0118F8040007F09AFA08F80400641C4B
:101280001CE0A869D0E74FF0FF06DCE7002C10DB7C
:10129000BC420EDAA6EB6000C1B295F828008007C8
:1012A00001D5C1F1FF0118F8040007F080FA08F831
:1012B0000400686A641C361ABC4202DA686AB042EA
:1012C000E4DBBC4218DA002C16DBA86970438012FC
:1012D0007043C0F34721E869002801DAC1F1FF013A
:1012E00095F82800800701D5C1F1FF0118F8040026
:1012F00007F05DFA08F8040095F82800800707D584
:101300004946B94506DC00290DDB404609E001E00D
:10131000641C01D5002081E7BC4204DC391B08EBCA
:10132000040003F060FA022078E72DE9F05F8A46B6
:101330000A9F06461D46B96901FB02F4A012002966
:1013400000DD401C97F82830504502DA980707D492
:10135000D2E0A0120AEB050C844502DA98077ED48D
:1013600080E044F39500521C4A4342F395044FEA4F
:101370002029221204F0FF08C0B2A9EB0A0491450B
:1013800005D0002903DA10B9FF209146641E91456B
:1013900026D1002C0BDBAC4209DA40444108980707
:1013A00001D5C1F1FF01305D07F001FA305597F822
:1013B0002800641C800706D5A9EB0A01A9424EDA71
:1013C0008CE0304609E0AC4200DD2C46002C46D0D3
:1013D00005DDA5EB040106EB040003F004FA88E048
:1013E0004FF0FF0B002943DAF969494241434FEAC4
:1013F000A128002C0DDBAC420BDA08FB00F1C1F395
:101400004721980701D5C1F1FF01305D07F0CFF901
:101410003055B969A8F1FF0041438812641E11D408
:10142000AC420FDAC8F1FF014143ABEB6120C1B21E
:1014300097F82800800701D5C1F1FF01305D07F062
:10144000B6F9305597F82800A41C800708D5A9EBF9
:101450000A01491EA9424CDC0029B2DC49E04BE0FC
:10146000AC4202DD0120BDE8F09F002CB1DA40E083
:10147000F969C0F1FF0041434FEAA128002C0EDBBF
:10148000AC420CDA00FB08F0ABEB6020C1B298076D
:1014900001D5C1F1FF01305D07F089F93055B96917
:1014A000C8F1FF0041438912641C0ED4AC420CDA2F
:1014B0004843C0F3472197F82800800701D5C1F1C0
:1014C000FF01305D07F073F9305597F82800641C70
:1014D000800707D5A9EB0A01A9420DDC0029BFF658
:1014E00070AF06E0AC4200DD2C46002C04D03FF784
:1014F00070AF4FF00200B6E74FF00000B3E7000016
:101500002DE9F04107460E464FF00008134809F058
:1015100029FA04461CE02146104809F035FA054630
:101520002068B84200D097B96068B04200D076B960
:1015300021460A4809F0B1FA216909B120468847D5
:10154000204612F093F8FBF7F7F94FF001082C460C
:10155000002CE0D14046BDE8F081000000D500201D
:1015600070B505460C46094809F0FCF90BE0016826
:10157000A94204D14168A14207D0002C05D0014600
:10158000024809F001FA0028F1D170BD00D5002011
:1015900010B50446442116F0A4FD4FF4FA70E06241
:1015A000002020626420A0620120A4F840000448CA
:1015B000E06194F8420040F0010084F8420010BD60
:1015C0002F16010838B504464FF480650095D4E91C
:1015D0000B200023194611F09EFF4FF46E73322248
:1015E000002100950EF07DFD0146A26A206A121AC4
:1015F0004A4300EBA22038BD38B504464FF480655D
:101600000095D4E90B200023194611F084FF40F225
:10161000B6334FF46172002100950EF062FD014671
:10162000A26A206A121A4A4300EBA22038BD38B5DC
:1016300004464FF480600090D4E90B200023194643
:1016400011F069FF0146A26A206A121A4A4300EBB0
:10165000A22038BD8B1A002B00DC531A4FF47A718C
:101660004B43B3FBF0F0002800D10120704700008D
:1016700070B54168054611B12868FFF741FF194868
:1016800009F002FA184E10B113F0B2FD706015485F
:1016900009F08DF9040024D02946442216F0F9FC03
:1016A0002868A84200D12460717894F8420061F360
:1016B000820084F84200C0070FD0616939B120462A
:1016C0008847216A01442162A16A0844A0626268D5
:1016D0001AB1206808B1216A9047FBF72DF920461E
:1016E00070BDFEE700D50020F85200200A88028075
:1016F0004A8842808A888280C988C18070470A8867
:1017000002804A8842808A888280C988C180704766
:101710000A8802804A8842808A888280C988C1807B
:1017200070470A8802804A8842808A888280C988F5
:10173000C18070470A8802804A8842808A888280F5
:10174000C988C18070470A8802804A8842808A8896
:101750008280C988C18070470A8802804A88428096
:101760008A888280C988C1807047C1884088081AE9
:10177000401C00B27047C1884088081A401C00B263
:101780007047C1884088081A401C00B27047C18861
:101790004088081A401C00B27047C1884088081A67
:1017A000401C00B2704781880088081A401C00B2B3
:1017B000704781880088081A401C00B270478188F1
:1017C0000088081A401C00B2704781880088081AF7
:1017D000401C00B2704781880088081A401C00B283
:1017E000704781880088081A401C00B270478188C1
:1017F0000088081A401C00B27047F0B504464FF448
:10180000FA66C1F341307710642501280BD121F429
:10181000C040B04207DCB84201DDC0F57A705843E1
:1018200090FBF5F001B2C2F3413001280BD122F454
:10183000C040B04207DCB84201DDC0F57A705843C1
:1018400090FBF5F002B2944201DA204600E0104627
:10185000884201DA0846F0BD944201DA2046F0BD24
:101860001046F0BDF0B504464FF4FA66C1F34130BE
:101870007710642501280BD121F4C040B04207DC69
:10188000B84201DDC0F57A70584390FBF5F001B223
:10189000C2F3413001280BD122F4C040B04207DC32
:1018A000B84201DDC0F57A70584390FBF5F002B202
:1018B000944201DA204600E01046884201DA0846E8
:1018C000F0BD944201DA2046F0BD1046F0BD002282
:1018D00008B51146104600F027F80090BDF800004A
:1018E00008BD002208B51146104600F036F80090F9
:1018F000BDF8000008BD18B54C09BDF80030D2088D
:1019000064F30203ADF80030C308BDF80000890895
:1019100063F3C70080B262F30C2080B261F34F30F2
:10192000ADF8000080B218BD18B54C09BDF8003004
:10193000D20864F30203ADF80030C308BDF800001C
:10194000890863F3C70080B262F30C2080B261F3B0
:101950004F30ADF8000080B218BD18B54C09BDF885
:101960000030D20864F30203ADF80030C308BDF8BC
:101970000000890863F3C70080B262F30C2080B2D4
:1019800061F34F30ADF8000080B218BD18B580B2D9
:10199000030243EA102083B288B2010241EA102018
:1019A000121D0C4980B2D40840EA004043EA0342C9
:1019B00008400A40121A624300EB5210084040EA05
:1019C000104080B2010241EA1020ADF8000080B260
:1019D00018BD00001FF8E00718B580B2030243EA03
:1019E000102083B288B2010241EA1020121D0C4976
:1019F00080B2D40840EA004043EA034208400A406B
:101A0000121A624300EB5210084040EA104080B2C4
:101A1000010241EA1020ADF8000080B218BD0000BC
:101A20001FF8E00781B2C1F3C402C2EBC20000EBB1
:101A30000220C01D4209184662F317404A07920E61
:101A400002EB513202EB420303EB0222D21C920959
:101A500062F30F20C1F30421C1EBC10202EB0121AB
:101A6000C91D490961F30700FF2161F31F60704739
:101A7000FF2208B511461046FFF76FFF0090BDF832
:101A8000000008BD7CB50E7BDDE90654022E08D9A6
:101A90004E88002E05D0A54203D0CDE900544469FC
:101AA000A0477CBD38B50446102116F01AFB012072
:101AB0006080FF202073BDF80010002060F3020159
:101AC00089B260F3C70189B260F30C2189B260F377
:101AD0004F31ADF8001088B20090BDF800000090C2
:101AE000BDF80000208038BD2DE9F04F85B082465A
:101AF00010B294468B460FFA82F9AAEB000EDDF87D
:101B000038800FFA8EF2049203F5B471ABEB000249
:101B10001E4613B203920AEB0002119C5844029233
:101B200012B207B2019088457DD04FF4B4718E4255
:101B300002D9A6F5B476B6B2884503D9A8F5B47033
:101B40001FFA80F80F99ACEB010000B200901098DA
:101B500018B101EBD1704010401C05B25A21B6FB00
:101B6000F1F0B8FBF1F1C0B2C9B2042800D10320F2
:101B7000042900D1032188427ED146457CD868B330
:101B8000012854D0022878D003287ED106F15A00CB
:101B900000B213F04BFC009910FB01F10AEBE130AD
:101BA000401B208030B213F041FC10FB09F10BEB1D
:101BB000E130401B608008F15A0000B213F036FC9F
:101BC00010FB09F10AEBE1302844A0800FFA88F0FD
:101BD00013F02CFC009910FB01F15AE130B213F024
:101BE00025FC009910FB01F10BEBE130401B6080FC
:101BF0005A3630B213F01AFC10FB09F10AEBE1304F
:101C00002844A0800FFA88F013F010FC10FB09F1B3
:101C10000BEBE1302844E08008F15A0000B213F0E9
:101C200005FC009900E0E6E010FB01F129E030B28C
:101C300013F0FCFB10FB09F10BEBE1302844E080D2
:101C40005A3630B213F0F2FB009910FB01F10AEBA7
:101C5000E1302844A0800FFA88F013F0E7FB0099E8
:101C600010FB01F10BEBE130401B608008F15A00E2
:101C700000B213F0DBFB02E036E009E005E010FB08
:101C800009F10AEBE130401B208005B0BDE8F08F80
:101C900006F15A0000B213F0C9FB10FB09F10AEB80
:101CA000E130401B208030B213F0C0FB009910FBE4
:101CB00001F10BEBE1302844E0800FFA88F013F0DB
:101CC000B5FB10FB09F10BEBE130401B608008F124
:101CD0005A0000B213F0AAFB009910FB01F10AEBC5
:101CE000E1302844A080D0E730B1012837D0022865
:101CF00061D003287ED099E001297CD108F15A00F7
:101D000000B213F093FB10FB09F10AEBE130401B2A
:101D100020800FFA88F0029013F088FB074630B25B
:101D2000804613F083FB874201DA029800E04046C8
:101D300013F07CFB009910FB01F10BEBE130401B31
:101D400060805A3630B213F071FB10FB09F10AEBD8
:101D5000E1302844A08001982844E08095E70229DA
:101D600064D1AEEB050020800FFA88F013F05EFB23
:101D700010FB09F10BEBE130401B608006F15A00CB
:101D800000B2019013F052FB074608F15A0000B26E
:101D9000804613F04BFB874201DD019800E040468E
:101DA00013F044FB009910FB01F10AEBE1302844E9
:101DB000A08030B269E0032938D106F15A0000B2A0
:101DC00013F034FB10FB09F10AEBE130401B2080DB
:101DD0000398401B608008F15A0000B213F026FB04
:101DE00010FB09F10AEBE1302844A0800FFA88F0DB
:101DF000804601E019E019E013F018FB009910FB90
:101E000001F730B2064613F011FB009910FB01F008
:101E1000874201DD404600E0304613F007FB0099A1
:101E200010FB01F00BEBE03096E729B1049820801D
:101E30006380A280E78028E708F15A0000B203908F
:101E400013F0F4FA074606F15A0000B2019013F0BD
:101E5000EDFA874201DA039800E0019813F0E6FA00
:101E6000009910FB01F10AEBE130401B208030B2F9
:101E700013F0DCFA10FB09F10BEBE130401B608042
:101E800002982844A0800FFA88F013F0CFFA10FBD4
:101E900009F10BEBE1305FE72DE9F0411D0017463A
:101EA0000E4604461AD0F07A02281AD9D4F81CC07B
:101EB000BCF1000F03D02046E047012811D02B468B
:101EC0003A4631462046FBF7ADFB012809D006A271
:101ED00039462046BDE8F04107F0A3BC02A23946CE
:101EE000F8E7BDE8F08100004E6F0A64617461009C
:101EF00038B58469049D002C01D00095A04738BDF9
:101F000038B50446182116F0ECF8002211461046A8
:101F1000FFF7F1FC0090BDF800000090BDF8000054
:101F20002081FF20E072401C60800120207538BDB8
:101F3000704700002DE9FF4FADB0887E3A9E98466D
:101F40000C4602287ED9206800287BD02D98006A94
:101F5000002877D0202216A816F09BF8206815904C
:101F6000B8F1000F6ED098F8000000286AD02D98C4
:101F70002F9982682AA808F032F8002862D0207FC2
:101F8000B0F1000A01D14FF0010A607F810703D44C
:101F90002F98FFF714FC0FE0B4F91210009141F6EE
:101FA000FF72CDE90120B4F9143041461FA8226820
:101FB00013F008FBBDF97C001599B4F91220002537
:101FC000B1F908906F1E02EB09011F912F99098842
:101FD000ADF80C102F994A88ADF80E20B4F9161000
:101FE0002791B4F918100A44ADF80E20EEB1E1B90A
:101FF0002F99B1F90210002917DAB3685A1A002A8A
:1020000000DCCA1A1F994FF48063494203EB410177
:102010008A4200DD37603168002906DB0D46BDF8D5
:102020000E10B2881144ADF80E10627F0021CDE988
:102030000012B4F91420249008EB05070346384633
:10204000159900E09FE008F09BFD47192BE0617FA8
:102050000020CDE90001B4F9142008EB0700249B0F
:10206000159908F08DFD3D464719BDF80E101F98D3
:10207000084400B2ADF80E008EB110F5806F0EDB93
:10208000306800280BDA35602F98BDF90E10B0F9D2
:102090000200081A70602F98B0F90200B06018F8BA
:1020A000050000286FD02D98BDF90E1080684944B6
:1020B000B0F902008142CADB5046CDF888A0BAF1DF
:1020C000020F02D0032816D029E0607F0090B4F9F7
:1020D0001430791B08EB0500159A13F0D4FA064664
:1020E0002F98FFF76CFB801BBDF80C1000EBD07035
:1020F00001EB600011E0607F0090B4F91430791BAF
:1021000008EB0500159A13F0BEFA06462F98FFF764
:1021100056FBBDF80C10801B0844ADF80C00D4E948
:10212000019AD14502D94846D1468246A07F800710
:1021300017D012A800F023FAA089ADF8480015982E
:1021400090F90E0000B90120ADF84A00A07E8DF88C
:102150005000A07FC1089DF8510061F301008DF887
:10216000510000202090FFF7B2FB2390FFF7AFFB58
:10217000029004A800F04EFF208AADF81400BDF9CB
:102180000C0026905FE163E1BDF80C102798002653
:102190000844ADF80C0008EB050025901E96781B4E
:1021A0002890B3E00021A9F57F420091FF3A09D0C1
:1021B000AAF57F42FF3A05D0A74A2918404612687F
:1021C000904700901EAB29AA21A9259808F0C0FCD1
:1021D000607FC00710D02198232802D0012E12D092
:1021E0000AE026B1012E06D0022E0AD004E01E9885
:1021F000012620908AE00026E0680290022E41D05D
:1022000042E0002682E0202807D11E992098081A73
:10221000072803D0A0890226239077E0209A2599E9
:1022200068461144062215F034FF00208DF80600A0
:102230009DF80100FEF782FE06469DF80000FEF7BD
:102240007DFE06EB001023909DF80300FEF776FE5E
:1022500006469DF80200FEF771FE06EB001B9DF896
:102260000500FEF76BFE06469DF80400FEF766FECD
:1022700006EB0010C2B223980BF0FF01C0B2FFF7CB
:1022800053FBC8E723980290299A219915980FF0DB
:102290003CF883464FF6FF70814522D0824520D01E
:1022A000009848451DD350451BD2BDF80C00ADF831
:1022B0000000BDF80E10ADF80210A28A0244ABF186
:1022C00001001044ADF804001F986A46401E0844FF
:1022D000ADF8060004A92D9800F088FEE089ADF85D
:1022E0000800BDF80800ADF8640003AA16A9219BF8
:1022F0002D9800F032F9BBF1000F07DDBDF80C009E
:10230000A18A014401EB0B00ADF80C0028991E983E
:1023100081423FF647AFA07F800723D52698ADF8CE
:1023200000002068BDF94A1001ABB0F9080001EBCC
:10233000D17100EBD070401000EB6100BDF80E10C1
:102340006A460844BDF80C10ADF80410ADF8020060
:10235000ADF80600BDF80800ADF8480012A92D98A8
:1023600000F000F9A07FC0071FD02698ADF800004C
:102370002068BDF80E1001AB028940891144091A8A
:1023800015986A4690F90D00081ABDF80C10ADF8C2
:102390000410ADF80200ADF80600BDF80800ADF875
:1023A000480012A92D9800F0DDF8617F0020CDE9EA
:1023B000000108EB0706B4F914203046249B159958
:1023C00008F0DEFB3D4647192F980088ADF80C0059
:1023D0002298022802D0032815D027E0607F0090C1
:1023E000B4F91430791B3046159A13F04CF90646AF
:1023F0002F98FFF7E4F9801BBDF80C1000EBD070AC
:1024000001EB600010E0607F0090B4F91430791B9C
:102410003046159A13F037F906462F98FFF7CFF993
:10242000BDF80C10801B0844ADF80C00BDF80E1070
:102430001F9808442D9900B2ADF80E008968B1F9D3
:102440000610884204DC18F8050000287FF49CAED2
:1024500031B0BDE8F08F00006453002038B5044669
:10246000202115F03EFEFF20A076FFF730FA009005
:10247000BDF80000A0810B4820604FF6FF7060603F
:10248000A060FFF724FA0090BDF80000E08105206D
:1024900011F032FB0090BDF8000020820020E076B1
:1024A00038BD0000D0060508036C002B00D018478B
:1024B0007047436C002B00D0184770472DE9F0415E
:1024C0000546C06B17460E46002826D0E86C11F072
:1024D00041F804001CD0E96C15F003FEFAF7A8F9E6
:1024E000296821626968E161A968A16100683A46CA
:1024F0002146007CC0F3801084F8240030682060FE
:1025000070686060EB6B28469847050001D003E0D7
:10251000FEE7204611F0AAF82846BDE8F08170B524
:102520000C46054601F07DFF206A2860E06968607E
:10253000A069A860FAF77CF9006894F82420016982
:1025400062F386110161AA6C12B1214628469047B8
:102550002046BDE8704011F089B830B4046AA44642
:1025600030BC604730B44C88002C06D00C7A022C6A
:1025700003D9446AA44630BC604730BC704738B5C4
:1025800004460A2115F0ADFD01206080FF20207275
:10259000BDF80010002060F3020189B260F3C701AA
:1025A00089B260F30C2189B260F34F31ADF80010AD
:1025B00088B20090BDF800000090BDF800002080B7
:1025C00038BD000010B504460A4A002052F83030E9
:1025D00023B1401CC0B21028F8D301E0102802D368
:1025E0004FF0FF3010BD42F8304002EBC0025160A6
:1025F00010BD00008CD600202DE9FF4F81B08B4626
:102600000E9C15461E46B4F90A10B4F90C00571A70
:10261000B4F9082004F1100AABEB020204F13C0902
:10262000B4286DDAB4F90E30B42B7DDA00287BD0F3
:10263000002BFCD0984277DDA94276DC616D7943AE
:102640004FEAA12CA16A7F1C79438912A0F20F14D2
:10265000582C01D8002909DB441E592C01D8002927
:1026600004DB5B38B32802D2002900DD0021A3F28D
:102670000F10582801D8002909DB581E592801D805
:10268000002904DB5B3BB32B02D2002900DD0021D3
:10269000ACEB010001EB60000124871AB74200DDBA
:1026A0003746002F0DDD3BB22A465946CDF800A033
:1026B000019800F09FF9040003D13946019802F017
:1026C00092F8B74200DD3746002F00DA00270BEB07
:1026D000070001B2F61B019833B20744CDF8009011
:1026E0002A46384600F086F9050003D131463846BF
:1026F00002F079F8AC4277D1204605B0BDE8F08F02
:1027000068DDB4F90E30B42B64DD984262DDA94275
:102710000BDB616DA46A79437F1C7C438912A41290
:10272000A0F20F17582F01E054E0A5E001D8002CCB
:1027300009DB471E592F01D8002C04DB5B38B32876
:1027400002D2002C00DD0024A3F20F10582801D87B
:10275000002C09DB581E592801D8002C04DB5B3BF8
:10276000B32B02D2002C00DD0024081B04EB600018
:102770000127841AB44200DD3446002C0DDD23B25B
:102780002A465946CDF80090019800F033F9070029
:1027900003D12146019802F026F8B44200DD344608
:1027A000002C00DA00240BEB040001B2361B019868
:1027B00033B20444CDF800A02A46204600F01AF9AE
:1027C000050003D13146204602F00DF8AF4251D149
:1027D000384692E74FF001084746B42805D040B18B
:1027E0000ADAA94203DC09E044E0A9420FDC032035
:1027F0000CE0A942FBDC0AE0A942F8DD33462A4698
:102800005946CDF800A0019800F0F4F88046B4F9DC
:102810000E00B42806D050B1B4F90A000CDAA84270
:102820000CDC0DE0B4F90A00A84207DC11E0B4F9B1
:102830000A00A8420DDC01E0A84201DC032708E001
:1028400033462A465946CDF80090019800F0D2F858
:102850000746B8F1000F09D047B1B8F1030F03D014
:10286000B8F1010F04D005E0032F03D1002044E7A5
:10287000012F01D0022040E701203EE72DE9F84377
:102880000546884640F26710411C089C1746002BFD
:1028900001DA002302E08B4200DB0346002C01DA60
:1028A000002402E08C4200DB04469C4203DAC3F5BC
:1028B000B470204403E0E01A002800DC181BA5F8DF
:1028C0006800AB81EC81A5F808806F81154828600D
:1028D000012028718B4200D9FEE7B42B01D20020E1
:1028E00000E00120002C01DB8B4200DDFEE7B42C70
:1028F00005D3A4F1B401B42901D2002600E00126D9
:1029000000903A46414605F1100000F0C6F8234613
:102910003A46414605F13C00009600F0BEF8BDE89D
:10292000F8830000F92501082DE9F8431E461746F3
:102930008846814600250C4C0DE00090D0F800C080
:1029400033463A4641464846E047002808D0022828
:1029500000D10125083420680028EED115B10220ED
:10296000BDE8F8830120FBE78CD6002010B5017983
:10297000022906D0052913D18068BDE8104010F067
:1029800075BE0446406900280AD00169002904DAAE
:10299000406810F06BFE6069EFE74169491E4161D4
:1029A00010BD000070B5124D060007D0002455F888
:1029B0003410B9B10879022805D002E0286800284F
:1029C00000D0012070BD887CB1F91020C0073046CE
:1029D00001F1080102D007F09AFB01E007F027FBA4
:1029E0000028EED0641CE4B2102CE0D3002070BDAF
:1029F0008CD60020F8B5069CA58A266A521B658AEB
:102A000012B2491B94F8285009B24FEAC57526B195
:102A100000948DB3FEF7E2FBF8BD85B1207C810701
:102A200028D000F00301012924D0022901D1511C32
:102A300020D4C043800719D1002A1BDC16E0227C79
:102A400002F00304022C15D0D543AD0712D0012C9F
:102A500001D100290EDC920701EB030208D0002A05
:102A600004DB494200D5002199420DDB0020F8BD6E
:102A7000002A02DA0120F8BD0CE04A42F6D49A425C
:102A800006DA991A104401E0002901DB01F0ABFEDF
:102A90000220F0E7FEF749FCEDE72DE9FC471C4674
:102AA000DDF8288016460F468146B42B01DDB43C84
:102AB00024B204F15A0000B212F0B8FC07EB601522
:102AC000204612F0B3FC06EB601000B2CDE900081E
:102AD0002BB232463946484600F002F8BDE8FC8782
:102AE0002DE9F0470F46DDE908699846154604468A
:102AF0002C2101F078FEB54206D1B9F1030F03D1C4
:102B00006D1E761E2DB236B2B54205DD4046B84682
:102B1000074630462E46054627816581A4F80C807D
:102B2000E68184F810906782A8EB07004B46A582E7
:102B3000002801DD024601E0A7EB0802711B002915
:102B400001DD0D4600E0AD1BAA4294F8282002DD0D
:102B500042F0010201E022F0010284F82820002561
:102B6000E561244E2660A5612571D6074FF48015D6
:102B70000DD020B195FBF0F64E43B612E66121B1BF
:102B800095FBF1F141438812A061E0690CE021B1AD
:102B900095FBF1F64643B612A66120B195FBF0F025
:102BA00048438012E061A0692062980709D003F0D1
:102BB0000300012808D0022813D0D843800714D07E
:102BC00006E022F0020001E042F0020084F8280052
:102BD000206A81106162002801DA48426062BDE823
:102BE000F087206A0028EFDCEBE7206A0028EBDDA5
:102BF000E7E70000F52901082DE9FE4F0546DDF85D
:102C000030900F461C4699F812009046C0F3000B16
:102C1000B9F91060684609F10801FEF78BFDBDF9AE
:102C20000210BBF1000F2FD041454FDCBDF906105B
:102C300041454BDBBDF900008119B94205DCBDF906
:102C400004203919921B914209DDBDF902108B193C
:102C500043453FDCBDF90620931B43453ADBBBF1FE
:102C6000000F18D0C01B00D50020A04230DCBDF9F9
:102C70000410C91B091A491C4218A24200DD211A7E
:102C8000002925DB2844F4E0414513DCBDF906109A
:102C900041450FDBCEE7C61BA6420BDC002E03DB53
:102CA0003146284601F09FFDBDF90400C71B7F1C7B
:102CB000002F02DC0020BDE8FE8FA74203DAE11BF3
:102CC000E81901F090FD1EB9A74201D10120F2E7F9
:102CD0000220F0E7BDF80430C21B181A401C0FFA9E
:102CE00080FCBDF80600401A401C03B2A8EB0100AE
:102CF00000B2B04202DA301A401E01E0991B401ABD
:102D0000D9F8141000B20223CF6803EB4003FB5A3A
:102D100037F81080A3EB0803ADF808308B684968DA
:102D200033F8103037F8100000EB010A02EB0C000A
:102D3000801B18440FFA80F99019C01A401E07B280
:102D4000BBF1000F4FF0000621D06DE0811B01EBBD
:102D50000A0010F801BC09EB06005FEA000808D47D
:102D6000A04506DA15F80810584605F020FD05F8CC
:102D70000800B7EB060808D4A04506DA15F80810D5
:102D8000584605F014FD05F80800761C36B2BDF96A
:102D900008008642DADB09EB0600A04201DA0146B0
:102DA00000E02146002901DA002002E0A04200DB19
:102DB000204600B2211A284401F015FDBDF9080093
:102DC000381A411CA14201DA0A4600E02246002AD4
:102DD00001DA002402E0A14200DA0C4621B22846C2
:102DE00047E0811B01EB0A0010F8010CC0F1FF0B5A
:102DF00009EB06005FEA000808D4A04506DA15F8DA
:102E00000810584605F0D3FC05F80800B7EB060893
:102E100008D4A04506DA15F80810584605F0C7FC96
:102E200005F80800761C36B2BDF908008642D8DBEA
:102E3000791CA14201DA781C00E02046002801DA62
:102E4000002704E0A14201DA7F1C00E027463AB2E5
:102E5000A9EB0200A11A884201DA034600E00B4602
:102E6000002B01DA002002E0884200DB084601B2B4
:102E7000A81801F0B8FC2BE72DE9F04115460646ED
:102E800088880A881C46801A401C02B2C8884B8871
:102E9000C01A401C00B2824200DA1046B5EB600F47
:102EA00000DD4510002D00DA002506F10800FEF7D0
:102EB00041FC3582B4743748306002203071002301
:102EC000BDB1354A00204FF47A77C0EBC00102EB68
:102ED0008101B1F91810A9421BD1C0EBC00002EB6F
:102EE00080004169491C41610269102D04DA012109
:102EF00003E07361BDE8F08129111144B94205DA9C
:102F0000102D01DA012100E02911571807617061C5
:102F1000F0E7401C0428D8D300242046C0EBC001B1
:102F200002EB8101D1F814C0BCF1000F07D12CB124
:102F3000D1F810C0D4F810E0F44500DA0C46401C7B
:102F40000428EBD33CB16069401CC4E90430102D67
:102F50000EDA01200DE01C2010F0FCFA040006D06F
:102F60001C2101F040FC4FF0FF3020610BE0FEE738
:102F700028111844B84205DA102D01DA012000E0CA
:102F800028111F182761204629467461BDE8F041C9
:102F9000FAF745B8F92B01081CD60020F0B5002639
:102FA000094D0746344605EBC4004068B84204D1D9
:102FB00055F83460204600F009F8641CE4B2102C87
:102FC000F1D33046F0BD00008CD600200021421C19
:102FD00008D0054A002352F8301042F8303002EB96
:102FE000C0004360084670478CD6002030B4D388B8
:102FF00054881B1B5B1C1BB2012B09DB93881488B4
:103000001B1B5B1C1BB2012B02DB036930BC184786
:1030100030BC704738B50446382115F062F8FEF729
:1030200027FD0090BDF8000024F8040FFEF720FDF6
:103030000090BDF800006080FEF753FC0090BDF8E2
:103040000000E080FF2525720220A072FEF749FCF7
:103050000090BDF800006083FEF743FC0090BDF8CF
:10306000000020850748206104F8015CA57584F8FC
:103070002650A57784F83250E07F20F03E001E30C5
:10308000E07738BDD00605082DE9F04FC7B083467C
:10309000DDE95065087B984614460F4602287DD925
:1030A000B7F90200002879D0AE4277D01AB2814633
:1030B0009246404500DD914601A8FFF7ABFF787BC3
:1030C00000F003008DF80600B86840B100208DF8CC
:1030D0000700B8680590387B8DF81E0005E0387B46
:1030E0008DF807003888ADF808002188A8F10102A2
:1030F000A1EB0803ADF8F8306188A1EB0800ADF84A
:10310000FA0021881144ADF8FC10B4F802C0ADF803
:1031100000316244ADF80411ADF8FE20ADF80201B3
:10312000ADF80621B7F802C06344ADF80031B7F836
:1031300002C060440FFA80FCADF802C17888081A1A
:10314000ADF804017988C01A511A4FF0FF3231925C
:103150000022401C09B200B2ADF8061142920028CC
:1031600013DDA1EB0C00401C00B200280DDD012393
:1031700047F6FF7240A932A8FFF77EFE0120429079
:10318000002132A8FFF71EFA3190002347F6FF72A4
:103190003EA938A8FFF770FE002100E028E038A81B
:1031A000FFF710FA439006F5B470A84205D005F574
:1031B000B4714FF4B4708E4220D147F6FF70ADF871
:1031C00004003EAA01A95846FFF710FF4398FFF7F5
:1031D000FDFE3198401C02D03198FFF7F7FE38A869
:1031E000FFF7C4FB4298002802D032A8FFF7BEFBCD
:1031F00047B0BDE8F08FA6F5B476B6B28642FAD2F3
:1032000002E0A5F5B475ADB28542FAD228B2459078
:103210000090B4F90220B4F9001033B20FA844931F
:10322000FFF72CFB00210FA8FFF7CCF94690B54221
:1032300003D9A81BC0F5B47000E0701BDBF80810C0
:1032400000913C282ADDB8F10A0F27D95A20B6FB95
:10325000F0F1B5FBF0F000F00300ADF8B40001A808
:10326000ADF8ACA0ADF8B05001F003012E902A9457
:10327000ADF8AE60ADF8B210ADF8B6903EA8CDE9AD
:103280002F0B2AA8FBF7CEFF2AA8FCF793F82AA851
:10329000FCF75FF92AA8FCF74AFA04E03EAA01A964
:1032A0005846FFF7A3FE0FA8FFF760FB38A8FFF70B
:1032B0005DFB429810B132A8FFF758FB4698FFF724
:1032C00085FE4398FFF782FE3198401C02D031986A
:1032D000FFF77CFE787B40078AD509F0FF022AAB16
:1032E00051464498FDF79AFDBDF8A80021882AAA06
:1032F0000844ADF8A800BDF8AC0021880844ADF83A
:10330000AC00BDF8AA0061880844ADF8AA00BDF879
:10331000AE0061880844ADF8AE0042A8009906F0FE
:103320005EFE42ADC0B1002347F6FF722AA92CA869
:10333000FFF7A2FD00212CA8FFF744F906465846E6
:103340003EAA01A9CBF80850FFF750FE3046FFF720
:103350003DFE2CA8FFF70AFB09F0FF022AAB5146FD
:103360004598FDF75BFDBDF8A80021882AAA08440E
:10337000ADF8A800BDF8AC0021880844ADF8AC0059
:10338000BDF8AA0061880844ADF8AA00BDF8AE00F7
:1033900061880844ADF8AE0042A8009906F01FFE0F
:1033A000C0B1002347F6FF722AA92CA8FFF764FDDD
:1033B00000212CA8FFF706F904463EAA01A95846A9
:1033C000CBF80850FFF712FE2046FFF7FFFD2CA8B0
:1033D000FFF7CCFA0098CBF8080009E770B514465F
:1033E0000D460646FAF738FA224629463046BDE829
:1033F0007040FAF700BC7CB50446087E0D460228F2
:103400000ED9A2686846296806F0E9FD002807D0B1
:10341000626B0AB120469047626D2946204690476C
:103420007CBD2DE9F04FCD6889B00C46804615B1C2
:10343000207C00286ED0207C012800D10025D8F8FF
:103440000400FEF7C2F90790D8F8082005A8216803
:1034500006F0C5FD00285DD0F9F7EAF9834600685B
:10346000D8F80090C16951BB007C400611D4D8F84F
:103470000400BDF91410B0F90020B0F90200891A57
:10348000BDF91620121A079800FB021109EB410042
:1034900014E0D8F80410BDF91630B1F90200B1F902
:1034A0000010181A079B584300EB400000EB09027C
:1034B000BDF91400401A00EB400010448146D4F8D6
:1034C00004A05FEA0A0013D02068FEF77EF90646E2
:1034D0002068BDF91410B0F90020B0F90200891A73
:1034E000BDF91620121A06FB02110AEB410A00E090
:1034F000002645B3DBF80000007C000710D46069AB
:103500000CF04FFD0246002108E0685C802802D9DB
:10351000FF2001E035E000206854491C9142F4DBB3
:103520006069FEF752F907466069BDF91410B0F9F9
:103530000020B0F90200891ABDF916202944121A98
:1035400007FB021500E00027D8F804004188008836
:1035500049420AB2404201B205A80CF05BFDDBF81B
:103560000000C069C8B160680028207E0CD001A9A5
:10357000009681E8A100534605A94846079A05F040
:10358000B1F809B0BDE8F08F8DE8A100A36805A9E6
:103590004846079AFDF7F3F9F3E7607E78B1616872
:1035A0000029217E23D00096CDE90370CDE90115D5
:1035B000534605A94846079A04F066FEE1E76068AD
:1035C0000028207E0AD001A9009681E8A100534678
:1035D00005A94846079A04F011FFD2E78DE8A1003B
:1035E000A36805A94846079AFDF726F8C9E7CDE97B
:1035F0000270CDE90015A36805A94846079AFCF7B3
:103600007DFFBEE72DE9F0471F469146DDE9082A18
:10361000B7F9024014FB09F001EB4001B7F90000D3
:103620000A9B01EB4005B3F9021001FB0AF102EB22
:103630004101B3F9002001EB4206B988081A401C89
:1036400000B24FEA40080AE028463146424614F0EC
:1036500020FD641C05EB490506EB4A0624B2B7F9C8
:103660000600A042F0DABDE8F0872DE9FF4F9BB0DD
:103670000C461B981546DDF8A0B0816817A8FEF728
:1036800062F817A8FFF78EF91390208818B96088A0
:10369000B0F5807F01D0012000E00020149006A842
:1036A0001C2114F01EFDE07A8DF83000207B0EAF57
:1036B00000F00F008DF831000697DDE9131001438B
:1036C0004FF000062CD1BBF1040F06D0BBF10E0F5A
:1036D0000AD0BBF1140F21D022E0A07A00BB1E98C3
:1036E00006A9CDE9065013E01B9829468268684672
:1036F00006F075FC00280ED01E9807960B950990D1
:103700002089ADF8200002208DF8280006954BE0B6
:103710001B98FFF770FE1FB0BDE8F08FA07A78B35A
:103720001B9880680188ADF838108088ADF83C009F
:103730001B9880684088ADF83A001B988068C08864
:10374000ADF83E002846FEF746F815902846FEF7ED
:103750001EF812900EA8FEF71AF881460EA8FEF782
:103760003AF88046F9F764F80DF0E0FB06460EA83B
:103770000CF017FC01464046B14217D84E4617E000
:10378000FFE72846FEF727F804462846FDF7FFFF27
:103790001E9907910A46610001FB002009900695D9
:1037A00002200B958DF8280006A9B1E7B6FBF8F6C4
:1037B0007043169040000FF0FBFE824616980FF003
:1037C000F7FE8146099002208DF82800BDF93E00E1
:1037D0000D90761EBDF83A00199630440B97CDF83F
:1037E0001CA0ADF83E00BBF1040F05D1208818B92C
:1037F0006088B0F5807F01D0022000E001208DF8C4
:103800002800C0E00EA910A8FDF79DFF688840427F
:1038100002B22888404201B210A80CF0FBFB1498B9
:1038200070B1CDE9024BCDE904A915991298CDE903
:10383000000110A9159B1E9A1B9800F0D7FD0BE004
:10384000CDE9014BCDE903A915980090024610A8D7
:10385000129B1E99F9F714FEA07A022861D92189DA
:1038600089B2C1F3C40212FB00F2ADF808204A0786
:10387000920E02EB513212FB00F2ADF80A20C1F3B6
:10388000042111FB00F1ADF80C10C0F1FF00002382
:1038900044E00AEB43073988ADF80410BDF8042072
:1038A000BDF80810C2F3C40616FB001101EBC116E7
:1038B00006EBC131BDF80060C1F3C45161F3C70626
:1038C0005107890EBDF80AC001EB523111FB00C14E
:1038D00001EBC11C0CEBC13C4FEA9C6C6CF3020683
:1038E00001EBC11C0CEBC131C1F3C25161F34F3686
:1038F000BDF80C10C2F3042212FB001101EBC1123F
:1039000002EBC131C1F3C45161F30C26ADF8006084
:10391000B1B20091BDF8001039805B1C16998B4242
:10392000B7D31398E0B14E46BDF93A7014E0BDF933
:10393000381043463A463046FEF7F6FF10B10228EB
:1039400004D006E03046414614F0CBFB02208DF84F
:1039500028007F1C46443FB2BDF93E00B842E6DA7B
:1039600006A91B98FFF747FDBDF83E001999401CBA
:10397000ADF83A00084400B20D99ADF83E00884217
:1039800001DDADF83E10BDF93A100D9881427FF788
:1039900039AF48460FF058FE50460FF055FEBAE6D4
:1039A00010B50C460846582114F09BFB1048606186
:1039B0001048206110482063104820621048A06120
:1039C000104860621048A0621048E06210486063CE
:1039D0001048A0631048E0631048206410486064F9
:1039E0001048A064104860652C20E06410BD000001
:1039F0008930010831410108DD330108FB3B010832
:103A00006B360108113D0108B53E01086941010806
:103A1000EB43010805360108FF3A01082D3A010879
:103A20007F3A0108F53B0108233401082DE9F041F4
:103A300017460C460646F8F7FBFE0546F8070ED07B
:103A4000A16A606921F0004114F04BFBA06A40F0CC
:103A50000041A1622868016941F0400107E0A06AC5
:103A600020F00041A1622868016921F04001016154
:103A700060690834C6E90004B460BDE8F081FEB5B1
:103A80000546006802900098164620F0E00000907D
:103A90000C466868FDF7A5FE009960F3942100913B
:103AA0006868C1884088081A0099401C60F35F511B
:103AB0000091A06A002801DA052000E0042060F3EC
:103AC00004010091206A2860E0696860A069A8602C
:103AD000F8F7AEFE006894F824206B46016962F3A3
:103AE0008611016104F1080231462846FEF7D4F937
:103AF000284600F096FC68460EF0A6F8FEBD70B5AC
:103B0000064615460C46D00701D0002070BDA80718
:103B100043D5A06A00F0004000F5C040A0622046F6
:103B20000CF03FFAA16A400021F00042824202D923
:103B300060F31E01A162A06A20F000400FF00AFDB0
:103B40002146606168B9A06A00F0004000F540605D
:103B5000A06220F000400FF0FDFC214660610028CB
:103B6000D4D00846D0E900128160E2606188E1812A
:103B7000A1892089081A401CA16A00B221F00041E5
:103B800000EB400291FBF2F12182A16A21F0004199
:103B900091FBF0F0411061822AE00846D0E9001262
:103BA0008160E2600CF0FDF94100A06A61F31E0043
:103BB000A06220F000400FF0CDFC6061A16A21F00E
:103BC000004114F08EFAA06A05F0010565F3DF707C
:103BD000A0626069002899D0306004F1080070602C
:103BE000B060F8F725FE0068016965F38611016190
:103BF000204670BD48690FF039BDF0B51D46074637
:103C000097B014460E46086800232A460FA90DF007
:103C1000D6FAF0B3BDF84420002A3FD0BDF842C028
:103C2000BCF1000F3AD02088BDF84610084401B21C
:103C3000ADF84C10306803894089181A638801EB8D
:103C40000C041844BDF84830801AC01A03B2ADF80D
:103C50004E30B868B0F900C064451FDBB0F90440CD
:103C6000A1421BDC9918B0F90220914216DBB0F991
:103C70000600834212DC29460F980DF09CFA0028BA
:103C80000CD00F99097B890708D10FAB13AA3146D5
:103C900000E005E000903846FAF7E6FD17B0F0BD09
:103CA000202DFBD3A5F57840FF38F7D0A5F50050BF
:103CB0000C38F3D02088BDF84610BDF848200844E1
:103CC00001B26088104402B2BDF84400104400B252
:103CD0000090BDF84200084403B214A80CF0A7F904
:103CE00001A8FFF797F902208DF807008DF82E0044
:103CF0008DF83A008DF81E00B089ADF82200012041
:103D0000ADF824003B6914AA01A938469847C5E7D5
:103D10002DE9F0471546B1F9022092B01C460E4637
:103D20008146002A7ED0307A02287BD9B5F900106E
:103D3000B4F90000814205D1B5F90230B4F902703E
:103D4000BB426FD0814200DA084602EBD271A0EB91
:103D50006100ADF84000B5F90000B4F90010B6F903
:103D60000220884200DC084602EBD27100EB6100C1
:103D7000ADF84400B5F90200B4F90210B6F902201A
:103D8000884200DB084602EBD271A0EB6100ADF87F
:103D90004200B5F90210B4F90200B6F902208142DE
:103DA00000DD084602EBD27100EB6100ADF8460081
:103DB00010A90846D9F8082006F011F9002875D096
:103DC00010A9D9F808A0C9F80810B5F90200B4F98B
:103DD0000210884206D123462A4631464846FAF761
:103DE000A7FE0EE0B5F90000B4F9001023468842A2
:103DF0002A463146484602D1FBF706F901E0FAF7B8
:103E000055FF707A010701D440074DD56846FFF78A
:103E100001F93088ADF8040047F6FF70ADF80000F6
:103E2000307A00E042E08DF80300B6F90200471056
:103E300040F3000000F10108707A400718D5288887
:103E40000EAAC01BADF838006888C01BADF83A0058
:103E50002888C119A1EB0800ADF83C006888C11999
:103E6000A1EB0800ADF83E0069464846FFF7BEF8F2
:103E7000707A000718D520880EAAC01BADF838004C
:103E80006088C01BADF83A002088C119A1EB08007A
:103E9000ADF83C006088C119A1EB0800ADF83E0008
:103EA00069464846FFF7A2F8C9F808A012B0BDE875
:103EB000F08700002DE9FF4F8BB01F461646032BFD
:103EC0007ED3002E7CD0B8000FF072FB04007BD0B4
:103ED00000253068206028467A1E15E006EB800138
:103EE00036F92030B1F904C0634505D1B1F902308B
:103EF000B1F906C0634505D004EB850309686D1C64
:103F00001960ADB2401C80B29042E7DB06EB87003F
:103F1000B6F9001030F9042C914205D1B6F902101F
:103F200030F9022C914206D004EB850150F8040CC4
:103F30006D1C0860ADB2032D43D37C48D0E900105E
:103F4000CDE90210002027E0BDF9081034F9202047
:103F5000914200DB1146ADF8081004EB8003BDF977
:103F60000A10B3F90220914200DB1146ADF80A10A5
:103F7000BDF90C1034F92020914200DC1146ADF857
:103F80000C10BDF90E10B3F90220914200DC11466D
:103F9000401CADF80E1080B2A842D5D30B9802A9F0
:103FA000826805A806F01BF858B10B9805A90026F1
:103FB000806809900B988160B4F90220012010E01C
:103FC00002E020460FF040FB0FB0BDE8F08F04EB9D
:103FD0008001B1F90210914201DA0A4606B2401C92
:103FE00080B2A842F3D32C2105FB01F00FF0E0FAD8
:103FF0008346B2460490D1464FF00008701E00D5AB
:1040000028446A1E09F101010792914200DD002156
:1040100034F8203034F8262034F821709B1A04EB51
:104020008000BA1A478804EB860004EB81014088BF
:1040300049883E1A081A0021089116FB02F110FB6C
:1040400003F0814267DA0120089001E00898E8B3A4
:1040500007980AF10106864200DD0026B9F1010742
:1040600000D52F4404EB860004EB8A01B0F902006E
:10407000B1F90220904216DB12D034F9263034F91F
:104080002A108B420CD04FF0010CCDE9000C5846A1
:10409000FEF726FD58460499FEF794FA0BF12C0B17
:1040A00008F10108B246A84523D004EB870004EBD1
:1040B0008901B0F90200B1F90220904217DB13D058
:1040C00034F9273034F929108B4200E023E00BD07B
:1040D0000026CDE900065846FEF702FD5846049931
:1040E000FEF770FA0BF12C0B08F10108B946A84550
:1040F000ACD3DDE90B0102AAFEF778FF0498FEF7C6
:104100004DFF04980FF0A0FA20460FF09DFA0B998E
:104110000998886058E7BAF1010600D52E4407983F
:1041200009F1010787429DDD00279BE7489E0108B2
:1041300070B514460D460646FBF71AFC2246294682
:104140003046F9F789FB224629463046F9F753FDF8
:10415000224629463046F9F740FE22462946304697
:10416000BDE87040FAF7FBBF2DE9FF4F99B00F464D
:1041700028984FF480314FF00A0BB0F90000DDE9C8
:104180002A6540420F9028984088B1FBF0F00F99C3
:104190000E9091FBFBF4289804F1010A40681290FC
:1041A000604200EB800001EB400920B211F03EF9C3
:1041B00001900FFA8AF011F039F95A34009020B2C8
:1041C00011F034F980460AF15A0000B211F02EF9CC
:1041D000019AC9F10A0101FB02F4009B01FB08F1FD
:1041E00000FB091103FB094391FBFBF093FBFBF27E
:1041F0000D9050110C900D9840110D90BDF9480094
:1042000000021090BDF94A0000021190B888398868
:10421000401A401C04B2F8887988401A401C00B249
:104220001790002049E014A80090B7F9021013ABD2
:1042300001EB0A02B7F9001008A805F00EFD16A858
:104240000090B7F9021015AB01EB0A02B7F90410A0
:1042500008A805F002FDDDF84CC01598149AA0EBF3
:104260000C0816980021831A0846012C07DD601EF1
:104270004FEA082191FBF0F11B0293FBF0F0289B21
:1042800080320CF1800C1B7DDB07299B1CD00DF1CB
:104290000C08CDF800C088E85100CDE90121CDE936
:1042A0000653DDE91B01DDE92623F8F705FC0AF1D9
:1042B000010006EB4406254400B217998246884265
:1042C000B1DB1DB0BDE8F08F042B4BD0052B10D017
:1042D000062B47D0142BEAD1DDE91B38CDF810802E
:1042E000DDE926EBCDE90010CDE902C2B1460020A0
:1042F00078E0DDE91BE3CDE900100393269B0293F0
:10430000B146E346DDF89C80002028E00099414357
:104310000BEB21230199414302EB21211B124FEAB0
:10432000212C08D403998B4205DABCF1000F02DB83
:1043300002998C4502DB002129540EE00CFB083366
:1043400003EB430303EB0E010B7891F801C003EB81
:104350000C2329F810308B782B54401C00B2A0425B
:10436000D4DBA4E70DF10C08CDF800C088E85100BB
:10437000CDE90121CDE90653DDE91B01DDE9262365
:1043800004F0CBFE93E70099029A414302EB21220D
:104390000199DDF80CC041430CEB212112124FEAC8
:1043A000212107D4DDF810C0624503DA002901DBC2
:1043B000714502DB0021295412E001FB0B2C03EBB9
:1043C0004C0C09EB4008BCF800C0A8F800C00BFB7F
:1043D0000EFC03EB4C0C624401FB0B210A782A54BF
:1043E000401C00B2A042CEDB61E770472DE9F043EC
:1043F00087B08946DDE91251DDE91076DDE90E8CE2
:1044000070B1C46A002C08D0CDF80080CDE9045109
:104410000396CDE901C74946A04707B0BDE8F08340
:10442000FEE7416B002900D00847704710B51749D7
:10443000174822F0D6FC38B11449154821F0EBFE9C
:104440001249134822F0CDFC12480CF089FF1148A4
:10445000432101704FF4007141800F4981600F4981
:10446000C1600F4901610F4941610F4981610F49E5
:10447000C1610F4901620F4981620F4941620449DC
:10448000C162BDE810400CF06FBF0000186C04085A
:10449000347B00207CD40020250B0108550A01083C
:1044A0006D0B0108BD0B0108850B0108A50B010868
:1044B0008D0A0108710A0108B50A01082DE9FC41BD
:1044C0008646807815460C4610FB04F000128242A6
:1044D00003DCBEF80000BDE8FC819EF808C00EEBCE
:1044E0008C0212F8023C13FB04F31B129D4202DB08
:1044F00032F8040CEFE70022012324E00EEB8307DF
:10450000BF7817FB04F73F12BD421ADC0EEB83079E
:1045100037F8040DADF804000198FDF783FA06465C
:10452000B888ADF804000198FDF77CFA0146B87828
:1045300010FB04F0BA79001212FB04F2C0EB222245
:1045400003E05B1CDBB29C45D8D8E2B3281A00B26A
:10455000C0EB002090FBF2F0C0B2C0F1FF02C1F34B
:10456000072313FB00F3C6F3072414FB023303EB0A
:10457000C31404EBC334BDF80050230F63F30205EA
:10458000C1F3074313FB00F3C6F3074717FB0233DE
:1045900003EBC31707EBC3339B0E63F3C705C9B225
:1045A00011FB00F0F1B211FB020000EBC01101EBB6
:1045B000C030800E60F30C25600E60F34F35ADF80F
:1045C0000050A8B287E7FFE7FEE74168002901DA5B
:1045D0000FF04CB870470000FEB50546407A16460D
:1045E0000C4640072ED0224F387820B9002000F02A
:1045F00043F801203870687A00F00700022817D0CD
:10460000304680EA640068400190002000906A46CD
:1046100001A91848FCF7B2FC01280BD0324621460C
:104620002846F8F71BF9009000280BD0002418E06A
:104630002046E6E700980422416802EBB1714FEA98
:10464000B1014160FEBD22462846FFF737FF0290C8
:104650000098BDF80810806800EB4400641C0180DD
:1046600024B20098B0F90E10A142ECDCFEBD0000AF
:1046700078520020330A010870B5094D04462868B5
:104680000EF0F4FF20460EF065FF2860054DA8608F
:1046900020B1214613F025FD6C6070BDFEE70000DF
:1046A0002053002078520020014600200F290AD212
:1046B000DFE801F009090909080A080C0E10120CBC
:1046C0000E1012001020704718207047012070470C
:1046D00002207047042070470820704701460020E0
:1046E000891E0D2909D2DFE801F00708080708072D
:1046F000070707070707070001207047014600204A
:10470000032901D0062900D101207047032130B1CF
:104710000078A0F120015F2903D8012070470846E6
:104720007047802801D302207047002070470000A6
:1047300038B5174C2078002829D10EF0ADFFF8F7D6
:104740007FF805F001FEF7F775FD05F003FEFDF7B4
:10475000EFFBF7F771FF4FF4B4710E4806F01FF945
:104760005C210D4806F01BF9F8F768F805F0D8FE53
:104770000A4800909DF80000112802D0002010B1D6
:10478000FEE70120FBE70CF0D6FC0120207038BDCD
:104790005C520020DCD40020E8D4002044332211F5
:1047A0002DE9F0410A4C07460A4D60680E46401C50
:1047B000C100606028680EF07DFF286038B1616834
:1047C00000EBC10040E902760846BDE8F081FEE753
:1047D000645200201053002013F05BBC13460A46BD
:1047E000194613F077BC13F07CBC13F07ABC13F0BD
:1047F00078BCFF2213F06EBCFF2213F06BBC2DE9D6
:10480000FF410C46074602F043F90646E00702D096
:10481000384602F0E5F8F8692043F861E00711D066
:104820000221384601F056FE60B1384600F016FF0E
:10483000050007D00CF0AAFF28460DF027F808B1B4
:1048400002F0CEF8384602F023F9B04202D114F05B
:10485000C07F07D0384600F041FF02F052F93846D9
:1048600002F04FF9E0060CD502AA6946384601F07D
:104870009CF86946384602F0D6F802A9384602F09C
:10488000D2F8BDE8FF81028C11438A4201D003F0C7
:10489000A2B870472DE9F047174688464FF6FF79D2
:1048A000054600234A46394605F004F9698C002480
:1048B0000426C1F30513EA6808E006EBC4001058AB
:1048C0005FEA801C01D4C00102D5641CA342F4D865
:1048D0004FF0806000EBB1204FEAB0506884C0F325
:1048E0000510C10010460EF0E5FEE860688C6FF020
:1048F0000703C0F3051009E0E96803EBC00C01EB06
:10490000C0026144D1E900C1C2E900C1401EA04219
:10491000F2D8E868082100EBC40013F0E2FBE96874
:1049200041F83480E86806EBC401425867F3170287
:1049300042504A4639462846BDE8F04702F0E4BCFA
:1049400010B504468068002813D10B484168491C03
:1049500041601C200EF0FEFDA06058B11C2113F038
:10496000C0FBA1680F204876A068017E41F00301DA
:10497000017610BDFEE700005C5200202DE9FC41ED
:104980000D460746012101F099FD002850D1384617
:1049900000F0A8FE044600F043FE06460CF0F6FACE
:1049A000A0420ED030460CF0F9FAA04209D03046B1
:1049B0000CF0DAFAA04204D030460CF0CDFAA04256
:1049C00036D14FF400263146384601F07EFD18BB43
:1049D0003846F7F746FD044607F114016846FCF730
:1049E0008EFEBDF800002946001BADF80000BDF8A2
:1049F00002006A46001BADF80200BDF80400204426
:104A0000ADF80400BDF806002044ADF806000846E5
:104A100005F0E5FA00280CD000230122294638468B
:104A200001F07AFC38461DE0012101F047FD10B18C
:104A30000020BDE8FC813146204601F046FD80B9EA
:104A4000D4E90501CDE90001002301226946204691
:104A500001F062FC29466A46084605F0C0FA0028C3
:104A6000E7D0204600F03AFE0400DDD10120E0E767
:104A70002DE9F0410E460746002401F019FC05001F
:104A800035D03146384601F007FC02282FD905EB16
:104A9000D570012101EB60053146384601F002FC7A
:104AA00028440FFA80F83146384601F0E9FB054604
:104AB0003146384601F0EAFB002D01DD294600E0D1
:104AC0006942002801DD024600E04242914205DDD4
:104AD000002D01DD284604E0684202E0002800DCE9
:104AE0004042404400B2002800DA204604463146E5
:104AF000384601F042FB05000ED03146384601F041
:104B000030FB022808D93146384601F030FB2844F2
:104B1000A04200DB044624B238463146692201F047
:104B200062FB05B2384631466A2201F05CFB00B2F6
:104B3000854200DD2846002801DD204404B22046DD
:104B4000BDE8F08170B50D4606465B2201F04BFBD7
:104B5000C4B230462946162201F045FB04B90124AF
:104B6000204670BD002803D00068884201D1012092
:104B700070470020704700002DE9F04107460546C8
:104B80000E464FF00008354800E02D68ADB1A96928
:104B90000142FAD0A869C0F30F1528460EF0DAFCDE
:104BA000041E31D0294613F09CFAC4E90076012591
:104BB0006F1F26B1B06880B333E04546EDE70CF0D7
:104BC0009DF906001CD0F26802B3706A401C810097
:104BD000706210460EF06EFDF060716A07EB8101A5
:104BE0004450A4F81480A4F8168000200CF09EF91C
:104BF000401E208300200CF0DFF9401E608322E07D
:104C000020460EF033FD0020BDE8F08104200EF0B8
:104C1000A1FCF06004607562E3E7FFE73046FFF750
:104C20008FFEB068016881B14168491C4160B0687D
:104C3000890000680EF03EFDB1680860B1684968FF
:104C400007EB810144502046DEE704200EF082FC91
:104C5000B16808600460B0684560F4E7F0FF0F00D9
:104C600070B5054601F04DFF002000F093FA28468C
:104C700010F036FA284600F06FF8012000F08AFAAA
:104C80004FF6FF724FF47021284602F03DFB284694
:104C900002F022FB0CF0EEFD030007D0284601F0E5
:104CA000E9FE18B1294618460CF01CFD284600F014
:104CB00015FD04000DD02A4622210CF011FA2A46D7
:104CC000232120460CF00CFA2846BDE8704001F084
:104CD00087BE70BD7FB50C46064601F0D9FE05467D
:104CE000E0060CD502AA6946304600F05EFE694631
:104CF000304601F098FE02A9304601F094FEF069BA
:104D0000A043F061E0070ED0304601F069FE304666
:104D100001F0BEFE38B1304600F0E0FC01F0F1FEDB
:104D2000304601F0EEFE304601F0B2FEA84202D15C
:104D300014F0C07F07D0304600F0D0FC04B0BDE8CE
:104D4000704001F0DEBE7FBD028C22EA01018A4282
:104D500001D002F040BE704770B50568044628686F
:104D600018B120602046FFF7F7FF25606A682846E3
:104D7000002A03D02146BDE87040104770BD2DE9E0
:104D8000F0414D680C46EDB1284600F02DFD064679
:104D9000284600F0F5FD074628460021102201F0C4
:104DA00022FAE98A12220844C01BE082401E608376
:104DB0002846002101F017FAA98A0844801BA08226
:104DC000401E208341F20200E061002D05D043F235
:104DD0000200E06143F20230E06140F0740040F410
:104DE0000060E06102D040F40040E061BDE8F08185
:104DF00010B501460348FFF7BFFE0446FFF730FF3A
:104E0000204610BDEC9C01082DE9F041074601F059
:104E1000E7FD384600F062FC4FF00004050026462E
:104E200008D1384600F0FCFB040018D02069B842D5
:104E300000D10126384603F0E1FC65B1284602F0B6
:104E400027FD0022222128460CF04AF900222421C5
:104E500028460CF045F9002E01D000202061BDE865
:104E6000F081000070B50C46084605F057FA0020A6
:104E700000F090F92046144A002102F01BFB0120AB
:104E800000F088F900212046FCF73AFB204600F0AC
:104E9000E5FB10B120460CF03CFDA068002811D0C5
:104EA0000068002518B10EF0E1FBA0680560A0685D
:104EB000C06818B10EF0DAFBA068C560A0680EF0FB
:104EC000D5FBA56070BD0000FFFF0F002DE9F04786
:104ED000A2B080460CF0B9F8044640460CF0F3F856
:104EE000012700260546122C72D0DFF89492152C6B
:104EF0006CD0182C7AD140460CF0ADF882460146B1
:104F00002846FAF7E1FC0021284601F0E0F850B10C
:104F100005F59070FEF742F8040004D0FDF726FD79
:104F200020460EF091FB0021284601F0BCF8002835
:104F30005CD06846FEF76EF88DF803608DF81A6055
:104F40008DF82A608DF836606A460021284601F007
:104F5000E9FB0021284601F0C7F9804600212846D8
:104F600001F0BCF9044605F1140120A8FCF7BEFBD2
:104F7000BDF88010A1EB0800BDF88410ADF88000EA
:104F800001EB0800ADF88400BDF882005146001B1B
:104F9000ADF88200BDF886002044ADF886000EA86A
:104FA00000F0F0F820A81B96CDE91070CDF83C90E9
:104FB000CDF848D00EAA1A2128460CF091F820AA64
:104FC00069465046FEF712F8D4E001E055E00DE0E6
:104FD00040460CF076F804460078022806D00021FE
:104FE000284601F074F820B10220207022B0BDE8FC
:104FF000F0870021284601F03DF98246002128462D
:1050000001F072F981460021284601F067F98046D7
:1050100005F114016846FCF769FBBDF80010524623
:10502000A1EB0900BDF80410ADF8000001EB090088
:10503000BDF80210ADF80400A1EB0800BDF80610A1
:10504000ADF8020001EB0800ADF8060069466068A3
:1050500004F0EDFF68B10021284601F018F8FD28A2
:1050600007D328460021602201F0BDF8C0B2FD2818
:1050700001D22770BAE72670B8E740460BF0EBFF85
:1050800080466846FDF7C6FF0021284601F00BF870
:1050900028B19DF8230040F001008DF823006A46F6
:1050A0000021284601F03EFB0021284601F01CF9B2
:1050B00007460021284601F011F9044605F11401C4
:1050C0008A4620A8FCF712FBBDF880004146C01BB1
:1050D000ADF88000BDF884003844ADF88400BDF818
:1050E0008200001BADF88200BDF886002044ADF8B8
:1050F00086000EA800F046F820A8CDE91060CDF893
:105100003C90CDF848D00EAA1A2128461B960BF0E9
:10511000E7FF0021284600F0DAFF20B1BDF80000CB
:1051200008B1012700E00027049C07B1049620AADB
:1051300069464046FDF75AFFE7B118200EF038FAED
:105140000746BDF9002000235146FDF795FE05F501
:1051500090713846FDF736FA64B18DF803608DF82A
:1051600022608DF82A608DF8366020AA6946404694
:10517000049427E70EAA1B2128460BF0B1FF35E760
:10518000EC9C010870B50D460446482112F0A9FFB9
:10519000256070BD01490870704700006C52002006
:1051A0002DE9FF41884608460BF04FFF0446404674
:1051B0000BF04FFF0546012C23D0082C23D0032CE5
:1051C0003ED02A2C3ED00D2C4CD00E2C7DD0092C5C
:1051D0007CD00A2C7BD00F2C7AD0292C79D0222C91
:1051E00078D0242C77D0132C76D0152C03D0182C03
:1051F00001D0122C34D104B04046BDE8F041FFF795
:1052000065BE2021FAE02021FFF79EFD40460BF00D
:1052100033FF0DF05EFB002822D10821284601F063
:105220004DF900281CD095F820004FF00101C0076F
:10523000284602D0FFF788FD30E0FFF724FB2DE081
:105240002021F8E000F05CF90646002406E0A8689A
:10525000006850F8240001F054FC641CB442F6D3FA
:10526000BDE8FF81082101F029F9F8B140460BF0B3
:1052700028FF0478132C06D0112C04D0142C07D04E
:10528000122C05D008E001212846FFF7FCFA03E0C4
:1052900001212846FFF758FD0A2CE1D004B028462A
:1052A000BDE8F04100221C210BF01ABF4FF4016150
:1052B000284601F003F90028D2D0284601F0CDFBA2
:1052C0000028CDD10027284607E06DE095E09AE060
:1052D000B0E0B5E0D1E0F2E0F6E000F085FA064695
:1052E000284600F0E1FA044640460BF0EAFE00785A
:1052F00012281BD011280CD013282BD01428AFD182
:10530000284600F049FA800703D0002E38DC002C34
:1053100036DC284600F0A7F90446284600F03EFB9C
:10532000E11704EB9171A0EBA1000BE0284600F01F
:105330009AF90446284600F031FBE11704EB91711D
:1053400000EBA10001B204B03A462846BDE8F041A6
:1053500002F088BA284600F01FFA8007E6D0002E37
:1053600001DC002CE2DD284601F089F804462846DD
:1053700000F00DFBE11704EB917100EBA1000BE0D5
:10538000284601F07CF80446284600F000FBE117AF
:1053900004EB9171A0EBA10001B204B03A4628469B
:1053A000BDE8F04102F048BA4FF4806101F086F8A0
:1053B00018B10121284602F022FA284600F04EF9E1
:1053C0000CF05EFA064602240DF04EFA10B9404683
:1053D0000BF052FE0DF089FA022801D0042800D10A
:1053E00006241EB144F00801284607E0214628465D
:1053F000FFF749FA082128461DE0402104B0BDE826
:10540000F041FFF740BA4021FFF79EFC284600F02C
:10541000F2FD02287FF424AF02AA6946284600F074
:10542000C4FA6946284601F0FEFA02A9284601F0AE
:10543000FAFA15E70E2104B0BDE8F041FFF784BC8D
:10544000002100F0FFFD04460021284600F04DFE3B
:10545000204302D0284601F054FB284600F050F8C3
:105460000646002406E0A868006850F8240001F011
:1054700048FB641CB442F6D3F2E60021012200F09E
:10548000B2FE06B228460021042200F0ACFE04B2AF
:105490000021284600F0D6FD07460021284600F0EE
:1054A00024FE384305D142F2D170864201D08442B5
:1054B000BFD104B02846BDE8F04101F022BB688CA2
:1054C00040F002006884F4E70021FFF7D1FA0146BA
:1054D00004B04046BDE8F0410BF022BE80680028D1
:1054E00009D0002902DA4268511803D443680A46F9
:1054F0008B4201D800207047006850F822007047A6
:105500008068002800D04068704770B50C4605469A
:1055100000F114012046FCF7F2F8A868002812D028
:105520002188808A081A2080A968A088898A08446E
:10553000A080A9686088898A401A6080A968E0888C
:10554000898A0844E08070BD70B50C46054600218C
:1055500000F0B1FD06462146284600F05BF8704297
:1055600002B2114620460AF048FD0021284600F00C
:1055700016FE2188084420800021284600F01BFEEA
:10558000A188081AA0800021284600F020FE61882A
:10559000084460800021284600F0F5FDE188081AE3
:1055A000E08070BD2DE9F0410646002100F00FFEBD
:1055B00005460021304600F0E6FD04460021304655
:1055C00000F079FD0746304600F04DF8401B001B07
:1055D000794200EB410000B2BDE8F0812DE9F041D5
:1055E0000646002100F0DBFD05460021304600F0B4
:1055F000E2FD04460021304600F05DFD07463046DE
:1056000000F03DFF401B001B794200EB410000B25F
:10561000BDE8F0810A4600F114011046FCF76FB8AE
:1056200010B5416809B100F05DF804460A4805F07C
:1056300099F90EE00022416A05E0C36853F8223070
:10564000A34208D0521C9142F7D80146024805F007
:105650009BF90028EED110BDDCD400208068002822
:1056600000D0806870471430FCF77FB870B50646EC
:1056700000F034F8051E08D0002408E02146284632
:10568000FFF72CFFB04201D1204670BD641C2846B4
:10569000FFF736FFA042F1D84FF0FF3070BDF0B4F5
:1056A000458C00240426C5F3051712E0C56806EBF7
:1056B000C40C55F80C505FEAC51C09D525F07F4590
:1056C0009D4205D1C06850F83400F0BC0EF080BF98
:1056D000641CA742EAD8F0BC00207047002800D024
:1056E0004068704700B50146FFF7F8FF0028FAD17F
:1056F000084600BD2DE9F047DFF8949080464C46FF
:10570000FFF7FEFE06460025DFF888A00FE0D8F878
:1057100008005146006850F82570384600F0D5FE64
:1057200020B9B7F91A00A04200DB04466D1CB5424F
:10573000EDD30021404600F050FD82460021404656
:1057400000F027FD06460021404600F0BAFC054661
:105750004C4505D0B8F81A00801B401B201A04B233
:10576000404600F051FC07464046FFF77CFFA0EBA7
:105770000A00801B694200EB4100391A404600F0E4
:105780000DF9081A00B2844200DD2046BDE8F0871A
:1057900001E0FFFF01000400806818B1407E00F0C6
:1057A0000F0070470F20704770B50C4605460C4936
:1057B000FBF7D6FE10B1806A404202E0284600F0B6
:1057C000E6F8208007492846FBF7CAFE10B1806A38
:1057D000404202E0284600F0E1F8608070BD000021
:1057E00041940108599401082DE9F84F064600211B
:1057F00000F03AFC012807D0B068002802D0008AE7
:10580000404200B2BDE8F88F0021304600F0D9FCDC
:1058100000900021304600F0C8FC8146002130464F
:1058200000F04FFC824641F6FF7B5C463046FFF7B6
:1058300067FE804600250EE0B0681949006850F800
:105840002570384600F041FE20B9B7F91400A04297
:1058500000DC04466D1C4545EED35C4506D0B28A9B
:1058600009EB0A001044001B04B200E00D4C304666
:1058700000F0D8FB0546304600F001FE0099411AC1
:10588000A1EB0901CAF1000001EB4000291A3046E2
:1058900000F07DF8084400B28442B3DD2046B1E751
:1058A0000100040001E0FFFF2DE9F047064600215A
:1058B00000F0DAFB01280AD0DFF8A09030464C4611
:1058C000FFF71EFE80460025DFF894A015E0B068C3
:1058D000002801D0B0F91000BDE8F087B06851464B
:1058E000006850F82570384600F0EFFD20B9B7F990
:1058F0001800A04200DB04466D1C4545EED3002194
:10590000304600F05EFC07460021304600F04DFCBA
:1059100082460021304600F0D4FB05464C4504D0B9
:10592000308BC01B401B201A04B2304600F07AFBBB
:105930008046304600F0A3FDC11BA1EB0A0069427E
:1059400000EB4101A8EB0101304600F020F8081AF5
:1059500000B28442C0DD2046BEE7000001E0FFFF48
:10596000010004008068002802D0007EC0F381009E
:1059700070478068002802D0007EC0F30110704795
:105980008068002802D0408A404200B27047806898
:10599000002802D0008A404200B270478068002888
:1059A00002D0408A404200B270472DE9F04F8DB0DE
:1059B00016460C464FF0FF37054600223B4611467F
:1059C000204600970AF033FB00223B461146304642
:1059D00000970AF02CFB1021284600F06FFD0028EC
:1059E00016D0284600F007FB070011D000200CF06D
:1059F00041FF8046022F08D010E00CF06AFFA84259
:105A000009D040460CF036FF8046B8F1000FF4D1C3
:105A10000DB0BDE8F08FB8F1000FF9D02846FFF7C0
:105A2000AFFF09902846FFF765FE0C902846FFF768
:105A3000DBFE07902846FFF737FF0B902846FFF75D
:105A4000ABFE8146002019F00C0F039014D0012FFB
:105A500010D0032F02D0022F07D00DE009980028A4
:105A600008DC0C98002805DC06E040460CF022FF1C
:105A70000C2801D101200390002002905FEA897078
:105A800014D0012F10D0032F02D0022F07D00DE029
:105A90000798002808DC0B98002805DC06E0404643
:105AA0000CF008FF032801D101200290DDE902017A
:105AB0000843ADD04FF480373946284600F0D4FA79
:105AC000012800D000200A903946284600F085FBC6
:105AD00001903946284600F05CFB0890394628467C
:105AE00000F063FB80463946284600F06AFB814699
:105AF00028460122394600F076FB0FFA80FB284643
:105B0000FFF7B1FD0090284600F0B9FC069003981D
:105B100000B158468246029800B158460590284682
:105B20003946212200F05FFBC0B2022808D2284685
:105B30003946312200F057FBC0B20228FFF468AFAB
:105B400009990098A02701440C98084400B20490D9
:105B50000398002870D004980028FBD0E88A708051
:105B6000688BF0800A9840B1A98A01EB0800308068
:105B7000ABF101010844B08007E0298BA1EB0900DB
:105B8000B080A0EB0B00401C3080DDE90001411A21
:105B90000898091A0598081A009909904843049929
:105BA00090FBF1F000B2039000200BF0ADF900EB98
:105BB0008001502000EB4100B0F5A07F0ADB0020FF
:105BC0000BF0A2F900EB8001502000EB410090FBAC
:105BD000F7F000E001200399884201DA084616E058
:105BE00000200BF091F900EB8001502000EB410008
:105BF000B0F5A07F0ADB00200BF086F900EB8001F6
:105C0000502000EB410090FBF7F000E001200999E3
:105C100000B2091A0AB2009B0499C91A09B20029F4
:105C20000BDCE98A019808447080698B0898091A8E
:105C30000598081A401EF08090E00C9B12FB03F3BD
:105C400093FBF1F1511A019AEB8A1144194409B2FC
:105C5000401E71800844F080B5F916200198104468
:105C6000814238DA708000200BF04EF900EB8001A1
:105C7000502000EB4100B0F5A07F0ADB00200BF0C4
:105C800043F900EB8001502000EB410090FBF7F05E
:105C900000E00120B6F902100844B6F90610884267
:105CA00019DD00200BF030F900EB8001502000EBF3
:105CB0004100B0F5A07F0ADB00200BF025F900EBD6
:105CC0008001502000EB410090FBF7F000E0012044
:105CD00071880844F080B5F91A200598B6F90610C5
:105CE000121A0898101A814238DDF08000200BF05B
:105CF0000BF900EB8001502000EB4100B0F5A07FD4
:105D00000ADB00200BF000F900EB8001502000EBD3
:105D1000410090FBF7F000E00120B6F90610081AE8
:105D2000B6F90210884219DA00200BF0EDF800EB0A
:105D30008001502000EB4100B0F5A07F0ADB00207D
:105D40000BF0E2F800EB8001502000EB410090FBEB
:105D5000F7F000E00120F188081A7080DDE9060103
:105D600001440B98084400B20590029800283FF4C3
:105D70004FAE05980028FAD0698B0898081AE08081
:105D8000A0EB0B00401C6080A88A2080288BA0809C
:105D90000698A0EB0801A1EB0901A1EB0A00019014
:105DA00006994843059990FBF1F000B2009000205D
:105DB0000BF0AAF800EB8000502606EB40004FF4F1
:105DC000A07B584509DB00200BF09EF800EB80001B
:105DD00006EB400090FBF7F000E0012000998842BC
:105DE00001DA084613E000200BF08EF800EB80008B
:105DF00006EB4000584509DB00200BF085F800EB6E
:105E0000800006EB400090FBF7F000E001200199D4
:105E100000B2091A0AB2DDE90513C91A09B200294C
:105E200016DCA98A0A9840B14144AAF1010008444D
:105E30002080298BA1EB090008E001EB08002080FD
:105E4000298BA1EB0901A1EB0A00401EA080DFE530
:105E50000B9B12FB03F393FBF1F1511A0A9A09B25F
:105E6000EAB3AA8A401E531808EB0A02991809B22D
:105E700021800844A080B5F914001044884233DD25
:105E8000208000200BF040F800EB800006EB400083
:105E9000584509DB00200BF037F800EB800006EBDB
:105EA000400090FBF7F000E00120B4F90010084436
:105EB000B4F90410884217DD00200BF025F800EB40
:105EC000800006EB400058450ADB00200BF01CF870
:105ED00000EB800006EB400090FBF7F001E039E0BA
:105EE000012021880844A080B4F90410B5F91820D5
:105EF00077E0A08000200BF007F800EB800006EBB5
:105F000040005D46A84272DB00200AF0FDFF00EB76
:105F1000800006EB400090FBF7F0B4F90410081A7B
:105F2000B4F90010884292DA00200AF0EDFF00EB8D
:105F3000800006EB4000A8425BDB00200AF0E4FF93
:105F400000EB800006EB400090FBF7F0A188081AF8
:105F500020805DE5AB8A4144194409B2401E21808E
:105F60000844A080B5F9142002EB0800814232DA1F
:105F7000208000200AF0C8FF00EB800006EB400004
:105F8000584509DB00200AF0BFFF00EB800006EB5C
:105F9000400090FBF7F000E00120B4F90010084445
:105FA000B4F90410884216DD00200AF0ADFF00EBC2
:105FB000800006EB4000584509DB00200AF0A4FFF2
:105FC00000EB800006EB400090FBF7F000E00120C2
:105FD00021880844A080B5F91820B4F90410A2EB78
:105FE0000A02A2EB0900814283DC11E5FFE70120F0
:105FF00093E70120AAE7806818B1007E00F0030053
:10600000704703207047000008B505496A46496893
:1060100000912C210BF064F8BDF9020008BD0000CE
:10602000089D010808B505496A46096800912C21B8
:106030000BF056F8BDF9000008BD0000089D0108EE
:10604000008C704710B5092200F0CDF8C0B210BD29
:1060500010B5092200F0C7F8C0B210BD10B5162265
:1060600000F0C1F8C0B210BD10B5162200F0BBF8A8
:10607000C0B210BD70B50C460546202200F0B3F842
:10608000024621462846BDE87040F6F71ABA10B518
:10609000212200F0A8F8C0B210BD10B5682200F0AF
:1060A000A2F8C0B210BD10B5342200F09CF8002850
:1060B00000D0012010BD10B5322200F094F800B2DB
:1060C00010BD10B5322200F08EF800B210BD10B530
:1060D000172200F088F8002800D0012010BD10B56C
:1060E000042200F080F800B210BD10B50A2200F0C2
:1060F0007AF880B210BD10B50A2200F074F880B2B0
:1061000010BD10B5602200F06EF8C0B210BD70B5C1
:106110000E460546FFF7F5FF02281AD9FF24FD2891
:1061200002D2C0EB0020040A0EB1002603E028468C
:10613000FFF7D4FA054655B131462846FFF7E1FF8F
:10614000022806D9FD28F2D24443240AEFE7022CA4
:1061500001D8002070BDFD2C01D3FF2070BD20466A
:1061600070BD10B5372200F03EF8C0B210BD10B5BA
:10617000382200F038F800B210BD10B5352200F01A
:1061800032F800B210BD10B5112200F02CF800B2A8
:1061900010BD10B5112200F026F800B210BD10B5E8
:1061A000122200F020F800B210BD10B5122200F04B
:1061B0001AF800B210BD10B5132200F014F800B2A6
:1061C00010BD10B5132200F00EF800B210BD10B5CE
:1061D000102200F008F800B210BD10B5102200F037
:1061E00002F800B210BD2DE9F8430E4607461546E9
:1061F0000121104601F050FF8046002414E06B4658
:106200002A4631463846FAF793FD0446012824D041
:10621000B8F1000F0CD0022C02D00EB1002603E022
:106220003846FFF75BFA0746002FE8D1012C14D05F
:106230001EB9012D05D0042D03D028460EF024FAF6
:106240000AE038680FE0012D0AD0C18A51B160B16F
:10625000012D0CD0B0F9160000900098BDE8F8832D
:10626000818AF3E700680028EDD10020F4E7B0F957
:106270001400F1E710B50B22FFF7B5FF00B210BD17
:1062800010B54122FFF7AFFF00B210BD10B542229A
:10629000FFF7A9FF00B210BD10B54522FFF7A3FF1D
:1062A000C0B210BD10B54322FFF79DFF00B210BD74
:1062B00010B54022FFF797FF00B210BD70B50C4635
:1062C00005465522FFF78FFF024621462846BDE8C6
:1062D0007040F6F7F6B85722FFF785BF10B56A226F
:1062E000FFF781FF00B210BD10B56922FFF77BFFF9
:1062F00000B210BD10B50122FFF775FF00B210BD4E
:1063000010B50722FFF76FFF00B210BD10B50822CD
:10631000FFF769FF00B210BD2DE9FF41074608886D
:10632000ADF800004888ADF802000888ADF8040018
:10633000C888ADF806008888ADF8080048880C4683
:10634000ADF80A00A088ADF80C00E088ADF80E00AA
:106350001D4616466946384601F023FD2B46324657
:10636000384601A901F01DFD2B463246384602A9E8
:1063700001F017FD2B463246384603A901F011FD06
:10638000BDF90000BDF90430984201DA054600E08D
:106390001D46BDF90820BDF90C108A4201DA1646E7
:1063A00000E00E46B54203DA984206DB184604E0E8
:1063B0008A4201DA104600E008462080BDF900302C
:1063C000BDF904108B4201DD1D4600E00D46BDF90C
:1063D0000820BDF90C00824201DD164600E00646A9
:1063E000B54205DD8B4201DD184604E0084602E0B7
:1063F000824200DD1046A080BDF90230BDF90600E2
:10640000834201DA1D4600E00546BDF90A10BDF9D8
:106410000E20914201DA0E4600E01646B54203DA3C
:10642000834206DA184604E0914201DA084600E0A9
:1064300010466080BDF90210BDF90630994201DDB9
:106440000D4600E01D46BDF90A00BDF90E20904240
:1064500001DD064600E01646B54205DD994201DD44
:10646000084604E0184602E0904200DC1046E08056
:1064700005221146204609F0C0FDBDE8FF81143019
:10648000FBF791B970B50546FFF728F9040012D063
:10649000E88AE18A451A2046FFF780FA0544002180
:1064A0002046FFF794FE2D1A00212046FFF703FE39
:1064B000281A00B270BDB5F9160070BDC0698143DD
:1064C00001D00020704701207047C069084000D00B
:1064D00001207047008C084000D0012070477FB534
:1064E0000D4606460221FFF7E9FF002820D0802153
:1064F0003046FFF7EFFFE8B902A93046FFF705F88D
:106500000022294602A803F052FE040012D04FF4E4
:1065100080313046FFF7D2FF70B101208DF80400C2
:1065200000956A46112130460AF0DAFD9DF8040014
:1065300004B070BD0020FBE72046F9E7F8B514462B
:106540000D4606465022FFF74EFE00B2608000283E
:1065500010D0304629465322FFF745FEC0B22073C3
:10656000022807D929463046FFF7D1FD022802D874
:1065700000202073F8BDFD2804D2217B11FB00F020
:10658000000A2073207B0228F4D952222946304683
:10659000FFF729FE024629463046F5F792FF0090A4
:1065A000BDF800002080304629465422FFF71BFE2C
:1065B000A060304629465122FFF715FE00B10120A8
:1065C000617B002D60F382016173D3D02946304690
:1065D000FFF763FD617B60F301016173F8BDF8B5FE
:1065E00014460E4605464622FFF7FDFDC0B2E07296
:1065F000022807D931462846FFF789FD00210228E5
:1066000001D8E172F8BDFD2804D2E27A12FB00F055
:10661000000AE072E07A0228F4D921804FF48070F9
:106620006080288BA98A4822401A401C00B200EBE7
:10663000D0704010A080688BE98A401A401C00B2DC
:1066400000EBD0704010E08028463146FFF7CBFDCC
:1066500010F0FF00A0720DD0472231462846FFF708
:10666000C2FD024631462846F5F72BFF0090BDF8E3
:1066700000002081002EC5D031462846FFF70DFDD1
:106680002073F8BDF8B514460D4606465622FFF7AE
:10669000AAFDC0B2A076022807D929463046FFF7E6
:1066A00036FD022802D80020A076F8BDFD2804D2CD
:1066B000A17E11FB00F0000AA076A07E0228F4D98A
:1066C00029463046FFF7FAFD0090BDF80000A08192
:1066D000304629465822FFF786FDA08230462946DB
:1066E0005922FFF780FD6082304629465A22FFF783
:1066F0007AFDA17F60F30201A1773DB129463046C2
:10670000FFF7CBFCA17F60F3C501A1772946304696
:10671000FFF7E1FD2060304629465B22FFF763FD6D
:106720002077F8BDF8B514460D460646FFF7EFFC96
:10673000074685B1022F09D80020E070A07684F8C2
:10674000220084F82A0084F83600F8BD2946304635
:10675000FFF7A3FCA070304629460B22FFF743FD4C
:106760002080E078002857D0304629462122FFF7C4
:106770003AFDC0B2E07002284ED929463046FFF7F4
:1067800079FC0090BDF80000A08030462946262202
:10679000FFF729FD48B1417A490706D0A31D0146FC
:1067A0000A22184611F075FC36E0304629462322AD
:1067B000FFF719FD0146E07B61F30200E07340073B
:1067C00021D029463046FFF755FC0090BDF8000067
:1067D000E080222229463046FFF705FD0246294681
:1067E0003046F5F76EFE0090BDF80000608130463F
:1067F00029462422FFF7F7FC20723046294625223D
:10680000FFF7F1FC2073304629462722FFF7EBFC07
:10681000E17B60F3C501E173304629463222FFF780
:10682000E2FC00B2208428B394F8220010B3304672
:1068300029463122FFF7D7FCC0B284F82200022893
:1068400018D9304629463322FFF7CDFC94F823109F
:10685000302260F3450184F8231029463046FFF7C3
:10686000C2FC024629463046F5F72BFE0090BDF8E3
:106870000000E08329463046FFF77FFCE084E8B162
:1068800094F82A00D0B129463046FFF76AFC84F814
:106890002A00022812D929463046FFF768FC2085D5
:1068A000362229463046FFF79EFC024629463046EE
:1068B000F5F707FE0090BDF80000A084A07E80B32D
:1068C000304629462822FFF78EFC206148B3304627
:1068D00029462922FFF787FCC0B2A076022820D9DA
:1068E0002069FDF713FF02286CD02A222946304682
:1068F000FFF779FC024629463046F5F7E2FD0090A5
:10690000BDF800002083304629462B22FFF76BFCA0
:10691000E076304629462C22FFF765FC00B10120C5
:10692000207794F8360070B329463046FFF7C0FC54
:10693000E08540B394F83600022824D92946304631
:10694000FFF7AAFC84F8360002281CD929463046F5
:10695000FFF796FC208629463046FFF797FC6086B5
:1069600029463046FFF79EFCA08644222946304641
:10697000FFF739FC024629463046F5F7A2FD0090A4
:10698000BDF80000A085FD2FBFF4DFAE14F8030FA3
:1069900010FB07F0000A04F8140BE07810FB07F076
:1069A000000AE070E07A10FB07F0000AE072E07C79
:1069B00010FB07F0000AE074E07F10FB07F0000A0C
:1069C000E077F8BD29463046FFF785FC606129462F
:1069D0003046FFF773FC0090BDF800002083A0E76D
:1069E0007CB50546F5F73DFD044605F11401684602
:1069F000FAF785FEBDF800006946001BADF80000FF
:106A0000BDF80200001BADF80200BDF804002044F0
:106A1000ADF80400BDF806002044ADF80600284695
:106A200000F001F87CBD7CB50C460546FEF7F8FD8C
:106A30000AF0D8FA00280FD021466846FAF75FFE20
:106A400069462846FDF79AFF002805D02846FEF73C
:106A5000E7FD6946F5F792FC7CBD0068002808D088
:106A6000017E8907F9D0007E00F00300012800D0E4
:106A7000002070470068002809D0017E11F00C0F3B
:106A8000F8D0007EC0F38100012800D000207047BC
:106A900010B504460849FFF718FD08B1002010BDE5
:106AA0002046FEF71BFE0028F9D00021FFF723FB4C
:106AB0000028F4D0012010BD010006007CB5054679
:106AC000F5F7CFFC044605F114016846FAF717FE06
:106AD000BDF800006946001BADF80000BDF80200DB
:106AE000001BADF80200BDF804002044ADF804001E
:106AF000BDF806002044ADF806002846FDF73EFF2D
:106B00007CBD10B5418C41F001014184FEF7EAFDE6
:106B1000418C41F004014184FEF782FD4068002869
:106B200003D0BDE8104001F09FBB10BD2DE9F04738
:106B3000994616460F468246FEF7E2FC804600253F
:106B400020E0DAF80800B9F1000F006850F825409D
:106B500005D04FF480212046FFF7B0FC88B9A08A09
:106B600000233844A082E08A32463044E082208B01
:106B7000394638442083608B304460832046FFF7D9
:106B8000D5FF6D1C4545DCD3BDE8F0872DE9FF47F7
:106B9000456816460F4604469DB300212846FFF778
:106BA000FEFA804600212846FFF711FB81464FF48C
:106BB00080212046FFF782FC48B1A98A07EB080034
:106BC000084407B2E98A06EB0900084410E02846A9
:106BD000FEF7DDFEAA8A02EB0801081A384407B264
:106BE0002846FEF7DBFEEA8A02EB0901081A304468
:106BF00006B200212846FFF75EFA391830440FB27A
:106C000006B2A08A381A07B2E08A301A06B20FB963
:106C1000002E43D02046FFF7E3FE02A92046FEF7F0
:106C2000F9FC4FF0000875B169462846FEF78CFC68
:106C30000022694602A803F0FAF95FEA000802D1CF
:106C4000284600F025FEA08A32463844A082E08A19
:106C500039463044E082208B002338442083608B07
:106C6000304460832046FFF761FF25B12246222190
:106C700028460AF035FA2046FFF7B2FE002D0DD067
:106C80000022694604F1140003F0D1F9B8F1000FB5
:106C900001D1002802D0284600F0FAFDBDE8FF87A8
:106CA0002DE9F0410E460746FEF763FEA0B93846CF
:106CB000FEF766FE04463846FEF71CFD00280BDA98
:106CC000002C09DD4042844200DB044622B23346F8
:106CD0000021384600F088FC3846FEF743FE0028C5
:106CE00025D13846FEF780FD04463846FEF7DCFD28
:106CF000054600213846FFF7B7F901280BD0002DD3
:106D000015DA002C13DD6842844200DB044621B210
:106D10003346002206E0002C09DA002D07DD334659
:106D2000002221463846BDE8F04100F05DBCBDE8D8
:106D3000F0812DE9F0470E4686B00546876802A926
:106D40003046FEF767FC3046F5F78BFB01460246FE
:106D500002A809F052F902AA394604A803F03FF943
:106D60004FF4002420B921463046FFF7A7FB00B1BD
:106D700001205FEA00090DF1100A10D02A46142103
:106D80003046C5F808A00AF0ABF92A46152130466E
:106D90000AF0A6F92A46162130460AF0A1F9214642
:106DA0003046FFF78BFB20B138680090786801907F
:106DB00006E006F114023946684603F010F988B17E
:106DC000C5F808D03046FEF79BFB8046002407E05C
:106DD000B068006850F82410284601F06DFF641C6C
:106DE0004445F5D3B9F1000F10D02A46172130469B
:106DF000C5F808A00AF074F92A46182130460AF0AE
:106E00006FF92A46192130460AF06AF9AF6006B0D8
:106E1000BDE8F0872DE9F14F82B00298FFF738FE08
:106E200000287CD10298FEF759FC009000210298BE
:106E3000FFF766FA834600210298FFF767FA0546D6
:106E4000009858B1FEF7CAFB81460098FEF7AAFBEE
:106E50000746CBF34130012803D013E02A465946B8
:106E60009AE02BF4C040B0F5FA6F0BDCB0F57A7FF6
:106E700001DDC0F57A7000FB09F0642190FBF1F0B0
:106E80000FFA80FBC5F3413001280ED125F4C04034
:106E9000B0F5FA6F09DCB0F57A7F01DDC0F57A70E4
:106EA0007843642190FBF1F005B200216B22029837
:106EB000FFF799F904B200216C220298FFF793F9C9
:106EC0000FFA80FA0298FFF7DAFA80460298FEF786
:106ED000CAFB0646C4F3413001280FD124F4C04058
:106EE000B0F5FA6F0ADCB0F57A7F01DDC0F57A7093
:106EF00000FB08F0642190FBF1F004B2CAF34130CA
:106F0000012811D12AF4C040B0F5FA6F0CDCB0F5BD
:106F10007A7F01DDC0F57A707043642100E05BE0A8
:106F200090FBF1F00FFA80FA0BEB040004B205EBD2
:106F30000A0005B200210298FFF78AF850B1012833
:106F400028D0801E082825D2DFE800F00C14212C60
:106F50003419393C00210098FFF780F8012819D135
:106F60000320EEE709EBD970401008EBD871A0EBD5
:106F7000610001E0A9EB0800204404B20AE007EB3D
:106F8000D770401006EBD671A0EB610000E0B81B93
:106F9000284405B22A462146029803B0BDE8F04FC6
:106FA000FFF7F4BD09EBD970401008EBD871A0EBE6
:106FB000610001E0A9EB0800204404B2E7E7A9EB77
:106FC000080006E009EBD970401008EBD871A0EB7F
:106FD0006100204404B2D2E7BDE8FE8F2DE9F04FF6
:106FE0000446408C87B0010501D540057ED420467B
:106FF000FEF774FB5FEA000878D02046FEF7F4FB4A
:107000000590608C002600054FF4FA6B42F2D17AAD
:1070100003D52046FFF733FA5DE000212046FFF755
:1070200069F90546504501D1012600E00026C5F367
:107030004130012805D125F4C040584501DC01202C
:1070400000E0002081464046FEF7C8FA074626B118
:107050002046F5F70DFF05462BE0B9F1000F28D0CB
:10706000B8F82200000518D400214046FFF742F985
:10707000504512D100212046FFF71DF8054600219A
:107080002046FFF78CF800EB050900212046FFF7AA
:1070900092F8411901EB09000AE025F4C040B0F56F
:1070A0007A7F01DDC0F57A707843642190FBF1F0BE
:1070B00005B2204600210222FFF795F80FFA80F969
:1070C000204600210322FFF78EF802B23B464946D4
:1070D0002846FAF7C7FB07462046FEF751FC049006
:1070E000608C4FF00009400505D500E06BE02046BC
:1070F000FEF7B9FA53E000212046FEF7F0FFA0F5B5
:107100001C510546D13906D000208146C5F34130D7
:10711000012802D007E00120F7E725F4C0405845D8
:1071200001DC012000E0002083464046FEF73AFAE9
:107130008246B9F1000F04D02046F5F725FE05463A
:107140001BE0BBF1000F18D0B8F82200400507D4AF
:1071500000214046FEF7C3FFA0F51C51D13936D0BF
:1071600025F4C040B0F57A7F01DDC0F57A7000FBF0
:107170000AF0642190FBF1F005B2204600210522BF
:10718000FFF731F80FFA80FB204600210622FFF7B7
:107190002AF802B2534659462846FAF72EFB05460E
:1071A00056EA090605D0DDE904210023204600F057
:1071B00018FB2046FFF763F9B8421BD12046FEF7C3
:1071C00052FAA84216D1002007B0BDE8F08F002186
:1071D0002046FEF770FF054600212046FEF7F7FF28
:1071E00000EB050B00212046FEF7CDFF411901EB16
:1071F0000B00C1E72046FFF7F3FB69462046FEF788
:1072000009FA02A94046FEF79FF9002202A9684642
:1072100002F00DFF060002D1404600F039FBE08A83
:107220006D1E2844608300212046FEF717FF0128C9
:107230001CD0A08A7F1E384420836A46292120461C
:1072400009F04EFF22462221404609F049FF204620
:10725000FFF7C6FB608C002240F00200608402A9A8
:1072600004F1140002F0E3FE36B904E0208BC01BE9
:10727000401CA082E1E710B1404600F009FB204627
:1072800000F002F801209FE738B50546F5F7E9F868
:1072900004460020ADF800006A461321284609F094
:1072A0001FFFBDF90000A04202D02846FFF798FB5F
:1072B000BDF80000A96831B930B12846FDF740FBA0
:1072C000BDF80000A968C882BDF90000A04202D044
:1072D0002846FFF785FB38BD70B505460021FFF74E
:1072E00009F8044600212846FEF7F9FE42F2D17162
:1072F0008C4203D0884201D0002070BD2846FFF7A1
:1073000000FC012070BD00002DE9F84F06465148F1
:1073100090460C460078002870D03046FFF760FB9E
:1073200004F47F040421404600F0B6FE0746022123
:10733000404600F0B1FE81460121404600F0ACFE1F
:1073400000901021404600F0A7FE05464FF6FF7B57
:10735000EFB1B4F5702F12D08CB130460021042269
:10736000FEF741FF00B242F2D17A504507D03046D5
:1073700000210122FEF737FF00B250454DD1002217
:107380002A21304609F0ACFE3046FFF7BAFB4FF435
:10739000702A544500D084BBD84500D02FB1304668
:1073A000FEF79CF908B1FFF7ACFB544500D024BBB5
:1073B0001DB3304600216E22FEF715FF00B240B922
:1073C000304600216D22FEF70EFF00B2B0F5807F3F
:1073D00001D0022514E0304600216122FEF703FFB0
:1073E000C0B2FF2807D1304600216822FEF7FBFE1D
:1073F00010F0FF0F03D0012502E00EE028E0002589
:10740000B06820B1817E65F38711817605E025B1F2
:107410003046FDF795FAB068F4E75D46A84502D01E
:10742000B9F1000F02D03046FFF72EFF3046FFF7CC
:10743000D7FAA84504D0009949EA0700084207D0C6
:10744000B4F5803F04D03046BDE8F84F01F01ABED5
:10745000BDE8F88F6C5200202DE9F04104460E463D
:10746000408C154600210423C0F305120AE0E068B1
:1074700003EBC107C059C70103D520F07F40A842E4
:1074800002D0491C8A42F2D88A4202D10020BDE8CB
:10749000F081E06850F8310031460DF08FF928B1E5
:1074A000324629462046FFF72FFF01E00028EED0A4
:1074B0000120ECE72DE9F05F0E0004461FFA82F888
:1074C00002F47F074FF6FF7B03D0F07908B94FF045
:1074D000000B00252B4658E0E068042101EBC50AAB
:1074E000814650F80A004FF6FF7281B200F47F0C1B
:1074F000904501D0414509D1B7F5702F01D0BC4569
:1075000004D12EB159F83510B14201D06D1C3CE0C8
:10751000800104D500233946204602F0CBFAE0680A
:1075200050F80A10CA0101D489010CD550F8350071
:107530000DF0A4F9E06850F835000CF097F8E16818
:10754000002041F83500284608230AE0E16803EBF3
:10755000C00C01EBC0026144401CD1E900C1C2E98A
:1075600000C1618CC1F30511491E8142EED8608CC7
:107570000109491E61F309106084C0F30510C100C0
:10758000E0680CF097F80123E060608CC0F3051010
:10759000A842A1D8002B09D0BBF1000006D00246BA
:1075A00039462046BDE8F05FFFF7AEBEBDE8F09F6C
:1075B00070B506460B480078002812D000200CE079
:1075C000002406E0E86850F82410304601F079FD08
:1075D000641C686AA042F5D8284609F0CDFC050075
:1075E000EED170BD6C520020F0B51546064691B044
:1075F0000C4651EA050078D0012B1DD03C4930469D
:10760000F9F77EFF3B493046F9F77AFF002209215E
:10761000304609F065FD012867D12A4621463046EB
:10762000F4F72BFF012860D111B03046BDE8F040DF
:1076300000220A2109F054BD3046FDF7F1FF07464C
:107640006846F9F7A5FF2C48009603902CB33846FE
:1076500009F06CFC401022460021F9F7FBFF64287A
:1076600001D2642002E0962800D996200B90304683
:10767000FEF78DF94142201A0891CDE909101D4805
:1076800001901E4807906A460921304609F028FDFE
:1076900001282AD16846F9F7EBFF002D25D038469E
:1076A00009F08AFC40102A460021F9F7D3FF64282C
:1076B00001D2642002E0962800D996200B90304633
:1076C000FEF76CF94142281A0891CDE909100848E3
:1076D00001900A4807906A460921304609F000FDEA
:1076E000012802D16846F9F7C3FF11B0F0BD0000D0
:1076F0005994010841940108A9910108F91501085C
:107700002DE9F0471546824699460C4651EA050098
:1077100065D0504600F074FB5046FEF738F9404201
:107720000FFA80F808EB040004B200215046FEF77F
:107730009BFC012813D0002C13DC25DA5046FEF701
:1077400053F806465046FEF7AFF8304400B2002822
:1077500000DA00204042844216DA04B214E0002C21
:1077600002DA4FF000040FE00EDD5046FEF73CF861
:1077700006465046FEF798F8304400B2002800DA7A
:107780000020844200DD04465046FEF707F94042DF
:1077900006B2701905B2002D02DD4FF0000510E0B1
:1077A0000FDA5046FEF7ECF807465046FDF7A2FF09
:1077B000384400B2002800DA00204042854200DA56
:1077C00005B2A4EB080001B2A81B02B251EA020004
:1077D00005D04B465046BDE8F047FFF705BFBDE872
:1077E000F08770B516461D4604461A4600F024F888
:1077F0002A4631462046BDE8704000F033B8F8B55F
:107800000F46054600F0FCFA002000902846FDF7E0
:1078100065FF044605F114060AE03B466A46294620
:10782000304601F0C7FC25462846FDF757FF0446C1
:10783000002CF2D1F8BD000070B50E461446054686
:107840000749F9F75DFE2846FEF7A1F8801B01B253
:1078500023462846BDE870400022FFF751BF0000D4
:107860004194010870B50E46144605460749F9F7DC
:1078700047FE2846FEF792F8801B02B223462846B0
:10788000BDE870400021FFF73BBF0000599401089C
:107890001FB5044602AA6946FEF787F8684608F055
:1078A00080FB20B902A808F07CFB002810D06846B5
:1078B00008F077FB18B169462046FFF7B4F802A834
:1078C00008F06FFB002803D002A92046FFF7ABF8B1
:1078D0001FBD002200F04CB970B50C460546FDF7FF
:1078E0002FF8A868848270BD38B50C460546002381
:1078F0006A460421FDF7D3FE012807D0002804D1F1
:1079000000222146284600F07AF938BD0098A042AE
:10791000F6D138BD2DE9F0410C4615461F46064606
:107920001946F9F76AF92A4621460DF055F822461C
:1079300039463046BDE8F041FFF7E6BC70B5154664
:10794000044600F0FDF929462046BDE8704000F0ED
:107950000DBA70B50C460546FCF7F2FFA868417EEB
:1079600001F00F01A14200D0447670BD70B50C4605
:107970000546FCF7E5FFA868017E64F38301017604
:1079800070BD70B50C460546FCF7DAFFA868017EAD
:1079900064F30511017670BD70B50C460546FCF721
:1079A000CFFFAB681A7E02F00300A04207D064F359
:1079B00001021A762846BDE87040FFF711B870BD85
:1079C00070B51546044600F0A5F929462046BDE8E5
:1079D0007040FFF789BF2DE9F34F89B08346008CD3
:1079E0000A9988427DD00390ABF8201058460A9A35
:1079F0000399F4F727FE0290002872D04FF4207408
:107A000020460BF0D5FD8046214610F06AFB00248D
:107A100020466BE0DBF80C00042202EBC90500EB0A
:107A2000C90A405920F07F4000F0B9F90190DBF815
:107A30000C00405920F07F4000F0AEF907900A9901
:107A40000198884350D1DAF8040080014CD405AA8B
:107A50006721DAF8000000F0CFFA012844D10027AE
:107A6000059D39E000261BE006EB860108EB81014D
:107A700006914868049000F092F90090049800F094
:107A80008BF9296831F81720069909898A4206D1AD
:107A90000799884203D1DDE90001884202D2761CB1
:107AA000A642E1D3A64216D104EB8400A98928F8A6
:107AB000201008EB8000298A4180A968C1602968EC
:107AC000641C31F81710018169680161DAF804104B
:107AD00021F07F4141607F1C286830F8170018B101
:107AE00000E042E0202CBDD309F101008146BBF843
:107AF0002200C0F30511494501D9202C8AD3002565
:107B00000EE005EB850108EB8106706800F044F992
:107B10000146009658460A9B039AF4F7F3FC6D1C45
:107B2000A542EED340460BF08FFD029801280CD001
:107B3000032810D0022818D15846FEF751FF0BB089
:107B40005846BDE8F04FFFF79FBB0BB05846BDE865
:107B5000F04FFEF745BF0BB05846BDE8F04F4FF66B
:107B6000FF724FF47021FFF7CFBB0BB0BDE8F08F71
:107B700013460A460921FFF7CDBE13460A46662181
:107B8000FFF7C8BE07B481B01346BDF80810ADF8C2
:107B90000010009A522104B0FFF7BCBE13460A46FB
:107BA0005321FFF7B7BE13460A465021FFF7B2BE76
:107BB00007B481B01346BDF80810ADF80010009A64
:107BC000202104B0FFF7A6BE13460A462121FFF785
:107BD000A1BE07B481B01346BDF80810ADF800107F
:107BE000009A302104B0FFF795BE13460A463121B2
:107BF000FFF790BE13460A463221FFF78BBE1346AD
:107C00000A460421FFF786BE13460A460A21FFF7FB
:107C100081BE13460A466021FFF77CBE07B481B0DF
:107C20001346BDF80810ADF80010009A362104B0D4
:107C3000FFF770BE13460A463721FFF76BBE1346A7
:107C40000A463821FFF766BE13460A463521FFF77C
:107C500061BE13460A461121FFF75CBE13460A4671
:107C60001521FFF757BE13460A461221FFF752BEF1
:107C700013460A461321FFF74DBE13460A46142148
:107C8000FFF748BE13460A461021FFF743BE1346CE
:107C90000A460B21FFF73EBE13460A464321FFF773
:107CA00039BE13460A464021FFF734BE13460A4642
:107CB0005B21FFF72FBE07B481B01346BDF8081053
:107CC000ADF80010009A552104B0FFF723BE13460B
:107CD0000A465721FFF71EBE13460A465821FFF7F2
:107CE00019BE13460A465921FFF714BE13460A4629
:107CF0005621FFF70FBE13460A460121FFF70ABEC1
:107D000013460A460721FFF705BE13460A46082117
:107D1000FFF700BE38B50C46054600236A46012130
:107D2000FDF7BDFC012807D0002804D10022214620
:107D30002846FFF7E0FF38BD0098A042F6D138BDD5
:107D400038B50C46054600236A460721FDF7A7FC17
:107D5000012807D0002804D1002221462846FFF739
:107D6000CFFF38BD0098A042F6D138BD38B50C46DB
:107D7000054600236A460821FDF791FC012807D03B
:107D8000002804D1002221462846FFF7BEFF38BD57
:107D90000098A042F6D138BD00F47F00704780B251
:107DA00070472DE9F0411E4615468846070025D04C
:107DB000F4F75DFB022813D000249EB13DB1384694
:107DC000FDF78CFC33462A464146FFF7EAFF002CBC
:107DD00014D0324641463846BDE8F04101F0BEBEFF
:107DE0000124EAE724B132464146384601F0B6FEA6
:107DF000002D03D03846FDF771FCD7E7BDE8F081D0
:107E000070B50B4D2978002910D101212970FDF79B
:107E100069FC044605E021F0040060842046F9F77F
:107E20009DF9618C4807F6D40020287070BD0000D1
:107E30006452002010B520F007F80F4A4FF4965313
:107E4000A2F51651A1F11C0008F067FF0B4808F0DD
:107E500073FF0A48F02101804FF4A0714180084966
:107E600041610849C160016941F004010161BDE857
:107E7000104008F08BBF00008CAD00200CD3002018
:107E800021D80008F087002010B50A480AF0B4FC99
:107E9000084802210170084941600AF0C1FC074C02
:107EA000606009F059FC0146A0606068BDE81040C0
:107EB0000AF02EBE5CD30020B50F01083852002016
:107EC0002DE9FC410E46002507462A46143102F0F2
:107ED000AEF8002826D001213046FEF7EFFA00BBAD
:107EE0003046F4F7C4FAE0B900208DF800006A4685
:107EF00012213046019709F0F3F89DF8000002289E
:107F00000FD03046FDF7FCFA401E04000ED4B068D6
:107F1000006850F824103846FFF7D2FF050009D159
:107F200002E00020BDE8FC81641EF0D59DF8000051
:107F300000B935462846F5E72DE9FC410025DFF874
:107F4000B4804FE0284490F83001E8BB002441E0C1
:107F5000011991F83011C1BBA5423AD000EBC40120
:107F600000EBC5003030303102F0B5F868B370680E
:107F7000B04600EBC40200EBC50168463031303238
:107F800002F0A9F9684608F00CF80646D8F8040093
:107F900000EBC500303008F004F80746D8F80400BC
:107FA00000EBC400303007F0FCFF3844864210D2AA
:107FB000D8F80400464600EBC50069463030F9F7B2
:107FC000A7FB0120716801E00BE002E0214481F889
:107FD0003001641CD8F804004646B0F85011A142A4
:107FE000B6D86D1CD8F80400B0F85021AA42A9D820
:107FF000BDE8FC817052002070B515468288C479B6
:10800000A2F57F43FF3B07D08CB3012C34D906681F
:10801000002306EB84022CE0002313E0026802EB4D
:10802000C302168826F440468E420AD11088010405
:1080300028D4400401D5304613E050682860012060
:1080400070BD5B1C9C42E9D824E032F8130020F498
:10805000404088420CD132F813100A0412D449046B
:1080600002D50CF011FBE9E706EB830010E011E00C
:108070005B1C9C42E9D80DE022F440438B4209D1BD
:10808000110401D5022070BD510401D51846E8E75E
:108090000068D3E7002070BD10B50C4602F038FD33
:1080A000204000D0012010BD2DE9F04107461546C3
:1080B0000E460B4802F07BFC040010D0A7604FF086
:1080C000FF3026602061002060610DF091F8E560CE
:1080D00004496060012008712046BDE8F081FEE798
:1080E000D0D400204053002010B504460146054876
:1080F00002F0D3FC044B01222046DA70BDE81040A8
:108100000BF0B4BAD0D40020405300202DE9F04742
:10811000494CA07810B10120BDE8F0870120A07083
:108120002078002528B10DF063F85FEA000A02D03C
:1081300007E0A570EFE72069401C2061642800D9A2
:1081400025613E4FA946A0463D4888F8039088F82F
:10815000049002F007FC386033E0394802F014FC68
:108160003C680646207DC0072AD10025204600F045
:108170007EF868B92569002D01DD681E20610DF0CB
:1081800037F86060A16811B10DB12046884701251C
:1081900098F8030020B9206910B92046FFF7A4FF22
:1081A00075B198F8041098F80300014308D03868B6
:1081B0000028C9D14FF0FF35214802F0D3FB11E070
:1081C0003E6039680029C8D1F4E7207DC00705D199
:1081D000204600F04CF8A84200D205462146184837
:1081E00002F0D2FB0400F0D150460CF0FAFFD8F8B0
:1081F0000C1044460844C8F80C00D8F808000CF0ED
:10820000F0FFB0F5FA7F13D3E16864225143B1FB6C
:10821000F0F0C0B26070642801D9002001E0C0F124
:10822000640060702646C4F80C900CF0E1FFB0606A
:1082300084F8029028466FE7405300201453002032
:10824000D0D4002001214161704710B504460CF0E4
:10825000CFFF2168401A401E606010BD10B5044673
:108260000CF0C6FF606010BD00214161704710B581
:10827000044640680CF0B5FF2168814201D8002017
:1082800010BD081A10BD00002DE9FF4F85B005464E
:10829000DDE913981E460F460846169CF9F795FA35
:1082A00003903846F9F76DFA0290012C13D0022C96
:1082B00013D0032C4CD14E4F2888ADF800003088E5
:1082C000B8F1000FADF8040009D098F80000FD28BF
:1082D00041D3484642E0474FEEE7474FECE7DDE940
:1082E00000104A46B847049000202DE0002420E00A
:1082F000BDF8040036F81410884205D1BDF800001E
:1083000035F8141088420ED005EB44004A46008828
:10831000ADF8000006EB44000088ADF80400DDE98C
:108320000010B847049005EB4400BDF81010018020
:10833000641C03988442DBDB079805EB4005129828
:1083400006EB400608F10100029980468842CDDB29
:1083500009B0BDE8F08F00FB09F0000A8246024632
:10836000DDE90010B847049000203CE000242DE037
:1083700018F8040048B3FD2801D3484602E000FB8A
:1083800009F0000ABDF8041036F81420914207D114
:10839000BDF8001035F81420914201D182450FD06C
:1083A00005EB440182460988ADF8001006EB440154
:1083B00002460988ADF80410DDE90010B8470490C2
:1083C00005EB4400BDF810100180641C0398844242
:1083D000CEDB0798159905EB40051298884406EB0B
:1083E00040060BF10100029983468842BEDBAFE7ED
:1083F0007BD30008F9D20008FFD300082DE9FF4F16
:1084000085B00646DDE913791D460C460846F9F7A6
:10841000DCF980462046F9F7B4F98346B9F1000F3C
:1084200006D0FD2F7ED9A8F10400049000201DE1A4
:10843000FD2F14D300244FEA48070BE030462946AD
:108440003A460FF026FE0798641C06EB4006129889
:1084500005EB40055C45F1DB09B0BDE8F08F00207D
:1084600021E0002415E006EB440A3A46BAF8000081
:10847000ADF8000005EB44000088ADF80400DDE92C
:108480000010F9F783FA0090BDF80010AAF8001068
:10849000641C4445E7DB079806EB4006129805EBA1
:1084A000400509F1010081465845DADBD4E74F4623
:1084B000002419E03A78AAB1FF2A06EB440018D04C
:1084C00082460088ADF8000005EB44000088ADF856
:1084D0000400DDE90010F9F759FA0090BDF800102A
:1084E000AAF80010641C7F1C444575DAB807E1D176
:1084F00072E005EB440109880180F3E73868E8B3CE
:10850000401C6DD03A78BAB1FF2A06EB440075D012
:1085100082460088ADF8000005EB44000088ADF805
:10852000040000E0ACE0DDE90010F9F72FFA00905C
:10853000BDF80010AAF800107A7807F1010AAAB174
:10854000FF2A06EB44005ED000904088ADF804009E
:1085500005EB44004088ADF80800DDE90110F9F7AB
:1085600015FA0190BDF80410009841801AF8012F07
:10857000BAB1FF2A06EB440049D000E02AE000909F
:108580008088ADF8040005EB44008088ADF8080051
:10859000DDE90110F9F7FAF90190BDF8041000982F
:1085A00081809AF80120AAB1FF2A06EB440032D05C
:1085B0008246C088ADF8000005EB4400C088ADF8E5
:1085C0000400DDE90010F9F7E1F90090BDF80010B2
:1085D000AAF80610241D3F1D049884428EDB39E062
:1085E00005EB440006EB440102880A8042884A8079
:1085F00082888A80C088C880ECE7FFE705EB4401E9
:108600000988018098E705EB44014988ADE705EB4F
:1086100044018988C4E705EB4401C988C180D9E7D2
:108620003A78AAB1FF2A06EB440024D0824600889B
:10863000ADF8000005EB44000088ADF80400DDE96A
:108640000010F9F7A3F90090BDF80010AAF8001087
:10865000641C7F1C4445E3DB0798159906EB400634
:108660001298894405EB40050398401C0390584537
:10867000FFF61DAFF0E605EB440109880180E7E74E
:1086800000202BE000241DE019F80400C8B1FD28EB
:1086900001D33A4601E07843020A06EB4400009019
:1086A0000088ADF8040005EB44000088ADF8080030
:1086B000DDE90110F9F76AF901900098BDF804109E
:1086C0000180641C4445DFDB0798159906EB4006E2
:1086D0001298894405EB40050AF10100824658458D
:1086E000D0DBB9E62DE9FF4F85B01D46DDE913B8B3
:1086F0000E46F4F79DF882463046F9F766F8814653
:108700003046F9F73EF80390B8F1000F4FF000073C
:108710001ED048E0002415E005EB4400CDF808B079
:108720000088ADF804007088079A384400B20090C1
:1087300030880599204403B2DAF80000D0F81CC054
:10874000E047641C4C45E7DB12987F1C05EB4005B5
:1087500003988742DEDB09B0BDE8F08F00241AE001
:1087600018F80400B0B100FB0BF0000A029005EB12
:108770004400079A0088ADF804007088384400B2BD
:10878000009030880599204403B2DAF80000D0F850
:108790001CC0E047641C4C45E2DB159912988844E4
:1087A00005EB40057F1C03988742D7DBD3E7FD2903
:1087B00002D2022901D80020704710FB01F000EB23
:1087C000C01101EBC030C0F3C750704770B5094D00
:1087D00004466868002808D044B12046F8F704FA37
:1087E000A9682044884200D3002070BD0248006878
:1087F00070BD000078520020205300202DE9F04188
:1088000004460022212108F06BFC00287ED0608CF9
:1088100040F48050608401E0FFF7F0FF0021204623
:10882000FCF75CFE0028F7D12046FCF717FF064650
:1088300000200AF01FF8054600271CE0A86AA042A5
:1088400002D0E86AA04203D1214628460AF0BAF8CD
:10885000686BA04200D16F63686DB04207D10AF027
:1088600013F8A04203D1214628460AF0ABF8284667
:108870000AF000F80546002DE0D12046F3F7E3FDAD
:10888000606804260028204602D0FCF7EFFE29E0AD
:10889000FCF7C6FE0546416A0022C06804E050F8B5
:1088A0002230A3420AD0521C9142F8D806E0E86870
:1088B00006EB8201415840F82210521C686A401EA3
:1088C0009042F4D8686A401E81006862E8680AF045
:1088D000F1FEE8601EE0096806EB80028A5841F864
:1088E0002020401C616889684A68521E8242F2D882
:1088F000606880684068401E4860616880008968E0
:108900000A68014610460AF0D5FE00E007E06168FB
:10891000896808602046BDE8F0410AF0A7BEBDE8BE
:10892000F08100002DE9F04F524F064685B078687F
:108930000168CC6BC96889682160016809698A0788
:1089400001D4C90723D008F037FB401E05B2786870
:1089500008F0ECFA401E03B20022114603A800956D
:1089600007F065FB03A9616078680068027CC06855
:10897000920705D5826942F002028261A16073E02C
:108980008169826961F341028261A6606CE03046D0
:10899000F8F70FFF81463046F8F7EDFE804678681D
:1089A00008F00AFB0146B6F90600814203DC78684C
:1089B00008F002FB401E05B242464946BA467868B6
:1089C000F8F782F981460027B6F902000DF1040B91
:1089D00028E03288ADF80420B288ADF80820ADF860
:1089E0000600ADF80A10C4F804B0C4F808B0DAF80C
:1089F00004000168C96889682160BDF90A10A942AC
:108A000001DDADF80A50BDF90A70BD4205D100681C
:108A1000C068816941F002018161204600F02CF8B4
:108A20000FFA88F000EB0908A8F10101A942D0DD96
:108A3000BD421CD03188ADF80410B188ADF80810E3
:108A4000ADF80600ADF80A50C4F804B0C4F808B098
:108A5000DAF804000168C968896821600068C068A4
:108A6000816941F002018161204600F005F805B0FE
:108A7000BDE8F08F705200202DE9F0415F4F0646AF
:108A800090B0786808F04EFAF168044609B13046B3
:108A90008847786800680188408811FB00F0E16829
:108AA000884201D1012000E00020216859B16168AD
:108AB00031B128B907E078680068816A01B1884758
:108AC00020690028F7D10024786808F05FFA014691
:108AD0007068FFF7F5F905467868416919B1706863
:108AE000FFF7EEF9044655EA040051D1786808F022
:108AF00063FA401E0FFA80F8786808F017FA401EF3
:108B000003B2002211460EA8CDF8008007F08FFABC
:108B1000306BB0B16846FAF77DFA78680EAAC16A80
:108B2000049190F829108DF81A10418DADF80410B9
:108B300090F829008DF80300336B6946304698475A
:108B400026E07868C06A98B106A909F0E1FB01281F
:108B50001ED16846F9F7D4F978680EAA90F8291062
:108B60008DF80B10C36A69463046F9F795F90FE0A6
:108B70006846FAF74FFA7868418DADF8041090F81E
:108B800029008DF80300694630467268FAF72EFA1C
:108B9000786890F82810C9070CD005B905693046E7
:108BA000294600F09FF97868406990B104B90446FD
:108BB00021460BE0406928B104B9044621463046FD
:108BC00000F090F90DB9786805692946304600F043
:108BD00089F9786808F0C8F90146304600F082F952
:108BE000786808F0B9F90146304600F07BF97868FA
:108BF00010B0BDE8F041F5F745BC00007052002010
:108C00002DE9F0412B4F002038607868B0F85051C2
:108C1000002D4DD0002603E0411991F83011D1B15B
:108C20006D1EF9D50068416B01B18847786801680D
:108C3000C9688A6922F001028A610168C9688A6983
:108C400022F002028A6190F82810002441F0040109
:108C500080F8281022E02E46E4E7011991F830113F
:108C6000D9B9B44205D10168C9688A6942F00102E4
:108C70008A610168C9688A6922F002028A6100EB90
:108C8000C4003030FFF74EFE786800EBC40030308F
:108C900007F087F9396808443860641C7868B0F8D0
:108CA0005011A142D9DC10F8281F21F004010170F5
:108CB000BDE8F081705200202DE9F04F0D4680464E
:108CC0008BB001212846FDF7F9FB00287ED128460C
:108CD000F3F7CDFB040028D0284600216122FDF7E0
:108CE00082FA00F0FF0BBBF1020F6FD306AB2246F6
:108CF00029464046F8F7E9F9012867D105F1140142
:108D00000127002206A80A9101F091F9A8B10020DC
:108D10008DF8200006A8099008AA1221284608F01C
:108D2000DFF99DF8200038B107E00BB02946404636
:108D3000BDE8F04FFDF7FDBF0027012C01D147F042
:108D400002073A4606A94046F9F7B8FB04003DD0B1
:108D5000284600216F22FDF746FA00B260F30F06A5
:108D60008146284600217022FDF73DFA00B260F3EB
:108D70001F468246C9F34130012818D129F4C04961
:108D8000B9F5FA6F13DC0A98F8F713FD014630B213
:108D900020F4C040B0F57A7F02DDC9F57A7000E0BA
:108DA00048464143642091FBF0F060F30F06CAF39C
:108DB000413001281AD12AF4C049B9F5FA6F15DCFF
:108DC0000A98F8F7D8FC0146301400E084E020F45B
:108DD000C040B0F57A7F02DDC9F57A7000E0484600
:108DE0004143642091FBF0F060F31F466846F9F7B9
:108DF00087F88DF80BB0284600216E22FDF7F3F9B5
:108E000000B2ADF80000B0F5616F02DDA0F5616061
:108E100003E0002803DA00F56160ADF800002846A1
:108E200000216D22FDF7DFF9ADF802002846002190
:108E30006822FDF7D8F98DF80C00294840680068D1
:108E4000007CC0F3C0008DF81400B8073AD5D4E90F
:108E50000001C4E902016089618A0844401E00B231
:108E6000E081B4F9061088422CDDE1812AE0B807E0
:108E700005D53B46224641462846F8F7F3F82946F1
:108E80004046FDF756FFA88A6A468119D8F80400C3
:108E90000088081AADF80400E88A00EB2641D8F8EB
:108EA00004004088081AADF8060021464046F9F74C
:108EB00000FBB8070CD5E089401C6081618A08443A
:108EC000401EE081B4F90A00BDF91E108842CEDDD3
:108ED00021464046F9F723FB0BB0BDE8F08F0000B8
:108EE000705200202DE9F0470F00814605D11B4844
:108EF000406808F04BF807002AD039464846FFF78B
:108F0000DBFE20E00026FCF7FBFA8046002408E0A8
:108F1000A868006850F82410E6B14846FFF7CCFE78
:108F2000641C4445F4D34A461721284608F0D8F873
:108F30004A461821284608F0D3F84A4619212846FF
:108F400008F0CEF82F463846FCF7C8FB0500D9D10B
:108F5000BDE8F087B942E3D10126E1E77052002075
:108F60002DE9F04F464C8DB0606801680A7CD2074D
:108F70007ED0C968496800297FD000F5AC7001F047
:108F800083FD002879D160680168C9688B680C93FB
:108F90000A68934200D14A68924607F0C7FF0B90D7
:108FA000202103A80FF09DF80025A0463CE04119C0
:108FB00091F83011B9BB00F5AC7001F0D3FC074655
:108FC000A0462EE0D8F804003946444600F5AC70BF
:108FD00001F0DAFC83466068394600EBC50203A85D
:108FE000303200F063FF0646401C19D000240DF11A
:108FF0000C0909E001F0F9FC09EBC401641C0A68E2
:1090000002604968416064B2D8F80400B44239464D
:1090100000F5AC70EEDB01F040FD38460AF026FBAF
:109020005F46002FCED16D1CD8F804004446B0F83E
:109030005011A942BBD8264600F5AC7001F092FC55
:1090400012E00B98CDF800A0CDE901047068DDE9CD
:109050000B2100682346C06B856BA84770682146CA
:1090600000F5AC7001F090FC0400EAD1706800E0FB
:1090700003E000F5AC7001F05FFC0DB0BDE8F08FCF
:10908000705200202DE9F0410746FCF739FA0646F8
:10909000002412E0B868006850F824502846FDF714
:1090A0009FFC00222A21284608F01AF82846FDF7DE
:1090B00097FC2846FFF7E6FF641CB442EAD3BDE8FC
:1090C000F0812DE9F0410646488C0D460022C0F3A0
:1090D00005100EE026B1E96851F83210B14207D10F
:1090E0004FF6FF724FF470212846FEF70DF902E0AB
:1090F000521C9042EED82846FCF702FA074600249C
:1091000007E0A868006850F824103046FFF7D9FF40
:10911000641CBC42F5D3BDE8F0812DE9FF5F8346B6
:10912000DDE90E87DDE91354129EF3F781FB006839
:109130003146FF22D0F8389020460EF0CBFF0020B9
:1091400082462DE01099414308EB212211994143B9
:1091500007EB212112124FEA212107D4019B9A42E9
:1091600004DA002902DB029B994202DB04F800A02A
:1091700009E0DDF80CC001FB0C210BEB410105EB14
:109180004002098811801599062907D135F8102069
:109190001FFA89F18A4201D104F800A0401C00B2F4
:1091A000B042CFDBBDE8FF9F002200680A2107F034
:1091B00097BF00002DE9FF4F85B090460C4608464A
:1091C000FCF78CFA06461021FDF778F900286FD0DD
:1091D0003046FCF7E1FA834600253046FCF7C9FB30
:1091E0001434CDE9024000B9059C00213046FCF75B
:1091F00068FF824600213046FCF7EFFF504407B27B
:1092000000213046FCF7C5FF504401B20191F08ABD
:1092100061883844411AB8F80200728B091A0FFAB3
:1092200081F90199511AE288891A401A00B2009016
:109230003046FCF718FA0199C01B401A00B204909E
:10924000B9F100010DDB0098002815DA0846B9F1E4
:10925000000F06DD05463046FCF792FB401B0AD4A2
:109260000AE00098002807DD404205B23046FCF7CE
:1092700041FAE84200D500250398012804D00228CD
:1092800006D003280CD114E0F08A6188384403E04A
:10929000718B0198081AE1882944401A284405B2C4
:1092A00000243046FCF75EFB0090A8B1029F14E05A
:1092B000BEE00498F18A00EBD07007EB60000A185A
:1092C000E0886188401A401C00B200EBD07005EBCA
:1092D00060000844101AE1E7059F00213046FCF7C2
:1092E00064FF50440FFA80F900213046FCF769FF13
:1092F0005044B18A0FFA80FA01EB09003988338BA8
:10930000421AB8F80010501AA3EB0A02BB8800B248
:10931000D21A891A09B200280ADB002912DA0028B9
:1093200006DD04463046FCF75FFA001B09D409E06D
:10933000002907DD484204B23046FCF7B5FAE042A6
:1093400000D500243046FDF79AF8A0EB0901A1EB07
:109350000A0001B20098012804D0022807D003288F
:109360000DD122E0B18A01EB0900398803E0318B8D
:10937000A1EB0A00B9882144401A204404B22E49C6
:109380003046F8F7BDF807462C493046F8F7B8F8EC
:10939000074306D000220A21304607F0A1FE01282B
:1093A00046D15FEACB7012D014E001EBD171B28AE2
:1093B00009EB61000244B8883988401A401C00B2A9
:1093C00000EBD07004EB60000844101AD5E7002CC5
:1093D00000DA00245FEA8B7002D4002C00DD002448
:1093E0005FEA4B7002D4002D00DA00255FEA0B70B3
:1093F00002D4002D00DD00250898B8F900100028DF
:1094000000D020460844A8F80000B8F9021002D1A4
:109410004FF0000000E028460844A8F80200089B2E
:1094200009B02A4621463046BDE8F04FFEF7DCB8C9
:1094300009B0BDE8F08F000059940108419401087B
:1094400010B50346FCF7A3FA084401B2BDE810408A
:1094500000221846F3F711B810B50346FCF79EFA40
:10946000084402B2BDE8104000211846F3F705B8E1
:10947000F8B505460C460846F9F7CCFD4FF48036A2
:1094800031462846FCF703FEE070022808D928463A
:1094900031462022FCF7A7FE0090BDF80000A08016
:1094A000284631463122FCF79EFEC0B2002784F8E0
:1094B0002200022814D9284631463222FCF793FEB6
:1094C00000B22084002809DD284631463022FCF70E
:1094D0008AFE0090BDF80000E08301E084F822706D
:1094E000284631464522FCF77EFEC0B284F836009D
:1094F00002281AD9284631464022FCF774FE00B2F1
:10950000E08500280FDD284643223146FCF76BFE3C
:10951000A086284644223146FCF765FE0090BDF83F
:109520000000A08501E084F8367031462846FCF73B
:10953000EEFDFD280AD2E17811FB00F1090AE17085
:109540004143080A84F8220084F83600E07830B9F4
:1095500094F8220018B994F83600002805D0314656
:109560002846FCF787FE20800120F8BD2DE9F84F42
:10957000044615460E464FEA61084FEA610AC807DD
:1095800001D1A8F10108600000900AF011F8074627
:109590002B46002025E003EB440B3BF8021C7143F3
:1095A000601E16D4002200EB0A0C27F81010A44508
:1095B00001DA33F81C208A1AA0EB0801012901D531
:1095C000198803E003EB410131F8021C401E1144ED
:1095D000E8D539461846009AFBF7FEF85B4609F1D4
:1095E00001008146A042D6DB4FF47F52B2FBF6F178
:1095F00000201FFA81FC14FB04F30CE035F8101076
:1096000041B1914202D125F810C003E091FBF6F17F
:1096100025F81010401C8342F0D8002139E005EBFA
:10962000410399461A887243002024E0002A02DA96
:109630004FF0000C01E04FEAA21C27F810C0A0EB8D
:109640000A0CBCF1000F02DCB3F800C003E00CFB15
:10965000041C35F81CC0A2EB0C0C00EB0802521CD9
:10966000A24200DB621E02FB041203EB440335F846
:109670001220401C6244A042D8DB4A46002005E08C
:1096800037F81030138002EB4402401CA042F7DB95
:10969000491CA142C3DB3846BDE8F84F09F0D4BFEE
:1096A0002DE9F0470E468AB01D4680460146174612
:1096B0009246541907A8F8F74FF807EBD77005EB57
:1096C000600147F30002891A891EADF820100121BC
:1096D00001EB6000ADF81E004046F8F788F8BDF8D1
:1096E0002010081AADF81C004046F8F756F8BDF8EF
:1096F0001E1000230844ADF822002A4607A901A83D
:10970000F9F7BAFB5746BAF1010F01D04FEA6A07E1
:10971000204609F04DFF80463546002034E02146C2
:109720004046FBF769F801A80090DDF804C023B2B9
:109730000FFA89F200214046E04738B198F800005E
:10974000800190FBF7F02880012017E06100284697
:10975000FBF74DF814E008EB000218F8001012F8BF
:10976000012C914204D105EB400131F8021C02E0CA
:10977000890191FBF7F125F81010401CA042EADBAB
:1097800005EB440509F101008146A042C7DB4046D4
:1097900009F05AFF01A8F9F7E9F8012F14D020B217
:1097A000324639460546FFF7E1FE0AF0010038442B
:1097B00001B2012927DD4FF47F5090FBF1F2002028
:1097C00097B204FB04F318E000203146644304E040
:1097D00036F8102092090A54401C8442F8DC0AB082
:1097E000BDE8F08736F8102032B1FF2A0FD0920181
:1097F00092FBF1F226F81020401C8342F2D8324648
:109800002846FFF7B3FE00203146644306E026F801
:109810001070F1E716F810200A54401C8442F9DC5D
:10982000DDE7F0B597B0074615460E4601A8F9F7F3
:10983000F1FBFF2211461046F8F75DF80090BDF8E5
:1098400000000090BDF80000ADF80800002432468A
:1098500001A93846F9F7CAFB0FA8F8F7FFFD2B4618
:1098600032460FA938460094F8F764FB17B0F0BDF4
:10987000FEB5066804460A46708C00250421C0F334
:1098800005130BE0F06801EBC507C059870104D54B
:10989000A76820F07F40B84203D06D1CAB42F1D8DE
:1098A000FEBDA18844295CD00EDC33294CD006DCF7
:1098B000202956D0222954D0302913D151E03429FF
:1098C00042D036290ED14CE0622940D006DC47292F
:1098D00047D0552945D0572904D135E0672933D0E1
:1098E000682931D062B3FF2A2CD0D4E903031B1AB4
:1098F000534300EB23200090F068012701AA50F8A1
:1099000035000AF065FE60B1DDE90001884208D14A
:10991000BDF80020BDF804309A4202D1884200D13F
:109920000027F068A188009A50F835000BF054F831
:10993000002FB5D0A288A1682068FDF7E5FCFEBD28
:10994000E068D8E72069D6E7FF2AFBDAF8E7E068A5
:109950000028F7D02369002BCDD0802ACBDB0093E1
:10996000CAE7002A01DCA0892AE0FF2A01DB208A5D
:1099700026E0208AD3B280B2020242EA1020A789F0
:1099800082B2B8B2070247EA10201B1DDF080E4B57
:1099900080B240EA004042EA024218401A40121ADD
:1099A0007A4300EB5210184040EA104080B20202A5
:1099B00042EA1020ADF8080080B20290BDF808001D
:1099C000ADF8000098E700001FF8E0072DE9F0412E
:1099D000046800262648A788256800F0C3FF10E029
:1099E000A1420BD008682268904207D18868A2681B
:1099F000904203D18888A288904237D01C4800F05A
:109A0000C3FF0100ECD1002E30D1688C0421C0F3DB
:109A1000051229E0E86801EBC603C058830122D58E
:109A2000A36820F07F4098421DD12146104801F0E4
:109A300034F8204609F01AFEE868394600EBC604FF
:109A400020680AF0BBFEE86850F836000AF015FE00
:109A500000280BD06068216820F07F422846BDE8CE
:109A6000F041FDF727BD761CB242D3D8BDE8F081A6
:109A700024D5002070B50468A068A28800F47F0691
:109A800031462068FCF7AFFBE060A5880020A0808D
:109A900023462A463146206800F00CF8A580A168CC
:109AA0002068F7F7F6F9A1880068E268BDE8704021
:109AB0000AF092BF2DE9FF5F074691460E4600244B
:109AC000254800F068FF05464FF4702B4FF0040A5C
:109AD0003CE0039885423BD029461F4800F058FFE0
:109AE00080462868B84230D1A868B04201D05E45AF
:109AF0002BD1A988494503D0A9F57F41FF3924D14D
:109B0000002411E0F8680AEBC40141588A010AD523
:109B10005E4503D021F07F41B14204D150F83400BA
:109B2000A9880AF04BFE641C788CC0F30510A04293
:109B3000E8D800212846F7F7E3FC2946064800F05C
:109B4000ACFF284609F092FD01244546002DC0D106
:109B500004B02046BDE8F09F24D500202DE9F74F42
:109B6000934682B0044600216E22FCF73CFB06B20D
:109B7000204600216D22FCF736FB05B216B9B5F57B
:109B8000807F67D0204600216F22FCF72CFBADF8C8
:109B90000000204600217022FCF725FBADF80200F2
:109BA000BDF9000004F11401C0F3413264274FF401
:109BB000FA688A464FF47A79012A14D120F4C04019
:109BC000404510DC0846F7F7EEFD0146BDF9000000
:109BD00020F4C040484501DDC0F57A70414391FB57
:109BE000F7F0ADF80000BDF90200C0F341310129E2
:109BF00014D120F4C040404510DC5046F7F7B5FDC5
:109C00000146BDF9020020F4C040484501DDC0F521
:109C10007A70414391FBF7F0ADF80200A08ABDF8DD
:109C20000010BBF1000F0844ADF80000E08ABDF859
:109C300002100844ADF8020006D0704206B24FF49C
:109C4000803090FBF5F005B26B462A46314603980A
:109C500009F062FF05B0BDE8F08FF0B5D0E9064627
:109C6000059D4FF480772EB9BC4203D108021860DD
:109C7000100239E0B0F928C0A1EB0C01B0F92AC0FC
:109C8000A2EB0C029EB1BC421AD1446906694C4356
:109C900006FB1244066A06EBA4041C6003694B43EE
:109CA0004169406A01FB023100EBA1001CE0066A39
:109CB00001FB04611960416A806902FB001013E036
:109CC000466907694E4307FB12666643046A04EB64
:109CD000A6241C6003694B43416901FB0231826980
:109CE000406A514300EBA1202860F0BD0000000055
:109CF0007F4D0108654E010800000000A1510108D8
:109D0000730073004A020000000001E001E000005F
:109D100000FF0055AAFF0011223344556677889949
:109D2000AABBCCDDEEFF000102030405060708090B
:109D30000A0B0C0D0E0F101112131415161718190B
:109D40001A1B1C1D1E1F20212223242526272829FB
:109D50002A2B2C2D2E2F30313233343536373839EB
:109D60003A3B3C3D3E3F40414243444546474849DB
:109D70004A4B4C4D4E4F50515253545556575859CB
:109D80005A5B5C5D5E5F60616263646566676869BB
:109D90006A6B6C6D6E6F70717273747576777879AB
:109DA0007A7B7C7D7E7F808182838485868788899B
:109DB0008A8B8C8D8E8F909192939495969798998B
:109DC0009A9B9C9D9E9FA0A1A2A3A4A5A6A7A8A97B
:109DD000AAABACADAEAFB0B1B2B3B4B5B6B7B8B96B
:109DE000BABBBCBDBEBFC0C1C2C3C4C5C6C7C8C95B
:109DF000CACBCCCDCECFD0D1D2D3D4D5D6D7D8D94B
:109E0000DADBDCDDDEDFE0E1E2E3E4E5E6E7E8E93A
:109E1000EAEBECEDEEEFF0F1F2F3F4F5F6F7F8F92A
:109E2000FAFBFCFDFEFF8080808181828283848535
:109E30008687898A8C8D8F91939597999B9EA0A2F6
:109E4000A5A7AAADAFB2B500FF1FFF1F01E001E05B
:109E50007424060800000020B0530000CA920208D3
:109E6000502E0608B05300206017010024C20008DD
:109E700070B5044600256FF02F0608E02068411CED
:109E80002160007805EB850106EB4101451820684B
:109E9000007800F004F80028F0D1284670BD303872
:109EA000092801D801207047002070472DE9F047AC
:109EB0000F46814690461146384600F00CF940B1F5
:109EC00000224146384600F0B2F828B10020BDE833
:109ED000F0874FF0FF30FAE70026384606F07BF8AF
:109EE000401E0FFA80FA384606F04FF8401E02B2C4
:109EF000B8F80210B7F90200091A09B200290FDDFB
:109F00003B88012663F30F0460F31F44BB880844B9
:109F100063F30F0560F31F45C9F80040C9F804500A
:109F2000B8F906007988411A511A09B2002913DDDF
:109F3000B7F9062090420FDA3A8862F30F04BA8824
:109F400060F31F4462F30F05084460F31F4509EBFB
:109F5000C600761C04604560B8F90200B7F902102B
:109F6000884200DC0846B8F90610B7F9062091428D
:109F700000DB1146B8F80030B7F90020091A9B1A27
:109F80001BB209B2002B10DD00290EDD62F30F04B5
:109F90001A4462F30F05421862F31F4509EBC6022B
:109FA00060F31F4414605560761CB8F904203B88A8
:109FB000D71AAAEB07031BB2002B0EDD62F30F04C6
:109FC00060F31F441A4462F30F05084460F31F4511
:109FD00009EBC600761C04604560304677E770B533
:109FE000B1F90040B2F900309C4200DD2346038005
:109FF000B1F90240B2F90250AC4200DC2C46448078
:10A00000B1F90450B2F90460B54200DB35468580F1
:10A01000B1F90610B2F90620914200DB1146C18069
:10A020000120AB4201DC8C4200DD002070BDF8B5A0
:10A030000D460446B0F90000B1F9001016468842FA
:10A0400047DBB4F90210B5F90220914241DBB4F9C3
:10A050000410B5F9042091423BDCB4F90610B5F9BF
:10A060000620914235DC96B3ADF800006088ADF86B
:10A07000020032466946284600F099F8002827D0A9
:10A08000A088ADF800006088ADF80200324669464D
:10A09000284600F08CF800281AD02088ADF800007F
:10A0A000E088ADF8020032466946284600F07FF8A5
:10A0B00000280DD0A088ADF80000E088ADF80200BF
:10A0C00032466946284600F072F8002800D0012088
:10A0D000F8BD0020F8BDB0F90020B1F904309A4273
:10A0E00013DCB0F90420B1F900309A420DDBB0F96D
:10A0F0000220B1F906309A4207DCB0F90600B1F946
:10A100000210884201DB0120704700207047F8B53B
:10A110000D460446B0F90400B1F900101646884215
:10A1200043DBB4F90600B5F9021088423DDBB4F90F
:10A130000000B5F90410884237DCB4F90210B5F913
:10A140000620914231DC76B3ADF800006088ADF8AE
:10A15000020032466946284600F029F818BBA0885C
:10A16000ADF800006088ADF8020032466946284626
:10A1700000F01DF8B8B92088ADF80000E088ADF80F
:10A18000020032466946284600F011F858B9A08806
:10A19000ADF80000E088ADF8020032466946284676
:10A1A00000F005F808B10020F8BD0120F8BD2DE948
:10A1B000FC4105460F46B1F90000B5F90010144600
:10A1C00088423BDBB5F90410884237DCB7F902005E
:10A1D000B5F90210884231DBB5F9061088422DDC52
:10A1E000002C76DD284605F0F6FE00EBD070461018
:10A1F000284605F0CAFE00EBD0704010864200DA17
:10A200003046844200DD04462888ADF800002888E6
:10A2100000222044ADF804006888ADF80200688888
:10A2200039462044ADF806006846FFF7C0FF40B14C
:10A23000BDF804002044ADF804003FE00020BDE874
:10A24000FC81E8880022001BADF80200E888ADF828
:10A25000060039466846FFF7AAFF28B1BDF804009A
:10A260002044ADF8040011E0A8880022001BADF8DE
:10A270000000A888ADF8040039466846FFF797FF4C
:10A2800050B1BDF80000001BADF80000BDF80200A1
:10A29000001BADF8020016E06888ADF8020068887F
:10A2A00000222044ADF8060039466846FFF77FFFDC
:10A2B00070B1BDF80000001BADF80000BDF806004D
:10A2C0002044ADF806003946684609F0C3FCB6E7FD
:10A2D000FFE70120B3E710B5B1F90030B2F9004053
:10A2E000A34200DB23460380B1F90230B2F90240F9
:10A2F000A34200DB23464380B1F90430B2F90440A5
:10A30000A34200DC23468380B1F90610B2F906208F
:10A31000914200DC1146C18010BD00000849496827
:10A320000AE04A68824202D00A68824203D10A7E69
:10A3300042F001020A7649690029F2D17047000013
:10A3400044520020704700000421014800F027BB60
:10A35000F4D400202021014800F021BB0CD50020BE
:10A360002DE9FF410446DDE90A571E004FF00000C9
:10A3700002D1B5F5807F2BD0039001900290ADF80B
:10A380000C100090ADF80410ADF80A20ADF80E20C6
:10A390003B462A463146684609F0BEFB3B462A4604
:10A3A000314601A809F0B8FB3B462A46314602A8CF
:10A3B00009F0B2FB3B462A46314603A809F0ACFB44
:10A3C000BDF90030BDF90420934209DA1D4608E0CA
:10A3D0002080491E6080A180521EE280BDE8FF817E
:10A3E0001546BDF90800BDF90C10884201DA064691
:10A3F00000E00E46B54205DA934201DA184604E061
:10A40000104602E0884200DB0846801E2080BDF92D
:10A410000030BDF90400834201DD1D4600E0054621
:10A42000BDF90820BDF90C108A4201DD164600E096
:10A430000E46B54203DD834206DD184604E08A423B
:10A4400001DD104600E00846801CA080BDF9023006
:10A45000BDF90620934201DA1D4600E01546BDF91C
:10A460000A10BDF90E00814201DA0E4600E00646F0
:10A47000B54205DA934201DA184604E0104602E0DC
:10A48000814200DA0846801E6080BDF90230BDF9C5
:10A490000620934201DD1D4600E01546BDF90A1075
:10A4A000BDF90E00814201DD0E4600E00646B542D0
:10A4B00005DD934201DD184604E0104602E08142CA
:10A4C00000DD0846801CE08088E700002DE9F041AF
:10A4D00015460E460746114C0AF08AFE80462B466A
:10A4E00032463946204607F03FFF20B10020A062E7
:10A4F000E06950B110E020462C210DF0F2FD4FF044
:10A500000040A0620020BDE8F08140460AF069FEEC
:10A51000E06108B90120E0612046F4E730D5002071
:10A5200010B51421074800F03AFA07F0E3FE40B1F5
:10A530000549016005494160054981600549C160DF
:10A5400010BDFEE718D50020DD1C020851200208CE
:10A5500015220208A91C020870B505460C460846DB
:10A5600010210DF0BEFD28680078012804D00228D3
:10A5700007D0042807D008E0A88A2080E88A6080F5
:10A5800003E0E86800E00A20606028684268002A6A
:10A5900003D02146BDE87040104770BD2DE9FE4351
:10A5A0000446808A10B9E08A002874D0D4F82C8040
:10A5B0005FEA080010D1204602F042FD5FEA000881
:10A5C00069D0204604F06CFC00220921404606F0C8
:10A5D00087FD607880075ED44FF4807900274D4670
:10A5E00046460021304609F0D7F9384407B2002129
:10A5F000304609F0D7F9C11700EB1160001210FBCB
:10A6000005F005B23046FBF769F80600E9D10FB94D
:10A610004D450CD0784201B24FF4803090FBF5F0FC
:10A6200002B26B4604F11400009609F075FAADF819
:10A630000860ADF8046094F8400000F00F000328B3
:10A64000404616D0FBF79CF905464046FBF752F80A
:10A6500003460C200090B4F916102A46404602F03A
:10A660009CFBADF804004046FBF796F8C10713D0F9
:10A6700018E0FBF719F905464046FBF7B5F8024626
:10A6800003200090B4F914102B46404602F085FBDD
:10A69000ADF80800E7E736E0BDF90810002901DD54
:10A6A000ADF80860810705D4BDF90810002901DA6A
:10A6B000ADF80860410705D4BDF90410002901DD9B
:10A6C000ADF80460000705D4BDF90400002801DAE4
:10A6D000ADF8046001AA02A920460BF01AFBBDF9EF
:10A6E0000420BDF908104046F1F7C7FE60788007E6
:10A6F00009D4208BBDF8081008442083608BBDF876
:10A70000041008446083BDE8FE832DE9FC5F044625
:10A71000C06A5FEA000B71D094F8400000076DD06A
:10A7200008F0A2F8019000684021457E5846FBF7EA
:10A73000C5FE4FF0000818B9A4F81E80A4F81C80CC
:10A740005846FBF70FF982465846FBF712F90646C2
:10A7500094F840004FF0640900F00F000C2802D07C
:10A7600003284CD09AE0A4F81C8056B1B4F91E50CE
:10A77000002708F079F800684946407EC0F164007F
:10A7800022E0E08BC5F1640110FB01F191FBF9F0CF
:10A79000E0835846FAF7AEFF05465846FBF7F0F857
:10A7A00002460C200090B4F91E102B46584602F0C9
:10A7B000F4FAE083024600231EE07A1917B210FB78
:10A7C00005F292FBF1F215B2002DF6D1ADF8007052
:10A7D000A4F81E806A46002120460BF09AFA41F642
:10A7E000FF72BDF900305142584602F0BFFDBDF87E
:10A7F00000100123084402B200214CE09AE0A4F8C2
:10A800001E80BAF1000F0AD0B4F91C50002708F0DE
:10A810002BF800684946407EC0F1640022E0A08B1E
:10A82000C5F1640110FB01F191FBF9F0A0835846DA
:10A83000FAF7DAFF05465846FBF736F803460320D9
:10A840000090B4F91C102A46584602F0A6FAA083DC
:10A85000014600231EE07A1917B210FB05F292FBA5
:10A86000F1F215B2002DF6D1ADF80070A4F81C80FD
:10A870000022694620460BF04CFA41F6FF72BDF902
:10A8800000305142584602F0EFFCBDF800100123A1
:10A89000084401B200225846FCF7A6FEA08B00280F
:10A8A00048D1E08B002845D1C6B95846FBF768F877
:10A8B00005465846FAF71EFF002D06DC00280DDD80
:10A8C000002D02DA01232A4604E0002806DA0123DB
:10A8D000404202B200215846FCF786FEBAF1000F52
:10A8E00019D15846FAF780FF05465846FAF7DCFFBB
:10A8F000002D07DC00280EDD002D03DA01230022E5
:10A90000294605E0002806DA01230022404201B270
:10A910005846FCF769FE0A215846019A06F0E0FB0A
:10A920006078800706D414F8400F20F00F002070E4
:10A9300044F8148CBDE8FC9F70B5054600F012F891
:10A9400004460CE02146284600F01EF80646214643
:10A95000284600F0A2F8204608F088FE3446002C75
:10A96000F0D170BD002800D04068704700B50346A4
:10A970000022FFF7F7FF03E01846521C00F004F82E
:10A980000100F9D1104600BD0068091D405870470C
:10A99000006840587047002800D080687047002247
:10A9A0004260C91C21F0030182600160704770B5EC
:10A9B00004460068083008F0CDFD050013D00146BC
:10A9C000002220460AF0A8FF2946204662680AF0C5
:10A9D0009AFF616819B12A4620460AF09DFF65601A
:10A9E000A06800B9A560284670BD2DE9F0410D466C
:10A9F00006000AD04DB1FFF7B5FFA84208D1304696
:10AA0000FFF7D5FF041E01D01EE00020BDE8F08155
:10AA10003068083008F09EFD041EF7D030682246EA
:10AA20004759304639460AF06EFF3A4621463046CD
:10AA30000AF072FF2246294630460AF06DFF2A4688
:10AA4000214630460AF05FFF2046DFE770B5044636
:10AA50000068083008F07EFD050013D00146002292
:10AA600020460AF050FF29462046A2680AF054FF0B
:10AA7000A16819B12A4620460AF045FFA560606822
:10AA800000B96560284670BD28B1416809B9806881
:10AA900008B1002070470120704770B504000DD048
:10AAA000FFF760FF00228842204608D1FFF76CFFC5
:10AAB000606010B1002201461EE0A26070BDFFF789
:10AAC0006AFF8842206808440AD10168A16029B160
:10AAD0002046BDE8704000220AF015BF626070BDDC
:10AAE00005682046FFF750FF0646024629462046E5
:10AAF0000AF009FF2A4631462046BDE870400AF0B8
:10AB00000BBFC0F30410072800D9072070470000CE
:10AB1000A0F57F41FF3905D0002804D0712803D269
:10AB200008490AE01F2070470749713880B2096858
:10AB300029B1064A5268904201D2085C7047002051
:10AB400070470000BC6E02082453002038530020D8
:10AB50002DE9F041094C90460E4662681D460746B5
:10AB600019469047306020B1286862683844002157
:10AB70009047C8F80000BDE8F08100005453002061
:10AB80002DE9F04F87B08A46DDE910581F469346FD
:10AB90000446002105B129805CB12078002809D045
:10ABA000BAF1000F05D0002618F0060F15D00020CE
:10ABB00004E0002007B0BDE8F08F401C215C0A29AA
:10ABC00004D00D2902D00029F7D100E0401C002D4F
:10ABD000F0D04FF0FF312980ECE75FEA887001D5B3
:10ABE00041F6FF77894608468DF81010059125E05B
:10ABF0000598CDF8189058B3002104ABCDE9023187
:10AC00000DF1180CCDE9008C20443B465A465146C4
:10AC10000AF036FC06997A1A314417B20EB288B19E
:10AC200005990844059021780A290BD00D2909D0EF
:10AC3000205C0A280ED00D280CD00598205C08B1A5
:10AC4000002FD5DC059848B105B12E800598B1E7F5
:10AC50000121D2E70598401C0590F3E7064A05A9B3
:10AC60002046526890470146002DEFD00022504602
:10AC700006F04BFB06B2E8E75453002000230278AD
:10AC8000232902D0012A0DD00FE02AB10021012A88
:10AC900004D0022A04D008E0012101E0017004E0A0
:10ACA000017001E0202902D00123184670470221DB
:10ACB000F6E72DE9F0410B460F468046024600219B
:10ACC00008460AF0E5FD05460026401C08F042FC57
:10ACD000040008D066553B464246691C0AF0D8FD80
:10ACE0002046BDE8F081FEE72DE9F047984614467E
:10ACF0000D468246DDF8209013E0660806FB0857F3
:10AD0000394650464A469047002808DD44F3000083
:10AD1000C0EB540407EB0805A4F1010401E005DAD7
:10AD20003446002CE9D12046BDE8F0873846FBE7E1
:10AD30002DE9FC5F0CAD9E4692468B4695E81201CC
:10AD4000DDE91132DDE90F7C96074FF0300519D4AB
:10AD500053B1D60708D002F00C0656EA080603D015
:10AD60005B1E01E00D55641C644504D2202CF9D310
:10AD700001E00D55641C5FEAC27903D09C4201D208
:10AD8000202CF6D3D60624D556050AD44CB16445FA
:10AD900001D09C4205D1641E03D0102F03D1641E44
:10ADA00004E0102F02D0022F0AD00EE0960603D442
:10ADB000202C1ED2782606E0202C1AD2582602E03B
:10ADC000202C16D262260E55641C202C11D20D5553
:10ADD000641C202C0DD2B8F1000F01D02D2506E007
:10ADE000550701D52B2502E0150702D520250D5565
:10ADF000641CCDE900EB064655468B4698469146C5
:10AE0000900713D1274606E02A46DDE900316D1C84
:10AE10002020B0477F1C4745F6D307E02A466D1C2B
:10AE2000641EDDE900311BF80400B047002CF5D1A9
:10AE30005FEA897006D409E02A46DDE900316D1C1D
:10AE40002020B047A5EB0A014145F5D32846BDE8CF
:10AE5000FC9F2DE9F04F8FB099468B46DDE918181D
:10AE6000DDE91C63DDE91A4786469246002009B9F0
:10AE700023F010035A0507AD00D5C9B1B1FBF4F2B8
:10AE800004FB1212D2B20A2A01D2303209E05FEA80
:10AE9000836C02D54FF0410C01E04FF0610C62442D
:10AEA0000A3AB1FBF4F12A54401C09B12028E5D339
:10AEB000CDF80880CDE90563CDE90050CDE9034721
:10AEC0004B46524659467046FFF732FF0FB0BDE879
:10AED000F08F2DE9FF4F8FB01CACDDE9239594E88E
:10AEE000030820AC94E8C004002450EA010201D118
:10AEF00025F010056A050DF11C0802D550EA010283
:10AF000017D032463B460DF08DF8D2B20A2A01D254
:10AF1000303206E0AB0601D5412300E061231A443C
:10AF20000A3A08F80420641C50EA010201D0202CDF
:10AF3000E7D3CDE90084CDF808B0CDE90595CDE99A
:10AF4000036A0FAF97E80F00FFF7F2FE13B0BDE8FA
:10AF5000F08F9A4200D28854704770472DE9FF4F16
:10AF600089B082460A980024169D002801D1DFF896
:10AF7000F0A367E1252802D02246641CE2E1491CC7
:10AF8000002608460C9101782B291BD004DC2029CF
:10AF90001BD0232904D11BE02D290ED0302909D044
:10AFA0000027C8B2FEF77BFFA8B10CA8FEF760FF30
:10AFB00007461CE046F0010601E046F00206401C90
:10AFC0000C90E0E746F00406F9E746F00806F6E7DD
:10AFD00046F01006F3E70C9801782A2907D180CDB6
:10AFE000002F02DA46F002067F42401C0C900C98BB
:10AFF0004FF0000801782E2917D1401C0C9046F420
:10B0000080660078FEF74BFF20B10CA8FEF730FFFA
:10B0100080460AE00C9908782A2806D101CD00283C
:10B0200000DC0020491C80460C910C9801786C29AA
:10B030000AD004DC68290FD06A2918D127E07429C6
:10B0400028D07A2913D125E0401C0C90017846F4D1
:10B0500080766C291BD00AE0401C0C90017846F0E9
:10B060008006682903D146F04006401C0C90024639
:10B070000078692822D015DC62281FD00DDC252835
:10B0800077D050281AD058287FF476AF16E046F4CF
:10B090000076EAE746F48076E7E763286AD064281A
:10B0A000F2D10BE073286FD004DC6F2806D0702833
:10B0B000EAD103E0752801D07828E5D178280DD0B1
:10B0C00058280BD070280BD0502809D06F2816D0E4
:10B0D000622816D00A2126F0100616E0102107E09B
:10B0E0005078102146F48876562804D1521C0C92D0
:10B0F0001078582807D01078502804D005E008218F
:10B1000008E0022106E046F020061078692803D006
:10B11000642801D026F00C06700501D526F0010642
:10B120001078692813D0642811D0562854D0B0055F
:10B1300060D5ED1D0020CDE90410CDF818800290F7
:10B14000CDE9077625F00705F5E8020121E0B00515
:10B1500028D5ED1D25F007050023F5E802020DF1C5
:10B160001009002A89E80A01CDE9077603DA0121EE
:10B1700002E0E4E070E000210023029119461B1A6E
:10B18000914102DA114604E08EE00021404261EB79
:10B190000201CDE90001DDE90A1322465046FFF71E
:10B1A00098FE4BE0F00503D501CD0BE0404210E0E6
:10B1B000700602D515F8040B04E03006F4D535F816
:10B1C000040B00B2CDE90218CDE90476C10F0028C6
:10B1D000ECDDCDE900012BE001CD4168096800916B
:10B1E00003680B98021B0A9801195046FFF7B6FE38
:10B1F000044424E0F00508D5CDE90218CDE9047631
:10B2000002CD0020CDE9001012E0700602D515F83D
:10B21000040B06E0300603D535F8040B80B200E0DD
:10B2200001CDCDE902180021CDE90001CDE9047678
:10B23000DDE90A1322465046FFF70BFE04460C9840
:10B24000401C0C900C99087800287FF493AE0B9862
:10B2500084427BD222467AE04FF00108B00707D53E
:10B260000BE02246DDE90A13641C2020D446E047A7
:10B27000404608F10108B842F3D3DDE90A1322463B
:10B2800015F8040B641CD446E047B00706D4D6E793
:10B290002246DDE90A13641C2020D047414608F10C
:10B2A0000108B942F4D3CAE755F804BBB8F100006D
:10B2B0005A4601D0014601E04FF0FF31584600E008
:10B2C000401C03780BB1491EFAD2A0EB02097005AD
:10B2D00005D548464146C14500D308468146B007DA
:10B2E00007D514E02246DDE90A13641C2020D44669
:10B2F000E047494609F10109B942F3D307E0DDE926
:10B300000A1322460BF1010B641CD446E0479BF85C
:10B31000000020B17105F2D5B8F10108EFD2B007F5
:10B3200006D48CE72246DDE90A13641C2020D047AE
:10B33000494609F10109B942F4D380E706E0224603
:10B34000641C2520DDE90A13D04778E7421E034636
:10B3500000200A99D0470DB02046BDE8F08F0000CC
:10B360005BAF010810B503004FF000000DD04A1E7E
:10B37000114200D0FEE71944491E91430A46B1F537
:10B38000004F02D20C2A01D9084610BD0C2010BD76
:10B3900008444A1E401E9043114200D0FEE7704709
:10B3A0002DE9F0410446012000250F4660862E4617
:10B3B0000BE01B490CF0DBFE10B16D1CADB202E0DE
:10B3C000608E401C6086761CB6B257F8260010B11D
:10B3D00001780029EDD1208EA8421ED0A06A002657
:10B3E00010B108F043F9A662E06A10B108F03EF926
:10B3F000E662E80008F0AEF8A06238B1680008F034
:10B40000A9F8E06218B1A16A11B102E0FEE7FEE717
:10B41000002569000CF065FE2586BDE8F08100007E
:10B420001406020870B5044640680D4608B1FFF7DF
:10B43000F9FF2268002A04D029462046BDE8704062
:10B44000104770BD89B204F0AFBC89B204F032BDC0
:10B4500070B50D46044600F04DF800B1FEE768688F
:10B46000616820F00300001D08446060204600F081
:10B4700049F8204670BD4068103120F00300884232
:10B4800001D301207047002070472DE9FC47054695
:10B4900048680C4620F0030001AA69460AF01DFA2C
:10B4A000DDE9006005EBC61101EB80098046D9F8A3
:10B4B000380060B164B1C4E9020504F10807C46052
:10B4C00038460421FFF764FF874202D0FEE7FEE71B
:10B4D000FEE7C9F838400123286903FA06F108435A
:10B4E000286105EB860003FA08F142690A434261CC
:10B4F000BDE8FC87406830F0030001D000207047B1
:10B500000120704710B5044600F08CF8046010BDAF
:10B510002DE9FC474FF0000780460E0001973D469D
:10B52000009745D00C460DF1040AE946802907D35F
:10B5300008460BF00FFB411F01208840401E0444C9
:10B540004A46514620460AF0C8F9019C092C2FDAD8
:10B5500008EB8400009940694FF0FF3202FA01F1D4
:10B56000454608400CD1641C2869A240104016D002
:10B570000BF0E8FA0446019005EB8000406980B1C9
:10B580000BF0E0FA05EBC411009001EB8000856B35
:10B5900075B1686820F00300B04203D2FEE73D4673
:10B5A000F6E7FEE7DDE90032294640460AF022FBD5
:10B5B0002846BDE8FC8710B50446FFF7A3FF4168A5
:10B5C00041F002014160606840F00100606010BD20
:10B5D00010B5044600F026F8416821F002014160F0
:10B5E000606820F00100606010BD70B506460D4631
:10B5F000084600F017F8040008D0207910F0010F79
:10B600000ED02846FFF776FF08B1FEE7FEE7214699
:10B61000304600F03EF821462846FFF719FF054660
:10B62000284670BD10B5426800F1080122F00302FF
:10B63000121F8C18FFF75EFF00B1FEE7204610BD19
:10B6400070B506460C004FF000001FD0FAB120790B
:10B65000154610F0010F1BD011462046FFF70BFFD7
:10B6600078B12946204600F025F805462046FFF728
:10B6700049FF6868294640F0020068603046FFF7DD
:10B6800004FF2046FFF7A4FF04F1080070BDFEE7A9
:10B69000FEE77CB5054648680C4620F003006A4684
:10B6A00001A90AF01AF9DDE90032214628460AF01C
:10B6B000A1FA7CBD2DE9F0410D4604460830091F72
:10B6C0004618606806F1080720F00300401BA0F14F
:10B6D000040838460421FFF75BFE874200D0FEE7EE
:10B6E000606808EB050120F00300091D884200D0C6
:10B6F000FEE7307900F0030040EA0800706020F0B7
:10B7000003000C2800D2FEE7207900F00300284354
:10B7100060603046FFF74FFF3046BDE8F08170B5FE
:10B7200005F0D1FC0546F9F7D9FF0446284605F097
:10B730000EF801462046BDE87040002209F07EBCAC
:10B740002DE9F04F0C4687B005460021F9F7C6FEFB
:10B7500060B32146284600F021F92146284600F032
:10B760006FF80021284608F08DF805900021284642
:10B7700008F0CAF804900021284608F03CF8012897
:10B7800000D0002080460021284608F017F9064620
:10B790000021284608F052F842F2D17907464E457A
:10B7A0000BD1688C000508D4012607E007B02046BD
:10B7B000BDE8F04F1C210CF094BC00262846F9F798
:10B7C0000DFFDFF878A0834628460021BAF8042050
:10B7D000FAF709FDD4F810C0A3682168CDF800C0BD
:10B7E000CDF80C80CDE90131C2B231465846059BF7
:10B7F00002F096FC20834F4504D1688C400501D4AB
:10B80000012600E000262846F9F7CCFE0746284628
:10B810000021BAF80820FAF7E6FCC2B260690025F8
:10B820006368E1688DE82B0031463846049B02F0DE
:10B8300077FC608307B0BDE8F08F000098520020CD
:10B840002DE9F34F81B00C46019802F051FA804681
:10B850000198F9F7C3FE8346404600F08AFB206159
:10B86000400007F0A5FE20602069400007F0A0FE20
:10B87000002541F69A79A06035E038F91510454E5B
:10B8800049452FD10027DFF810A11CE03946019867
:10B89000F9F724FE51460090FAF717FE90B9009888
:10B8A00002F038FA01280DD1009802F029FAA842D6
:10B8B00008D10098FAF7E3FDB04203DB0098FAF7ED
:10B8C000DEFD06467F1C0198F9F71AFEB842DDD866
:10B8D000002E03DBA06820F8156003E0A1680020BB
:10B8E00021F815006D1C2069A842C6D800252F46F6
:10B8F000284641F69B764A4615E038F91010B142C9
:10B9000004DB0D44A5F5F8559B3D0BE0914204D1B5
:10B91000A16831F81010394403E0A36823F810102F
:10B9200039440FB2401C21698142E6D800210198B8
:10B9300007F0A8FF2169C1F1010200FB02B0C01BA2
:10B9400001B2002900DA002100224FF0FF37104633
:10B9500010E038F91030B3420BDBA3F5F8539B3BF2
:10B960001AB211FB02F3B3FBF5F3A76827F8103006
:10B970000746401C23698342EBD8002F07DBA81A37
:10B980004843B0FBF5F0081AA16821F81700BDE89C
:10B99000FE8F000001E0FFFF010006002DE9F84FD7
:10B9A0000C46834602F022FB804600F0E2FA60611A
:10B9B000400007F0FDFD60606069400007F0F8FDA1
:10B9C000002541F69A79E06035E038F91510474EC8
:10B9D00049452FD10027DFF818A11CE03946584609
:10B9E000F9F77CFD51460090FAF76FFD90B9009889
:10B9F00002F00EFB01280DD1009802F0FFFAA842D8
:10BA000008D10098F9F72FFEB04203DB0098F9F750
:10BA10002AFE06467F1C5846F9F772FDB842DDD86B
:10BA2000002E03DBE06820F8156003E0E1680020E9
:10BA300021F815006D1C6069A842C6D800252F4664
:10BA4000284641F69B764A4615E038F91010B14277
:10BA500004DB0D44A5F5F8559B3D0BE0914204D164
:10BA6000E16831F81010394403E0E36823F810105E
:10BA700039440FB2401C61698142E6D80021584622
:10BA800007F042FF81465846F9F78CFD6169C1F124
:10BA9000010209FB0200C01B01B2002900DA0021EB
:10BAA00000224FF0FF37104610E038F91030B34253
:10BAB0000BDBA3F5F8539B3B1AB211FB02F3B3FB6C
:10BAC000F5F3E76827F810300746401C63698342A6
:10BAD000EBD8002F07DBA81A4843B0FBF5F0081A93
:10BAE000E16821F81700BDE8F88F000001E0FFFFD2
:10BAF000010006002DE9FF4F87B0C878189CC007E9
:10BB00000D46002801D0E84800E0E848059001D043
:10BB1000E74800E0E748824601D1E54800E0E54813
:10BB200004906188A2884FF0000BA1EB02015846F7
:10BB300009B25A46D4F810C010E002EB82034FF06D
:10BB40001007E66807EB8307F75DFF070AD00827B1
:10BB500007EB8303F35AC91A09B2521C9445ECD877
:10BB6000002246E00C2707EB8303F35A184400B287
:10BB7000F3E709EB89031022E66802EB83020092E7
:10BB8000B25CD20733D1A8B191FBF0F70C2202EBE3
:10BB9000830E36F80E207A43042707EB830736F925
:10BBA00007C0062707EB8307F75F12B2974202DD53
:10BBB000904601E0FEE7B846C44501DD674602E075
:10BBC000974200DD1746974205D0009A4FF0010CCE
:10BBD000E34646F802C0E668082202EB8302B75249
:10BBE000E36833F80E20801AC91B00B209B209F1CC
:10BBF0000102236991464B45BBD8BBF1000F90D1A0
:10BC00000021079807F0F1FD012800D000208346AD
:10BC10000020ADF80800ADF80C0003A902A8CDE99A
:10BC200000012089B4F9022003B22878169909F09E
:10BC30007FFEE97811EA0B0F07D00798F9F7CEFCE1
:10BC4000BDF808100844ADF8080009990798F9F7FD
:10BC500045FC0BE098493046FAF737FC78B1E878B4
:10BC600009AAC0F38001079802F0ADF9060003D0DD
:10BC7000DDE909018842EDD10BB0BDE8F08F00216C
:10BC8000304607F0CBFDE8B30027384621690FE0C6
:10BC9000E26800EB800352F82320B24207D100EBA8
:10BCA0008002E168082000EB82000F5E02E0401C89
:10BCB0008142EDD8E878C007708C04D020F4806011
:10BCC00040F4006003E020F4006040F48060708481
:10BCD00006F11400804651468847B84228D03046C5
:10BCE000FAF77EFEB08AADF80000F08AADF80200E7
:10BCF000308BADF80400708BADF806003946404635
:10BD0000059A00E010E090476A462921304605F088
:10BD1000E7F93046F9F7E2FC3246222105F0E0F976
:10BD20003046FAF75DFE03E0708C20F440607084CA
:10BD300068784FF0000901280FD0022815D1049926
:10BD400006F114008847B4F90010491C21F00101E4
:10BD5000081A00EBD070401005E0049906F11400B9
:10BD600088472188081A0FFA80F9E87810EA0B0F43
:10BD700008D006F1140051468847BDF80810081A8B
:10BD8000ADF80800304600216B22FAF72CFA0FFAC2
:10BD900080F8304600216C22FAF725FA07B23046C7
:10BDA000FAF76DFB00903046F9F75DFC0146C8F3E9
:10BDB0004130012810D128F4C040B0F5FA6F0BDCF7
:10BDC000B0F57A7F01DDC0F57A70009A50436422A5
:10BDD00090FBF2F00FFA80F8C7F3413001280ED142
:10BDE00027F4C040B0F5FA6F09DCB0F57A7F01DDC9
:10BDF000C0F57A704843642190FBF1F007B2B18A34
:10BE00001498411A01EB080002B2F18A1598401A01
:10BE1000384401B2E878C007002802D0BDF9080014
:10BE200000E04846104407B201D0484601E0BDF9A1
:10BE3000080008440FFA80F857EA080019D0304685
:10BE4000FAF7CEFDB08A3844B082308B3844308364
:10BE5000F18A01EB0800F082718B01EB080070831E
:10BE60003046FAF7BDFD0023424639463046FAF720
:10BE70005DFEE87810EA0B0F0CD106F11400514674
:10BE8000884717990844BDF80C100844BDF80810FD
:10BE9000084406E0BDF80C1017980844BDF80810D7
:10BEA000081AADF80800DAE6470002083D0002086B
:10BEB000CBFF01087FFF010801000600F8B504462A
:10BEC00005F001F90546204605F0BFF8064628466C
:10BED000F9F704FC04462B2E37D00A2E34D106F095
:10BEE000C3FC10B1007901282ED069462846F9F725
:10BEF0005BFC94F82C0010F00C0F28462ED0F9F7BC
:10BF00006DFB05460021204607F07BFC0128BDF9AA
:10BF1000000005EBD5711ED000EB610090FBF5F041
:10BF200001B2002900DA0021608D0025884200D08E
:10BF300001250122204609F081F8002D04D00022BD
:10BF40001C21204605F0CCF8F8BD618DBDE8F84015
:10BF5000002209F073B8C0EB6100DFE7F9F722FBBC
:10BF6000BDF9021000EBD07201EB620191FBF0F021
:10BF7000D6E70146002041F6FF7200E0401C31F98F
:10BF800010309342FAD1704708B50846114604F0C4
:10BF9000B2FD0090BDF8000008BD00002DE9F04F93
:10BFA00093B0834605F051F80646584605F08BF8E5
:10BFB0000446122E7ED0152E01D0182E7BD1FAF712
:10BFC0005EFA06902046F9F74EFB059020460021C8
:10BFD0003222FAF708F90546204600211222FAF724
:10BFE00002F928440FFA80F8204600211322FAF7BC
:10BFF000FAF828440FFA80FA204600211022FAF7B6
:10C00000F2F8284407B2204600211122FAF7EBF893
:10C010002844618E0FFA80F901EB0800ADF83C006E
:10C02000A08E3844ADF83E0094F8390000F00300CB
:10C0300001287DD00FA9E08ECDE90001DDE90521C1
:10C04000B4F9303003A8FEF78BF9BDF80C10A08AC4
:10C050000844ADF80C00BDF80E10E08A0844ADF8B5
:10C060000E00BDF81010A08A0844ADF81000BDF80D
:10C070001210E08A0844ADF8120004F114010D46D4
:10C0800010A80D9103F06CFF03A9284603F068FF88
:10C090005946D24807F07AFB012860D110A90D98C3
:10C0A00003F05EFF152E5AD1E08D002857D0A08DE9
:10C0B000002801E056E052E051D0E08E00284ED03A
:10C0C000584604F0C8FF064601A80D9903F048FF42
:10C0D000204606F0C7FA054694F8390000F0030040
:10C0E00001287CD0BDF81000BDF80C10401ABDF836
:10C0F00004100844ADF80800BDF81200BDF80E1099
:10C10000401ABDF806100844BDF80410ADF80A0046
:10C1100001EB0800ADF80400BDF80600BDF80810FA
:10C120003844ADF80600A1EB0A00ADF8080000E0C5
:10C130007DE0BDF80A10A1EB0900ADF80A0094F803
:10C14000381001F0030001286FD089076DD0022854
:10C150006CD00023194630460D9AF5F79DFE13B0BA
:10C16000BDE8F08F584604F0ACFF05460078022881
:10C17000F5D094F838004FF00106C14389074ED03E
:10C1800000F0030102294AD0C0F38400042801D042
:10C19000012844D1204600214622FAF724F8C0B2F3
:10C1A000FF283CD1208ED0BB584604F08AFF0746BA
:10C1B000E08EB0F5807F34D02046F9F754FA8046FF
:10C1C0002046FAF75CF9014604F13202E08ECDE92F
:10C1D00000020023424602A8FEF7C2F800E02BE06E
:10C1E000BDF80800A18A00220844ADF80800BDF897
:10C1F0000A00E18A0844ADF80A00BDF80C00A18AE3
:10C200000844ADF80C00BDF80E00E18A0844ADF812
:10C210000E0002A93846FDF70AFF00289FD12E70B4
:10C220009DE7002204F11401F4E730E0C5E003A922
:10C230002046F9F7EFF920E7B4F92C0029B2401AAB
:10C24000BDF80410401C00EBD070A1EB6001ADF80C
:10C250000410BDF80810BDF80620A1EB6000ADF891
:10C260000800B4F92E002914401A401C00EBD070CD
:10C27000A2EB6000ADF80600B4F92E00401ABDF83C
:10C280000A10401C00EBD070A1EB60003CE707A84F
:10C29000F5F736FE07AA00212046FAF7A0F9E08E4E
:10C2A000ADF81E00208EADF81C00608EADF82000A9
:10C2B000A08EADF8220094F83800BDF80C10C0092B
:10C2C0008DF8300001EB0800ADF83400BDF80E0029
:10C2D000BDF810103844ADF83600A1EB0A00ADF8F7
:10C2E0003800BDF812100DAAA1EB0900ADF83A0014
:10C2F000B16810468846FDF772FE002890D00DA860
:10C30000B060B4F92800B4F92C1090FBF1F201FBF5
:10C310001207B4F92A00B4F92E1090FBF1F201FBD8
:10C320001200BDF90610084400B2ADF816008842AC
:10C3300003DDE18D401AADF81600E18D80B20844AE
:10C34000401E2FE0BDF90410C81900B2ADF814006A
:10C35000884203DDA18D401AADF81400A18D80B292
:10C360000844401E0DE005AA07A93046636AF5F7A8
:10C3700093FDBDF814002844ADF81400BDF8180072
:10C380002844ADF81800BDF91400BDF90810884222
:10C39000E9DBBDF8161028140144ADF81610BDF8FD
:10C3A0001A100844ADF81A00BDF91600BDF90A10BC
:10C3B0008842C7DBC6F80880D1E605A8F6F74EF834
:10C3C00005AA00212046FAF75DF900200090636A73
:10C3D00005A930460D9AF5F7ADFDC0E6A06F02083D
:10C3E0002DE9F0438FB0044604F06DFE0546F9F7E1
:10C3F00075F9064601A8F6F731F801AA0021304682
:10C40000FAF740F9284606F065FD28B19DF82100AD
:10C4100040F001008DF82100204604F01CFE8168E8
:10C4200004460F4606F114020DA8FDF7D8FD0028BA
:10C4300050D00DA8A0600BA9304601F0F3FDA88AEA
:10C44000ADF82400E88AADF82600288BADF8280066
:10C45000BDF82E00ADF82A0009AA1046A168FDF724
:10C46000BEFD4FF000080DF1240978B1A6682846FA
:10C47000C4F8089006F033FD034605F1140201A943
:10C480002046CDF80080F5F755FDA660A88AADF8E6
:10C490002400BDF83200ADF82600288BADF8280046
:10C4A000688BADF82A0009AA1046A168FDF797FD30
:10C4B00078B1A6682846C4F8089006F010FD034637
:10C4C00005F1140201A92046CDF80080F5F732FDF0
:10C4D000A660A7600FB0BDE8F08300002DE9F04F23
:10C4E000CDB0054604F0EFFD0446008E00287CD058
:10C4F000284604F0B0FD4590608C40F0080161844E
:10C50000204643A9F9F786F80026B4F8208026844F
:10C51000608C374640F00801354661842DA8F6F757
:10C5200079FD3BA8F5F79AFF4FF4A0292DAA4946BB
:10C530002046FAF7F7F83BAA49462046FAF7A2F850
:10C54000608C20F008016184A4F82080002120463E
:10C5500007F0F2F94C900021204607F081F94B904A
:10C560000021204607F0A6F94A900021204607F056
:10C57000B9F9499011A84599F8F704FEB248CDE9F8
:10C58000120503A8159025A8CDF87890169050E1D3
:10C590007F1CBFB2606AADA150F827000BF0E7FD29
:10C5A0000028F5D0E06A30F81600C0F30011002929
:10C5B00076D10025C0F3002101B10125C0F3801020
:10C5C00010B145F0800518E0A08EB04215D15FEAA9
:10C5D000886001D545F020055FEA887001D545F0F7
:10C5E00002055FEA487003D500E02AE145F0040542
:10C5F0005FEA087001D545F00805A06A00EBC601A6
:10C6000023A803F0A4FCBDF88C10BDF80C01014474
:10C61000ADF88C10BDF88E20BDF80E110A44ADF8AF
:10C620008E20BDF890201044ADF89000BDF8920027
:10C630000844ADF8920045B32584608C40F00801B1
:10C64000618403A8F6F7E6FC25A8F5F707FF4FF489
:10C65000A02903AA49462046FAF764F825AA4946C4
:10C660002046FAF70FF8A4F82080608C20F008012B
:10C670006184E06A30F81600C0F3C02000289DF8FD
:10C68000B1000ED040F001000DE003A82DA9382222
:10C690000BF0FFFC25A83BA920220BF0FAFCE8E7F1
:10C6A000C3E020F001008DF8B10023A8149011AA76
:10C6B0001A211F96204604F013FD9DF82F00410813
:10C6C000C9063CD520F03E001E308DF82F00B4F98D
:10C6D00014304A99BDF98C2019448A4203D120F0C4
:10C6E00008008DF82F00B4F918204998BDF9901072
:10C6F000101A814205D19DF82F0020F010008DF80E
:10C700002F00B4F916204C98BDF98E1010448142C8
:10C7100005D19DF82F0020F004008DF82F00B4F90A
:10C720001A204B98BDF99210101A814207D19DF83A
:10C730002F008108490061F345008DF82F00BDF8F6
:10C740009210BDF98E00091A491C0FFA81F9A90649
:10C7500008D5E16A31F81610490503D5A0EB0900A8
:10C76000ADF88E0023AA03A94598F6F73FFC25985B
:10C770004890606ABDF9A8B0BDF9A6A050F827009E
:10C78000469043A803F02DFC9DF8B120CDF800A001
:10C79000CDE901025B4647A8489A469908F012FF86
:10C7A00023A803F01EFCBDF91C31BDF88C10C01A83
:10C7B00000EBD07001EB6001ADF88C10BDF8920079
:10C7C000BDF88EC0BDF91E21A0EB0C00401C00B2CC
:10C7D000801A00EBD0700CEB600000B21944ADF889
:10C7E000901081180AB2ADF88E00ADF89220A9061B
:10C7F0000ED5E16A31F81610490509D509EBD97152
:10C80000A0EB6100ADF88E00A2EB6100ADF89200E4
:10C810000020009023AA25A9469B4598F5F78AFB9E
:10C8200011AA1B21204604F05BFC761C7F1CB6B2CB
:10C83000BFB2208EB0423FF6ADAE608C20F0080053
:10C8400060844DB0BDE8F08F686F02080A000000F8
:10C850002DE9F04790B0054604F035FC0446284623
:10C8600004F0F9FB06460BA92046F8F76DFE94F894
:10C8700048000025C10600D50125800601D545F0F8
:10C8800002050021204607F09FF8A0F51C51D13980
:10C8900004D1608C000501D445F0040503A8F5F728
:10C8A000DDFDB4F84400ADF82200B4F84600ADF860
:10C8B00024008DF8295003AA00212046F9F7E2FE52
:10C8C0009DF828004FF0010808B98DF82880E06B2A
:10C8D0000490206C059004994FF6FF7081421ED0A1
:10C8E000059981421BD04FF480292746552249469D
:10C8F0002046F9F778FC024649463846EFF7E1FD55
:10C900000090BDF80000ADF81A00204620224946EC
:10C91000F9F769FC0090BDF80000ADF81C0094F830
:10C92000480041F6FF7A00F00700022801D00328F2
:10C930001AD19DF82800022801D0032814D1BDF98E
:10C940001E10CDE9001A0295BDF92030039A0DA8FA
:10C95000616A08F037FE0BA803F049FBBDF93410FB
:10C96000884201DA8DF8288094F8480004F13007F5
:10C9700000F00700032805D00BA803F00CFBB0F56E
:10C98000806F00DA00270BA90EA8B268FDF727FB1D
:10C9900000287DD094F8480040070BD12046F8F7D6
:10C9A000EFFF404202B200210BA803F033FB608B83
:10C9B000ADF8320094F848000DF1380900F0070096
:10C9C000022813D0032811D000970BAA03A93046E0
:10C9D000636AF5F7AFFAB068C6F80890804694F835
:10C9E000480000F0070003280FD058E0D6F8088070
:10C9F000C6F8089000970BAA03A93046636AF5F7BA
:10CA000099FA4046C6F80880E6E7BDF91E10CDE960
:10CA1000001A0295BDF92030039A0DA8616A08F04A
:10CA2000D1FD0BA803F0E3FABDF93410884219DAFE
:10CA300020221146039804F068FCB4F84410BDF8B5
:10CA4000342000EB400011440844ADF82200B4F853
:10CA50004600ADF8240000970BAA03A93046636A8C
:10CA6000F5F768FA0BA803F096FA0146BDF936000F
:10CA7000814214DAB4F84410ADF822100399B4F8E6
:10CA80004620098910440844ADF82400009700E0CE
:10CA900007E00BAA03A93046636AF5F74BFAC6F81C
:10CAA000088010B0BDE8F0872DE9F04393B0074649
:10CAB00004F0CBFA0546384604F005FB04464FF473
:10CAC0008026152D7ED0182D7DD1384604F0C3FA6E
:10CAD000054603A8F5F7C2FC03AA31462046F9F73C
:10CAE000D1FD0EA9204601F09DFA0EAA10A8A96852
:10CAF000FDF775FA002866D0204601F061FA8146FC
:10CB000006F0E8F928B19DF8290040F001008DF801
:10CB100029002046F9F7B3FC0646484606F0DFF93F
:10CB20000146BDF91E00CDE9000602220292BDF9C0
:10CB300020300DA8039A08F045FD2046F8F793FD34
:10CB4000B4F9161000EBD076B9F9160001EB6601C6
:10CB5000471A4846F8F787FDB90391FBF0F7002123
:10CB6000204606F004FF0399B0F90800B1F9081057
:10CB7000081A00EBD070BDF836104010091A09B23F
:10CB8000ADF83610E28A794302EB660202EBA1317E
:10CB90000E1A0021204606F03AFE8046204600216B
:10CBA0001222F9F720FB0746204600211322F9F74D
:10CBB0001AFBA28A07EB08011144ADF82C10ADF85E
:10CBC0002E6001E023E01FE0218B081AA0EB080093
:10CBD000ADF83000BDF836003044ADF832009DF8B5
:10CBE000290040F002008DF8290010A8AC68A86068
:10CBF000484606F074F90346002000900BAA03A9EA
:10CC00002846F5F797F9AC6013B0BDE8F0833846D5
:10CC100004F021FA05460EA9204601F003FA684601
:10CC2000F6F7F8F96A4631462046F9F77BFD0EAA79
:10CC300069462846F6F7DAF9E6E72DE9F043A1B0B0
:10CC4000054604F040FA0446284604F004FA8146FA
:10CC50000021204606F034FE07460021204606F05B
:10CC600047FE06460021204606F06CFE05460021E0
:10CC7000204606F0FBFDA38AE28AADF87A20218BDC
:10CC8000ADF87C10B4F81AC0891BADF87C103B4499
:10CC9000ACEB0000ADF878305119ADF87E00ADF87E
:10CCA0007A106846F6F7B6F96A464FF40031204626
:10CCB000F9F738FD1EAA69464846F6F797F9204667
:10CCC000F8F7D1FC0646208BA18A401A401C801B35
:10CCD00005B2606A411C06D06843C11700EB1160C1
:10CCE000001207B208E02046F9F7AAF9C0F30000E5
:10CCF00008B12F4600E00027204600211622F9F750
:10CD000072FAC0B2012801D1E81B07B2A08A4FF421
:10CD100040353844ADF870003044ADF87400E08A16
:10CD2000ADF87200608BADF876002946204606F01B
:10CD3000C7FD07462946204606F0DAFD804629460B
:10CD4000204606F0FFFD06462946204606F08EFDE9
:10CD5000BDF87010BDF87420C91BADF8701002EB5F
:10CD60000801ADF87410BDF87210891BADF872108F
:10CD7000BDF876100844ADF876000EA8F6F74AF92B
:10CD80000EAA29462046F9F7CDFC1CAA0EA9484652
:10CD9000F6F72CF921B0BDE8F0832DE9FF4F81B003
:10CDA0000C4680462021DDF838A0F9F787FB0028E3
:10CDB00078D0BAF1030F404621D0F8F7DAFD81466A
:10CDC00005F062FD0546002708F1140000903E467C
:10CDD000BAF1030F3946404614D006F0A1FD824651
:10CDE0000021404606F030FD83464846B9F1010F68
:10CDF00059D002285FD0B9F1030F63D138E0F8F7BA
:10CE0000B1FDDCE706F04AFD83460021404606F00E
:10CE10005DFD82464846B9F1010F19D002281FD0A6
:10CE2000B9F1030F4ED1009803F0C9F8A0EB0B0144
:10CE3000A1EB0A00B8F8141000EBD0720BEB620003
:10CE4000084407B205F1140003F0B9F8A98A23E0F9
:10CE5000B8F81410B5F9146001EB0B0007B231E01B
:10CE6000B8F81810B5F91860A1EB0A0007B229E06C
:10CE7000009803F07EF8A0EB0A01A1EB0B00B8F8D4
:10CE8000161000EBD0720AEB6200084407B205F1FD
:10CE9000140003F06EF8E98A00EBD07001EB60003B
:10CEA00006B20FE030E0B8F81610B5F9166001EBE5
:10CEB0000A0007B206E0B8F81A10B5F91A60A1EB3B
:10CEC0000B0007B2A01E049900B2002910DAB9F1D4
:10CED000000F15D0BE4221DC12E0002C01DDA41CA5
:10CEE00024B2E01704EB9070801005B0BDE8F08F1D
:10CEF0000399002912DAB9F1000F01D0BE420DDB0F
:10CF0000002CEADA0446E8E70498E04202D50498E7
:10CF1000404204B20398001B00D5039C2046E4E77E
:10CF200070B5044605F0A0FC48B1006882680AB1FB
:10CF3000217A9047207E810743D4C0077CD1012607
:10CF40000021606806F038FC00251AE0016899B1FC
:10CF5000017ACA0910D0802904D0227A21F08001F8
:10CF6000914209D14168E160016820468847207EEE
:10CF7000810726D4C0075FD16D1C2946606806F082
:10CF80001BFC08B1002EE1D12146002006F0FEFB7B
:10CF9000051E03D00021606806F00EFC002619E093
:10CFA000016891B1017A0A060FD411B1227A914237
:10CFB0000BD14168E160016820468847207E8107E7
:10CFC00001D5012070BDC00736D1761C314660689E
:10CFD00006F0F2FB10B1012DE2D02FE0012D2DD192
:10CFE0006068416851B3217E490727D4217A2329FB
:10CFF00019D0242917D0A903F9F760FAF0B1207AE3
:10D0000011381C280FD2DFE800F019191919191965
:10D0100019191919190E0E190E0E191919190E0EC2
:10D020000E0E19190E196068406860602046FFF7FF
:10D0300077FF0546012801D0002070BD284670BD4D
:10D040002DE9F04F89B0054600200290039005F0CD
:10D050000BFC00680026B146047E686A0090288BAD
:10D06000A98A08442883688BE98A08446883009861
:10D07000E5E04FF000084FF48077CDF81C80009871
:10D080000EE0002106F088FC40440FFA80F80021F1
:10D09000504606F087FC47433F125046F8F71EFB08
:10D0A0005FEA000A5046ECD1A8690190B8F1000F80
:10D0B00002D1B7F5807F0AD0C8F1000001B24FF469
:10D0C000803090FBF7F207AB01A806F025FDBDF913
:10D0D0000410002900DC4942BDF90600002800DCEC
:10D0E0004042814201DD012601E04FF0010910219B
:10D0F0000098F9F7E3F900287ED0B046CB46CA463F
:10D1000047460098F8F748FBC10700D188468107D9
:10D1100000D40027410701D44FF0000B000701D4D1
:10D120004FF0000A0098F8F72BFC06900098F8F7EB
:10D13000E1FA05900098F8F757FB04900098F8F78B
:10D14000B3FB0699002902DC0599002912DDBBF129
:10D15000000F03D0BDF90610A14207DABAF1000FA3
:10D1600008D0BDF906106242914203DC0099029199
:10D170000C2103910499002901DC002810DDB8F18D
:10D18000000F03D0BDF90410A14205DA47B1BDF983
:10D1900004106242914203DC009902910321039141
:10D1A0000699002901DC4FF0000B0599002901DCEC
:10D1B0004FF0000A0499002901DC4FF00008002814
:10D1C00000DC0027B8F1000F03D0BDF90400A04235
:10D1D00016DA27B1BDF904006142884210DDBBF1C7
:10D1E000000F03D0BDF90600A04209DABAF1000F22
:10D1F00011D0BDF9060000E00DE0614288420ADC72
:10D200000EB1032000E00C2095F8401060F30301FC
:10D2100085F8401016E04FF480710098F9F74EF948
:10D2200036EA00000ED14FF400710098F9F746F984
:10D2300039EA000006D10098F8F750FA009000286B
:10D240007FF417AF029858B195F84000039961F345
:10D25000030085F840000298E86200202883688374
:10D26000029809B0BDE8F08F2DE9FF5F0646F8F798
:10D2700079FBB0F1000A72D041F6FF74002130460C
:10D2800006F00CFB80460021304606F01FFB81466D
:10D290003046F8F735F98346002758E0B068324940
:10D2A000006850F827502846F9F70FF9F0BB4FF403
:10D2B00080512846F9F702F9C0B35046BAF1010F80
:10D2C00005D0022809D0BAF1030F3FD11AE0B18A84
:10D2D000B5F9145001EB080004E0318BB5F9185092
:10D2E000A1EB09000399019A294409B200B29142C5
:10D2F0002CDB029A914229DC081A00B200281CDDBE
:10D3000001461BE005F1140002F059FEA98A00EB6A
:10D31000D07001EB600005B206F1140002F04FFE80
:10D32000A0EB0801A1EB0900B18A00E00EE000EBE0
:10D33000D07208EB62000844D4E74142002C01DDC2
:10D34000224600E06242914200DA04467F1C5F45BB
:10D35000A4D3A4F5F850FF3804D0604200B204B062
:10D36000BDE8F09F0020F9E7010004002DE9FF5F10
:10D370000646F8F7FEFAB0F1000A72D041F6FF74E3
:10D380000021304606F0CCFA80460021304606F0F7
:10D390005BFA81463046F8F7B3F88346002758E039
:10D3A000B0683249006850F827502846F9F78DF8E0
:10D3B000F0BB4FF480512846F9F780F8C0B35046CF
:10D3C000BAF1010F05D0022809D0BAF1030F3FD1FD
:10D3D0001AE0F18AB5F9165001EB080004E0718BF0
:10D3E000B5F91A50A1EB09000399019A294409B231
:10D3F00000B291422CDB029A914229DC081A00B259
:10D4000000281CDD01461BE005F1140002F0B1FD0F
:10D41000E98A00EBD07001EB600005B206F1140060
:10D4200002F0A7FDA0EB0801A1EB0900F18A00E0E2
:10D430000EE000EBD07208EB62000844D4E74142F2
:10D44000002C01DD224600E06242914200DA0446EF
:10D450007F1C5F45A4D3A4F5F850FF3804D0604288
:10D4600000B204B0BDE8F09F0020F9E7010004001D
:10D470002DE9FF4F83B00F46DDE910A4934600214C
:10D48000039806F095FA05460021039806F0D0F9B6
:10D49000F9788A070BD5CB0742F2D17202D09542B8
:10D4A00002D007E0904207D121F00200F870F8782E
:10D4B000C00701D0744800E074480190F878C007B4
:10D4C0000CD072485946814600206080A0802061BF
:10D4D0002080A060E060CDF800B0A2E06A48F1E7EB
:10D4E0000099594506D04FF400013046F8F7E6FFA1
:10D4F00000287DD166493046F8F7E7FF002878D14B
:10D500000021304606F08AF95FEA00085CD0206905
:10D51000401C2061A28802EB0A01A180217DC9077D
:10D5200062D000EB8000800006F042F805001BD0BE
:10D53000E16851B12069401E00EB8000820028465E
:10D540000AF0A7FDE06806F07FF820694FF00001BF
:10D5500000EB800005EB800040F8146CF878C00701
:10D56000304602D0022201E0FEE70522F8F73BFE3A
:10D57000216900B201EB810105EB810121F8100C5A
:10D58000F8784FF00001C007304601D0032200E0D8
:10D590000622F8F728FE216900B201EB810105EBB4
:10D5A000810121F80E0C2069002100EB800005EBC1
:10D5B000800040F8088C206900EB800005EB8000BB
:10D5C00040F8041CE5600FE0019930468847F9787F
:10D5D000890705D5B4F904100A1806998A4226DC91
:10D5E000A28850441044A08030464946884701E054
:10D5F0001DE00BE00146B4F90000814202DD304637
:10D60000494688472080A068401CA060F878400701
:10D6100002D54FF0FF3000E0012000994118009141
:10D6200005D40398F7F75AFF061E7FF459AFB4F9F3
:10D630000400002802DDA0EB0A00A080206908B1E8
:10D64000069801E0B4F904006080CEB10098584516
:10D6500016D103996A468968096851F82050F8780C
:10D66000C0F38001039800F0AEFC4DB12846494656
:10D670008847208001992846884760800120A06063
:10D68000009807B0BDE8F08F7F6401086756010875
:10D69000010006002DE9F04FB34D93B00446002180
:10D6A0006A88F8F7A0FD9DF81710421C62F300018C
:10D6B000820862F34101C00860F382018DF81710FF
:10D6C00020460021AA88F8F78EFD8DF81400204628
:10D6D0000021EA88F8F787FD8DF815002046002123
:10D6E0002A89F8F780FD8DF816000021204606F003
:10D6F0007CF8012800D0002083469DF817004FF0E9
:10D700000001C00720460CD006F0F8F806469DF848
:10D7100017004FF00001C007204605D006F0ACF816
:10D7200004E006F0A9F8F1E706F0E8F881469DF874
:10D730001700C007204602D0F7F750FF01E0F7F7C7
:10D7400031FF0C90204600213222F8F74CFD0546AF
:10D75000204600211022F8F746FDE18A28444718A8
:10D760002046F8F71BF9381AADF83400204600219E
:10D770001222F8F738FDA18A284445182046F8F708
:10D7800006F9281AADF83C009DF817009DF81680A0
:10D79000C00701D00DAD00E00FAD0021204606F01E
:10D7A00007F911900021204606F042F810909DF8EC
:10D7B0001700C10709D01099A1F51C52D13A02D126
:10D7C000618C490509D5C10709D11199A1F51C52F0
:10D7D000D13A04D1618C090501D44FF00008BBF1A6
:10D7E000000F0CD0C0070AD1B8F1000F03D0B8F178
:10D7F000010F02D003E0012000E000208046002756
:10D80000ADF83870BA46B8F1000F3AD09DF817005D
:10D81000400703D5A0684268521E13E0002211E0C1
:10D8200000200B9006A8CDE9009005A920460C9B8E
:10D83000FFF71EFEBDF81810BA1911440FB20AF115
:10D84000010A0246A0684068904201DD002AE7DA3A
:10D85000BAF1000F01D0B81B07B29DF81700C0073E
:10D86000204602D0F7F79EFE01E0F7F7B7FE0EA9BB
:10D87000CDE9005101460FFA8AF33A46404608F0D6
:10D8800057F89DF81710480703D5A0684068401E58
:10D8900000E000208046BBF1000F04D0C80702D191
:10D8A0002888384428800DF1180AA068416841454D
:10D8B00046DDB8F1000F43DB01200B90CDE9009A63
:10D8C000424605A920460C9BFFF7D2FD0746BBF157
:10D8D000000F08D09DF81700C00704D12888BDF8B4
:10D8E0001810401A2880BDF934300C9A02A8019310
:10D8F00080E80406BDF93C0000903B46424605A97D
:10D900002046FEF7F7F8B846099805F09DFE00207E
:10D910000990BBF1000F03D09DF81700C00709D094
:10D920002888BDF818100844BDF838103144084460
:10D930002880BAE7BDF8381028883144401AF7E744
:10D94000119942F2D170814202D01099814202D1E4
:10D950002046F9F743FB00222B21204603F0C0FBB1
:10D9600013B0BDE8F08F00008C5200202DE9F74F76
:10D970000546007F93464FF0000AC00760D14FF084
:10D980000108EC680026C1467CB9287FC0F3C000BE
:10D99000401E304254D1B9F1000F51D001992846B0
:10D9A00088474FF000080446C1460EB9261E47D0EE
:10D9B000B8F1000F06D0214628465A469047044643
:10D9C000B0423DD04FF00108002CDDD02068F8F7C0
:10D9D00037FB0006D8D427681FE001213846F8F746
:10D9E0006DFDB0B12FB101213846F8F767FD002871
:10D9F000CAD1E868A04223D0B0B1284600F024FA8A
:10DA00000246E8680F21006803F06AFB012817D17D
:10DA100006E03846F7F762FE0746002FDDD1E8E75B
:10DA2000E8680068F8F7DCFF2846EC6000F00CFAC4
:10DA30000246E8680E21006803F052FB012802D07C
:10DA40005046BDE8FE8FE8680068F8F7C9FF29690D
:10DA500009B1284688470120F3E770B5426B818CF5
:10DA600012F0060F06D0C2F34102022A04D0012AA6
:10DA700005D022E0008D00E0C08C08441CE0B0F925
:10DA80002C40468DA2B2B24202D202F5B47214B258
:10DA9000B0F92830C58C9AB2AA4202D202F5B4700D
:10DAA00003B2301900EBD0704010854201DA6818DB
:10DAB00002E0834203DD501881B208B270BD084411
:10DAC000FAE72DE9F34F87B0074680466946F7F736
:10DAD000A1FD3846F8F7D3FC03903846F7F7C3FDAD
:10DAE00006900021384605F0E5FE814600213846C3
:10DAF00005F0F8FE05460021384605F01DFF0646F4
:10DB00000021384605F0ACFE02900021384605F0B1
:10DB100001FF04460021384605F0BAFE04F0010179
:10DB200004EBD47201EB620100F0010200EBD07053
:10DB300002EB6000491C401C09B200B20B2900DB5B
:10DB40000B218B460B2800DB0B2082460B2D00DBC4
:10DB50000B250B2E00DB0B2602980B2801DA07465B
:10DB600000E00B27002469E0D8F8280000EBC4018E
:10DB700004A802F0ECF9BDF910004946484513DC51
:10DB8000BDF90020B9F10B0F00DB0B21511A08443D
:10DB9000ADF81000BDF91200B0421EDCBDF9022044
:10DBA0000B2E07DA314606E0BDF80020A2EB0A0191
:10DBB0000844EDE70B21511A08440399ADF812000F
:10DBC000BDF91400491B891E88421EDBBDF90010F7
:10DBD0000B2D014407DA284606E0BDF80220A2EB2F
:10DBE0000B010844E9E70B2008440699ADF814003E
:10DBF000BDF91600C91B891E884217DBBDF902104A
